:020000040000FA
:040000006FD00400B9
:101000006F10C04F00000000000000009020002082
:10101000DC270020A9BDF9F5A02800200000000071
:1010200000000000A0280020902000200000000008
:101030000000000090200020000000009020002010
:101040000000000090200020902000209229002025
:1010500090200020902000206C340020A82900203F
:10106000000000009020002090200020382900205F
:1010700090200020062900209020002090200020B1
:101080009020002090200020902000209020002020
:101090009020002001A04111B7170040985F3AC688
:1010A000945F3247E39CE6FE324541018280411164
:1010B000814601468145114506C697100000E7802C
:1010C000C0C3B727004011472383E780B7F700E08C
:1010D00003A707D16D9B23A8E7D003A707D15D9B8A
:1010E00023A8E7D07300501001000100B240410175
:1010F00082800111814601468145114506CE971037
:101100000000E78080BFB727004011472383E780B6
:10111000B717004083C6E70203C5E704130780083A
:1011200093F6C60F1365350093E6160073360780F5
:101130001376860832C001000100930570052380F4
:10114000B704130680FA2380C7040100010023823C
:101150000702238007040248732808800100010069
:10116000733807801378880842C201000100238089
:10117000B7042380C704010001002387D702238717
:10118000A704238007049246F3A60680010001000D
:10119000F336078093F6860836C4010001002380E9
:1011A000B7042380C7040100010083C6B70493E697
:1011B0000602A385D70423800704A246F3A606806F
:1011C00001000100B7F600E003A506D11365450054
:1011D00023A8A6D003A506D15D9923A8A6D07300A5
:1011E00050100100010073370780137787083AC653
:1011F000010001002380B7042380C704010001001F
:1012000003C7B7041377F70DA385E704238007040A
:10121000B247F3A7078001000100F2400561828018
:101220003971B7F5070022DC81462A843010E105C8
:10123000194506DE02D42316010297100000E7804C
:10124000C0ABB717004083C6E7041307800893E6D6
:101250003600733607801376860832C40100010019
:10126000930570052380B704130680FA2380C70412
:101270000100010023820702238007042245732511
:1012800005800100010073350780137585082AC6A3
:10129000010001002380B7042380C704010001007E
:1012A0002387D70423800704B246F3A606800100F3
:1012B0000100F336078093F6860836C80100010066
:1012C0002380B7042380C7040100010003D507026F
:1012D000F176FD16E98E2390D70223800704C246DB
:1012E000F3A606800100010037F500E0832605D152
:1012F00093E646002328D5D083D6070265751105ED
:1013000093F60660C18EC98EC206C182733507800E
:10131000137585082ACA010001002380B7042380C1
:10132000C7040100010003C5F70013650504A38786
:10133000A7002390D70223800704D246F3A6068095
:10134000010001001165618D1DE973370780137776
:1013500087083ACC010001002380B7042380C7042A
:101360000100010003C7B70413670702A385E70460
:1013700023800704E247F3A707800100010037F745
:1013800000E0832707D1DD9B2328F7D0730050109E
:101390000100010013078008F337078093F78708DF
:1013A0003ECE01000100B717004093057005238071
:1013B000B704130680FA2380C7040100010083D616
:1013C0000702C606C5822390D70223800704F2468F
:1013D000F3A6068001000100F336078093F6860825
:1013E00036D0010001002380B7042380C704010028
:1013F000010003D80702F176FD16B3F6060123902B
:10140000D702238007048256F3A60680010001005C
:1014100021E173370780137787083AD20100010072
:101420002380B7042380C7040100010003C7B70469
:101430001377F70DA385E704238007049257F3A7DA
:10144000078001000100514597000000E780E0415E
:10145000F250625421618280397152D481462A8AC5
:1014600001468145114522DC26DA06DE4AD84ED6F1
:101470003714004097100000E78020888347E4027B
:101480000347E4049304800893F7C70F13673700FA
:1014900093E71700F3B6048093F6860836C601007A
:1014A00001009309700523003405130980FA230015
:1014B0002405010001002302040223000404B246B3
:1014C000F3A6068001000100F3B6048093F68608B7
:1014D00036C8010001002300340523002405010063
:1014E00001002307F4022307E40423000404C24795
:1014F000F3A70780010001001305500297000000C8
:10150000E780400EB7F700E003A707D11367470055
:1015100023A8E7D073B70480137787083ACA01007D
:1015200001002300340523002405010001000347C6
:10153000F40013670704A307E400230004045247E0
:10154000732707800100010073B7048013778708B1
:101550003ACC0100010023003405230024050100DA
:1015600001002167336AEA002310440323000404C6
:101570006247732707800100010003A707D15D9B25
:1015800023A8E7D0730050100100010081460146F6
:101590008145114597000000E7802076F3B4048070
:1015A00093F4840826CE01000100230034052300B3
:1015B0002405010001008347640493E71700230317
:1015C000F40423000404F247F3A70780010001009C
:1015D000F2506254D2544259B259225A2161828047
:1015E000011113078008F337078093F787083EC27D
:1015F00001000100B7170040930570052380B70470
:10160000130680FA2380C7040100010083C6B704D3
:1016100093F6F60DA385D704238007049246F3A61C
:1016200006800100010093760502D5CEF3360780CF
:1016300093F6860836C4010001002380B704238096
:10164000C70401000100B70614007D89558D88C7C5
:10165000010001000100010023800704A246F3A657
:1016600006800100010073370780137787083AC6A8
:10167000010001002380B7042380C704010001009A
:10168000010001003727004093061005A303D7800F
:1016900023800704B247F3A70780010001009307E6
:1016A0008008F3B7078093F787083ECE010001005A
:1016B000B7170040130770052380E704130780FA6B
:1016C0002380E7040100010003C7B704136707087C
:1016D000A385E70423800704F247F3A707800100EE
:1016E00001000561828093760504BDC6F33607804C
:1016F00093F6860836C8010001002380B7042380D2
:10170000C70401000100B7061400938606047D8912
:10171000558D88C7010001000100010023800704E6
:10172000C246F3A6068001000100733707801377D5
:1017300087083ACA010001002380B7042380C70448
:10174000010001003727004093062005A303D7803E
:1017500023800704D24781B7733707801377870840
:101760003ACC010001002380B7042380C7040100A4
:10177000010098471367070C98C723800704E247C6
:1017800019BF0111814601468145114506CE9700DA
:101790000000E780805693078008F3B7078093F72F
:1017A00087083EC601000100B71700401307700507
:1017B0002380E704130780FA2380E7040100010077
:1017C00003C76704136717002383E7042380070414
:1017D000B247F3A7078001000100F2400561828053
:1017E0004111814601468145114597000000E7807F
:1017F000C05013078008F337078093F787083EC46B
:1018000001000100B7170040130670052380C704CC
:10181000930680FA2380D70401000100FD5523962A
:10182000B70223800704A245F3A50580010001004B
:1018300073370780137787083AC6010001002380B9
:10184000C7042380D7040100010003C7670413679E
:1018500017002383E70423800704B247F3A7078018
:101860000100010001A0BD473305F50201007D150F
:1018700075FD8280411122C426C206C6AA84014495
:1018800063179400B24022449244410182800504CF
:101890001305803E420497000000E78000FD418070
:1018A000C5B700009305000273A045808245739080
:1018B000153492402242B2424243D2436244F2443F
:1018C000025592552256B2564257D2576258F25894
:1018D00006499649264AB64A464BD64B664CF64CC4
:1018E000065D965D265EB65E465FD65F0961730053
:1018F00020304111B7170040985F3AC6945F3247D5
:10190000E39CE6FE324541018280B7170040130791
:1019100000032388E7028547171700002324F744B4
:1019200073002030411122C406C63704002097609E
:1019300000E0E780A0031C408297D5BF3737004006
:10194000834747009146BD8B6389D70099466394CE
:10195000D70083475740730020309736000083C676
:1019600026ED93871600173600002303F6EC034795
:101970008700973700009387A7DBB6972380E7009F
:10198000B7E70400BC4F0946894517150000034519
:10199000A5F58297C9B7371700408357E709C18B70
:1019A00081C7C147231FF70873002030B787004065
:1019B00003C76700098B6309071003C77700930605
:1019C000000313770703630DD70817380000034897
:1019D000B82117360000130666200547B306060136
:1019E0002380E60083C57700173700001307871FA1
:1019F000429793F5F50F2300B70003C5870097358D
:101A000000009385E51DC2951375F50F2380A50091
:101A10000347070089451377F703630CB70C63E7A7
:101A2000E50A6306071A8545630CB712973700006D
:101A300083C7971B3307F600034707001377F70F99
:101A400019CB850793F7F70F0D476363F71A17371D
:101A50000000A30BF718B787004009472383E7006E
:101A6000B787004083C77700E207E18763DE07049A
:101A70009737000083C7571717370000130707165B
:101A80003E9785462300D7001737000013078715B8
:101A90003E97930600032300D70017370000130773
:101AA00027143E97A14685072300D70093F7F70F29
:101AB0000D476364F71417370000A307F712B787C1
:101AC000004009472383E70073002030930610028B
:101AD0006300D70E930620026305D7069306000223
:101AE000E316D7F403C727021377C70F136727003E
:101AF000D5A803C767001377070465CB03C7A70200
:101B000017380000130808EF17350000130545E6E5
:101B1000134707082385E70203C7A7021377370F88
:101B2000136787002385E702814713070004B30585
:101B3000F5008C41B306F80091078CC2E399E7FEEB
:101B4000F5B503C7A702134707042385E70203C7B8
:101B5000A7021377C70F136727002385E702F9B59C
:101B600003C767001377070449C303C76702173821
:101B700000001308E8DB17350000130525D31347D1
:101B800007082383E70203C767021377370F13673A
:101B900087002383E702814713070004B305F5009C
:101BA0008C41B306F80091078CC2E399E7FEBDBDF6
:101BB00003C76702134707042383E70203C76702CB
:101BC0001377C70F136727002383E70285B503C781
:101BD00067001377070411CB03C727021377370F6A
:101BE000136787002381E70291B5238006003DBD7E
:101BF00097370000A38A07FEB9BD97370000A38579
:101C000007FE75BD2303048015472303E48001000C
:101C10002302A480828083076480E3CE07FE23032F
:101C20000480828083076480E3CE07FE03454480FE
:101C3000828083076480E3CE07FE2302A480828033
:101C4000411126C44AC24EC006C61377F50BAD47F4
:101C5000AA892E899544630CF70019459700000066
:101C6000E78080FA97000000E78020FB8D444E85D6
:101C700097000000E78040F9FD59FD146398340196
:101C8000B240A244124982494101828013550901A0
:101C90001375F50F97000000E780E0F92209F1BF06
:101CA000011126CC06CEB704080097000000E7809B
:101CB000C0F6154597000000E78000F5970000008A
:101CC000E78080F697000000E78000F62AC69700BC
:101CD0000000E78080F432459377150089EB1365A7
:101CE00015001375F50FF240E24405618280FD1482
:101CF000E9F00145CDBF397126DC4ADA4ED852D61B
:101D000056D45AD25ED006DE62CE66CCB7E700E08B
:101D10007D5783AA070022C603AA470023A0E7181D
:101D200023A2E718B7170040130770052380E704C4
:101D3000130780FA2380E70483C74704930B75FFDA
:101D4000B684E20793FBFB0F8546AA892E8B328966
:101D500037240040E187015763FA76016308D50014
:101D60008946130700026313D5000157D98F93F7F3
:101D7000F70FB71C00402382FC0411472303E480C3
:101D80001305F00F97000000E78000E8094C97006A
:101D90000000E78080E863657C15B7050700DA95E9
:101DA00037870700795563FEE504B3879500636ABA
:101DB000F704370B0800A94733EB65016395F90871
:101DC00081E8814497000000E78020E5268515A87A
:101DD000DA85094597000000E780C0E6050903455C
:101DE000F9FFFD14050B97000000E780C0E481C4F3
:101DF0009377FB0FE5F797000000E780A0EA69F111
:101E00007D55B7170040130770052380E7041307BB
:101E100080FA2380E70403C74704418B2382E70449
:101E2000F250B7E700E023A0571123A24711E25474
:101E300032445259C259325AA25A125B825B724CD6
:101E4000E24C21618280A547639BF90685691309ED
:101E5000F00FB3069900B3742B01B6941349F9FF40
:101E6000B3749900856B33796901416B9387F9FFEE
:101E7000B3F7270199E363FC340193D94900C147C3
:101E8000E3E637FF3DBF0569C1697D19D9B7130581
:101E9000800D6388690113050002638479011305CD
:101EA0001008CA8597000000E780C0D9970000009D
:101EB000E78040DF31D54E99B38434416DBFDA8578
:101EC0002D4597000000E780E0D7CA94E30B99EE18
:101ED000050997000000E78020D5A30FA9FEFDB7F4
:101EE0009387F9FF93F7F70F636DFC0C83C71C040E
:101EF000130730086315F706370708006361EB0620
:101F0000B3079B00B706100063FBD704334BEB000D
:101F100089476399F9068980D549E38404EADA851B
:101F2000094597000000E780E0D111090327C9FFA8
:101F300091472320E48003076480E34E07FE2303D8
:101F40003481FD17EDFBFD14110B81C49377FB0F5A
:101F5000E9FF97000000E780E0D461F155B5B717BD
:101F6000004003C75704B70708001377070219E3B7
:101F7000B78707007955E376FBE833079B00E3F961
:101F8000E7F841B58547E380F9F0DA852D459700FC
:101F90000000E78020CB9389F4FFE38404E29700FC
:101FA0000000E78060C893F7390091EB8326048036
:101FB0000327090093074900E396E6E03E89CE84B3
:101FC000D9BFB5476399F9001305900B970000003E
:101FD000E78080C3FDB3B1471305B00AE388F9FE7B
:101FE00099476397F904B7050800B365BB002D4511
:101FF00097000000E78000C581448D4BA149970000
:102000000000E78060C26396740183270480232068
:10201000F9008504E39534FF8327048013172B010F
:10202000635507002312F90069BB2322F90051BB55
:102030009D47639FF90281451305B0049700000096
:10204000E78040C0BD442320090023220900FD5938
:1020500097000000E78040BD93F77400CA9703C75C
:102060000700FD14398D2380A700E39334FF91BB53
:10207000A1476397F90697000000E780A0C281445A
:10208000630D0B008D479304C0036308FB009304AA
:10209000000563048B01930440041375C507E30234
:1020A00095D2194597000000E78000B69700000020
:1020B000E780A0B6054597000000E780E0B42685DC
:1020C00097000000E78020B7094597000000E780EF
:1020D00080B697000000E780E0BCE31405CE0DB3A6
:1020E0009147639FF9001305600697000000E780A1
:1020F000A0B197000000E78040B213059009F9B540
:10210000E38109CCF1547DB9BD6601471736000063
:102110001306C6CA938606A685458347060093F72D
:10212000F70F91C382800507E3F9E6FE97370000B9
:102130002386B7C8DDB77D166206618693178601D0
:10214000E18763D407000145828093172600330797
:10215000F500AE9718439C4363E7E7007D16E37FE5
:10216000F7FC7D55828005458280FD15E205E185FD
:1021700013978501618793F7F50F63480700FD15F5
:10218000139725002A97584365D7138517006205D2
:10219000618582803308B5021C4283A80600B335EE
:1021A000B502C29733B50701AE9846958548636777
:1021B000B5006394A50063E3070181480C43C6950D
:1021C0000CC388C21CC28280814713978701618734
:1021D0006343B7008280139727002A9723200700C4
:1021E0008507E5B78147014793968701E18663C577
:1021F000B60013351700828093962700AA96944262
:102200008507558FD5B793D755408A07AA979C4322
:1022100005453315B5007D8D828017F3FFDFE7029A
:10222000833D2A8497000000E78060F405C593177A
:1022300025003E940327C4FF814711EB7D15160549
:102240003E954205418517F3FFDF6700033D058397
:102250008507E5B70145C5BF8147139787016187AA
:102260006343C700828013972700B386E50094423A
:102270002A97850714C3D5B77D1662066186014784
:1022800093178601E18763D5070013351700828015
:1022900093172600B306F500AE9794429C437D1633
:1022A000B58F5D8FF1BF8A05AA9501476363B500BD
:1022B000828083A6C5FFF11593D71600D98F9CC1E4
:1022C0001397F601E5B72A830148014701456343A7
:1022D000D7008280B387050183A80700B3070601F2
:1022E0009C43C697AA976384F80033B51701050786
:1022F000B3080301620723A0F80061871108C1BF7A
:102300002A8301478147014563C3D7008280338810
:10231000E50083280800330EE600032E0E00338804
:10232000A8403308C8416384080133B50801850714
:10233000B308E300E20723A00801E1871107E9B72A
:1023400017F3FFDFE702232B0111B286B2842E863A
:10235000AA850A8597000000E780C0FA2A84A6852E
:102360000A8597000000E78020E8333480000604E7
:1023700013351500018D056117F3FFDF6700E329B1
:1023800017F3FFDFE702A3244111AA89AE8A328B3B
:10239000B68402C202C402C60144131C8401135C49
:1023A0008C4163499C02939B1400FD1B0549138CCF
:1023B000F4FFF15C330489016204618463407407B3
:1023C00092478E04CE9423AEF4FE410117F3FFDF53
:1023D0006700632313192400B30B2B01014A9317E1
:1023E0002A00D69783A50B0088437800340050005C
:1023F00097000000E78040DA050A93178A01E18719
:10240000F11BE35EFCFC92474E9905042320F90082
:10241000A2473EC2B24702C63EC441B7131A890161
:10242000135A8A41131D240093178A01E18763CF51
:10243000970092470A044E941CC0A24705091379DD
:10244000F90F3EC2B24702C63EC4ADB7B3079A0306
:1024500013152A0056950841780034005000050AEB
:10246000EA97DA978C4397000000E780E0D26DBFCF
:10247000197106C212C416C61AC81ECA22CC26CEAC
:102480002AD02ED232D436D63AD83EDA42DC46DED4
:10249000CAC0CEC2D2C4D6C6DAC8DECAE2CCE6CE44
:1024A000EAD0EED2F2D4F6D6FAD8FEDA97150000CA
:1024B0009385C58A8841E700050092402242B242D6
:1024C0004243D2436244F244025592552256B256D8
:1024D0004257D2576258F25806499649264AB64A98
:1024E000464BD64B664CF64C065D965D265EB65E58
:1024F000465FD65F096173002030000097210020FD
:10250000938141B0174100201301C12F17F5FFFF40
:10251000130585AF970500209385C5AE17160020DB
:102520001306C6FD63FAC5008322050023A05500EB
:1025300011059105E3EAC5FE1705020013054503E1
:1025400097150020938585FB171600201306066556
:1025500063FAC5008322050023A0550011059105EB
:10256000E3EAC5FE171500201305456397450020D3
:102570009385C5D06377B500232005001105E36D71
:10258000B5FEFD42739002BC8D4273904280B7222B
:102590000000938282887390023097020020938219
:1025A00062A693E2320073905230975200009382F9
:1025B00062B4739012346FB0B42473002030397158
:1025C00001436EC619A0397141536AC866CA62CC0C
:1025D0005ECE19A0397101535AD056D252D44ED67C
:1025E0004AD826DA22DC06DE3301614082824111BC
:1025F0004AC026C222C406C68282B24D4101024DA3
:10260000924C224CB24B4101024B924A224AB249AF
:102610004101024992442244B240410182803D433B
:102620002A876373C3029377F700BDEFADE5937616
:1026300006FF3D8ABA960CC34CC30CC74CC7410772
:10264000E36BD7FE11E28280B306C3408A0697028D
:10265000000096966780A6002307B700A306B70080
:102660002306B700A305B7002305B700A304B700EE
:102670002304B700A303B7002303B700A302B700E6
:102680002302B700A301B7002301B700A300B700DE
:102690002300B700828093F5F50F93968500D58DC2
:1026A00093960501D58D61B7939627009702000098
:1026B00096968682E78086FA9680C1171D8F3E9691
:1026C000E374C3F8A5B73367B500FD530D8B79E705
:1026D000B7877F7F9387F7F710419441B372F60075
:1026E0003363F600BE92B3E262006397720C631824
:1026F000D6065041D441B372F6003363F600BE9261
:10270000B3E262006398720A631BD60410459445D5
:10271000B372F6003363F600BE92B3E262006391D7
:10272000720A631ED6025045D445B372F600336375
:10273000F600BE92B3E26200639A72086311D60299
:1027400010499449B372F6003363F600BE92B3E2C7
:102750006200639372085105D105E30FD6F6131793
:10276000060193970601631CF7001357060193D7E0
:1027700006013305F7409375F50F91E98280418397
:10278000C1833305F7409375F50F91E1828013778C
:10279000F70F93F7F70F3305F740828003460500E4
:1027A00083C60500050585056313D60065FA330564
:1027B000D640828011059105E312D6FE0145828044
:1027C0002105A105E31CD6FC014582803105B10538
:1027D000E316D6FC014582804105C105E310D6FC15
:1027E00001458280B717004003C777051377E70FCD
:1027F000A38BE704130700F8A38DE7043D47238C60
:10280000E70413075003A38CE70403C7A705137756
:10281000D70F238DE7048280B717004003C7E70472
:102820000D8941111377C70F498F93068008F3B6BE
:10283000068093F6860836C60100010093067005EF
:102840002380D704930680FA2380D7040100010077
:102850002387E70423800704B247F3A7078001001A
:10286000010041018280B717004003C7E7020D89CC
:1028700041111377C70F498F93068008F3B606807E
:1028800093F6860836C60100010093067005238082
:10289000D704930680FA2380D70401000100238720
:1028A000E70223800704B247F3A707800100010075
:1028B0004101828041112A83014E930E407E130F05
:1028C0000019930F400663E56E1293080019130375
:1028D0004006B3781503854E0D4FA14F3373650243
:1028E0000D891335150063EFBE121308F6FF794604
:1028F00072984208135808013307C70213D617000D
:10290000BE0732976146B3F6C60213068070B386DF
:10291000C6023697A166F58F42075D8FB716004055
:1029200083C7F60293F70708A303F100034671007B
:1029300083C7F60293F70708E394C7FE8347710045
:10294000B716004093F7F70F6388071293078008C4
:10295000F3B7078093F787083EC401000100B7175B
:102960000040930670052380D704930680FA2380E5
:10297000D7040100010023AA070383C6170393E6C7
:102980000608A388D70223800704A247F3A707807D
:10299000010001001166B71700407D16D45BC85FC7
:1029A00093854703A98EF18EF5FA93068008F3B656
:1029B000068093F6860836C601000100930670056E
:1029C0002380D704930680FA2380D70401000100F6
:1029D00098C103C7170313670704A388E70223807E
:1029E0000704B247F3A7078001000100410182807C
:1029F0007D133368E3039308E016630E0800336821
:102A0000F3039308D016630808009378330093B853
:102A100018009388D81633081E01131E0801135E90
:102A20000E0155B56393E503054863860800014828
:102A3000630303002A8871087298FD15131E0801AC
:102A4000C205135E0E01C18179BD13F8150063F450
:102A5000BF007908D5B713381800E5BF83C7F60261
:102A600093F70708A303F1000346710083C7F6023A
:102A700093F70708E394C7FE8347710093F7F70FB6
:102A8000F1DFE9B531714AD966CB06DF22DD26DBFD
:102A90004ED752D556D35AD15ECF62CD6AC96EC7D2
:102AA000AA8C02D897100000E780C0B92A89930742
:102AB0008008F3B7078093F787083EDA010001002A
:102AC000B7170040130770052380E704130780FA47
:102AD0002380E7040100010003C7F7021377770F93
:102AE000A387E70203C7F70213678700A387E702FC
:102AF00023800704D257F3A7078001000100054592
:102B000097000000E78060D6130780C13347E902D1
:102B1000116A93070AE893065002BD69930BA0045B
:102B2000814A014B13048008930470057D1AB34752
:102B3000F9023307D7023EC0FD873ECC938709A632
:102B40009309803E3347F7023AC27D873AC4334740
:102B500039038549B399990193D93940B306D7020E
:102B6000B30B7703B3C6F602B3CBFB0236C6FD86C2
:102B700036C893D6FB4136CEB7460F00938606245F
:102B80003349D9028566938606FAB3969601B389CE
:102B9000E902130760553309D90293060010B3897F
:102BA000E9023349D902B3C9F9029316390036CA8A
:102BB00037190040FD8636D0930D090493D7F941AB
:102BC0003ED2F336048093F6860836DC010001001D
:102BD000930770052380FD00930680FA2380DD00B3
:102BE000010001008346390593F6860FA309D90435
:102BF0008346390593E61600A309D90423800D0006
:102C0000E256F3A6068001000100130C80FA116D54
:102C1000F336048093F6860836DE01000100930740
:102C200070052380FD0023808D0101000100834693
:102C30003905216693E60602A309D90483560905DE
:102C4000B3E6A6012318D90483560905D18E2318AB
:102C5000D90423800D00F256F3A60680010001007E
:102C60008346390593F606026381061A0346390541
:102C7000218A6DDE081897100000E780A0A0733647
:102C8000048013768608B2C20100010023809D00F3
:102C900023808D0101000100B717004003C63705EE
:102CA0001376F60DA389C70403C63705136606021B
:102CB000A389C704835609052166B3E6A601231834
:102CC000D90483560905D18E2318D90423800D0019
:102CD0009646F3A60680010001008346390593F667
:102CE0000602638B061483463905A18AEDFE97F030
:102CF000FF1FE780403AAA8636D497F0FF1FE7808F
:102D00008039A256E30AD5FE835609054255B3E63B
:102D1000A6012318D90497100000E7806098834625
:102D20003905A18AEDDE0356090583462905824748
:102D30003376CA00B306DA0293D5F641B296B38869
:102D4000F640E24733B8C6002E983308F840A24751
:102D5000B3B616013308D84063C70701631DF800F6
:102D6000924763FA1701C247634FF80E6395070154
:102D7000B24763EAF80E894663E9660FF246931597
:102D8000180013D3F8015E8613951800B365B300DD
:102D900042D646D497C00100E780409C3258050BCC
:102DA000137BFB0F63470001631A0838A25863873F
:102DB000083813081500B336A800B69513D6F501E8
:102DC0003298B336C800AE9613581800FE06B3E624
:102DD00006017336048013768608B2C6010001002E
:102DE00023809D0023808D01010001000356C9024C
:102DF000B296C206C1822316D90223800D00B646C0
:102E0000F3A606800100010021B5F336048093F695
:102E10008608B6C00100010023809D0023808D013B
:102E2000010001008346390593E60602A309D9048F
:102E300023800D0086460DB5F336048093F6860890
:102E4000B6C40100010023809D0023808D01010094
:102E500001008346390593E60602A309D9042380BD
:102E60000D00A646BDB5E30B0BF0F336048093F6D8
:102E70008608B6C801000100930680FA23809D00F1
:102E80002380DD00010001008346390593F5FC0F26
:102E900093F6860FA309D90483463905CD8EA3097D
:102EA000D90423800D00C646F3A606800100010068
:102EB000130580FA03463905930639051D8A631CFC
:102EC00096297336048013768608B2CC010001007F
:102ED000130680FA23809D002380CD0001000100AD
:102EE00003C606001376F60D2380C60003C606004F
:102EF000136606022380C600835609051166D18E2B
:102F00002318D904835609052166D18E2318D904C4
:102F100023800D00E646F3A606800100010013069B
:102F200080FA8346390593F60602638006268346B7
:102F30003905130C3905A18AFDDA0818970000003D
:102F4000E7804074F336048093F68608B6D001001B
:102F50000100930680FA23809D002380DD0001009C
:102F6000010083460C00116693F6F60D2300DC0089
:102F700083460C0093E606022300DC008356090515
:102F8000D18E2318D904835609052166D18E2318C2
:102F9000D90423800D008656F3A6068001000100A7
:102FA000130680FA8346390593F60602638A0620E3
:102FB00083463905A18AEDFE97F0FF1FE780A00D3B
:102FC0002A8C97F0FF1FE780000DE30C85FF8356E6
:102FD000090511664255D18E2318D90497000000C7
:102FE000E780006C8346390513063905A18AFDDAAE
:102FF000F336048093F68608B6D4010001009306E8
:1030000080FA23809D002380DD00010001008346BB
:10301000060093F6F60D2300D60023800D00A65679
:10302000F3A6068001000100835609050346290521
:10303000D247B376DA003306CA021305800C9355E3
:10304000F6413696330DF6408257333CD6002E9C1F
:103050003336A601330CFC40330CCC4033088503D7
:1030600092564E86B335A5033305A503C29597B096
:103070000100E780A06E63468001631E0C16630C9E
:103080000D16130615003335A6002E959356F5013F
:103090003696B335D600AA959396F50105828585B7
:1030A000D18E6346B000639D051A638B061A0356E2
:1030B000C90215823305D6003336C500B295634880
:1030C000B000639105241306F00F637DA6228946A4
:1030D00063F3561593078008F3B7078093F78708C3
:1030E000BED601000100371700409307700523008A
:1030F000F704930780FA2300F704010001008356C8
:10310000C70289678117D58FC207C1832316F702CB
:1031100023000704B657F3A7078001000100FA5007
:103120006A54DA544A59BA592A5A9A5A0A5BFA4BDB
:103130006A4CDA4C4A4DBA4D296182801308F5FF7A
:103140003335A800FD152E951356F5013298B33688
:10315000C800AA9695B9F336048093F68608B6CAD5
:103160000100010023809D002380AD0001000100CB
:1031700083463905CD8EA309D90423800D00D64698
:10318000F3A606800100010035B3F336048093F600
:103190008608B6CE0100010023809D002380CD006B
:1031A000010001008346390593E60602A309D9040C
:1031B00023800D00F646F3A606800100010095B3BA
:1031C000F336048093F68608B6D20100010023800E
:1031D0009D002380CD00010001008346390593E660
:1031E0000602A309D90423800D009656F3A6068093
:1031F0000100010045BB9306F5FF33B5A600FD15A0
:103200002E959355F501AE96B3B5B600AA951396D3
:10321000F501858269B5F336048093F68608B6D841
:1032200001000100930680FA23809D002380DD00C9
:10323000010001008356C9020566011693F6F60FD8
:10324000D18EC206C1822316D90223800D00C65634
:10325000F3A6068001000100850A93FAFA0F95B2E1
:1032600033E6B60045C20356C9023305D0403338B1
:10327000A000B305B040B385054115826345B00099
:10328000D1E16371A608894663F05605930780086B
:10329000F3B7078093F78708BEDA01000100B7177C
:1032A0000040130770052380E704130780FA23808A
:1032B000E7040100010003D7C7027D8B2396E702D4
:1032C00023800704D65781BDF336048093F6860821
:1032D000B6DC01000100930680FA23809D00238064
:1032E000DD00010001008356C9020566011693F650
:1032F000F60FD18EC206C1822316D90223800D009B
:10330000E656B9B793078008F3B7078093F78708A5
:10331000BEDE01000100371700409307700523004F
:10332000F704930780FA2300F70401000100035615
:10333000C70293975600B297C207C1832316F702BC
:1033400023000704F657C1BB914763EEB70217D7B6
:1033500001001307272C8A05BA959C41BA978287EA
:10336000B717004003A7470B1345F5FF698F23AA42
:10337000E70A03A7070B698F23A8E70A03A7070A31
:10338000798D23A0A70A8280B717004083A6470B38
:103390001347F5FFF98E23AAD70A83A6070B558D8D
:1033A00023A8A70A83A6070A758F23A0E70A8280AD
:1033B000B717004003A7470B498F23AAE70A03A7C3
:1033C000070B1345F5FF45BFB717004083A6470B12
:1033D0001347F5FF758F23AAE70A03A7070A598D3C
:1033E0004DB7B717004003A7470B498FEDB791477B
:1033F00063EEB70217D70100130707238A05BA95B2
:103400009C41BA978287B717004003A7470D134521
:10341000F5FF698F23AAE70C03A7070D698F23A87F
:10342000E70C03A7070C798D23A0A70C8280B717A0
:10343000004083A6470D1347F5FFF98E23AAD70C4A
:1034400083A6070D558D23A8A70C83A6070C758F9F
:1034500023A0E70C8280B717004003A7470D498FD0
:1034600023AAE70C03A7070D1345F5FF45BFB717C0
:10347000004083A6470D1347F5FF758F23AAE70C7D
:1034800003A7070C598D4DB7B717004003A7470D89
:10349000498FEDB79357E50093F70730C98FC207FF
:1034A0000547C1836382E5048DC10947638DE50447
:1034B0000D476380E50637170040231FF708835642
:1034C0002709D58F2319F708828037170040035644
:1034D000670993C6F7FFF18E231BD7088326C70C15
:1034E000558D2326A70CC1BF371700400356670927
:1034F00093C6F7FFF18E231BD7088326870C558DC3
:103500002324A70C4DBF3717004083566709DD8E73
:10351000E1B73717004083566709DD8EE9BF79713F
:1035200022D43714004026D24AD0035924028354AF
:10353000040206D64209C2044ECE52CC56CA1359D2
:103540000901C1802DE11379F9F793F4F49F420941
:10355000C20413590901C18093078008F3B707809B
:1035600093F787083EC4010001009307700523000C
:10357000F404930780FA2300F404010001002311EE
:1035800024032310940223000404A247F3A7078016
:1035900001000100B250225492540259F249624A89
:1035A000D24A45618280B7F5070081463000B105F7
:1035B000194597F0FF1FE7800074A2471397270172
:1035C000E34A07FC1369090893E40440930980085F
:1035D000F3B7098093F787083EC001000100930A02
:1035E000700523005405130A80FA230044050100E6
:1035F00001002311240323109402230004048247B2
:10360000F3A7078001000100294597F0FF1FE7801D
:103610008025F3B9098093F989084EC201000100A1
:1036200023005405230044050100010083570402D0
:1036300093E707202310F402230004049247B9B74C
:10364000B71700408847420541819377050491EB05
:103650009377F5013755E801130505803345F502E9
:1036600082809377050C130700046397E700937734
:10367000F50137459C1CCDB72165130505D0828027
:1036800037E700E01C435443A183E206D58F1CC1F9
:10369000FD572320F7182322F7188280131785007F
:1036A000B7E700E023A0E710618123A2A710828082
:1036B000B7F700E08847CC47828081473737004022
:1036C000A14663C4C700328582800345B740E38EBC
:1036D000A6FE3385F5000345050085072304A740B2
:1036E000CDB797070020938767E19C4317370020E9
:1036F0001307C7B83E95636EE50017370020130720
:1037000067F06368A700170700202329A7DE3E851E
:103710008280FD57EDBF8280411122C406C62A84F3
:1037200097000000E78000F22947B307E502B240A6
:103730008D83B3D7870222449507B3D7E702373783
:103740000040C207C1832316F700410182807165E2
:1037500041111305052006C697000000E78000FC14
:10376000B7370040130770F82381E7000D47A381A6
:10377000E70013070004A380E70005472387E7005D
:10378000B2404101828037370040834727001A0545
:1037900093F7F703C98F93F7F70F2301F7008280A0
:1037A000B737004003C7170019C9D98DA380B700E8
:1037B00003C70700136787002380E700828093C553
:1037C000F5FFF98DA380B7008280AE872A87B736D0
:1037D000004021463738004089E7170300006700A2
:1037E000C3F383C8B600E30916FF05078348F7FF54
:1037F000FD17C20723041801C183F9BF411122C478
:1038000006C62A8497000000E780C0E32947B30773
:10381000E502B2408D83B3D7870222449507B3D720
:10382000E70237370040C207C1832316F740410142
:103830008280716541111305052006C697000000BE
:10384000E78000FCB7370040130770F82381E7409A
:103850000D47A381E74013070004A380E740054715
:103860002387E740B24041018280CC41411106C626
:10387000328503C6150083C5050022064D8E42061B
:103880008D654186138875A2630C0611634BC804CD
:10389000138845A26300060D634AC800938535A2CC
:1038A0006301B6082390060029464DA0138855A24F
:1038B0006305060D938565A2E316B6FE8D451D468C
:1038C00063E6E5081146198E63F3C7003E86B7E745
:1038D00004002390C600FC4797D50100938505D7C7
:1038E0009DA0138895A263030611634E060D1388ED
:1038F000A5A263000613938505A5E315B6FA9945BD
:103900001D4663E5E504198E63F3C7003E86B7E7FD
:1039100004002390C600FC4797050020938545C806
:103920001DA09D451D4663E3E5022146198E63F304
:10393000C7003E86B7E70400FC472390C600970502
:10394000002093852526BA9582970146B24032859C
:1039500041018280AD451D46E3EAE5FE3146198E00
:1039600063F3C7003E86B7E704002390C600FC4718
:1039700097D50100938505D0F9B7B1451D46E3E71A
:10398000E5FC3546198E63F3C7003E86B7E70400B1
:103990002390C600FC4797D501009385A5CE65B757
:1039A0008D451D46E3E4E5FA1146198E63F3C70021
:1039B0003E86B7E704002390C600FC4797D5010078
:1039C000938585C949B78D451D46E3E1E5F8114664
:1039D000198E63F3C7003E86B7E704002390C60044
:1039E000FC4797D501009385A5CBB1BFA5451D46E2
:1039F000E3EEE5F42946198E63F3C7003E86B7E788
:103A000004002390C600FC4797D50100938585C527
:103A10001DBFB5451D46E3EBE5F23946198E63F34C
:103A2000C7003E86B7E704002390C600FC4797D541
:103A300001009385A5C001BFB7E7040003A30713E6
:103A4000970600209386C6B44146A5451705002079
:103A5000130505AB02832D455DE703C50500094746
:103A6000631FE50803A84500411106C60347180077
:103A700032850346080022074168518F930828FECB
:103A80006307170563E9E80005186303070323903C
:103A90000600294591A8130648FE630AC7041518B5
:103AA000E31707FF15463E87637BF600154701A81D
:103AB000130600023E876374F60013070002B7E79F
:103AC00004002390E600FC471316070111A83E8668
:103AD00091C30546B7E70400FC472390C6004206A1
:103AE000CC45418282970145B24041018280130654
:103AF00000083E87E375F6FC13070008C9B723905A
:103B00000600054582808280416779176304E504D9
:103B1000411122C406C685472A84639FF500B7E792
:103B2000040022852244B24003A387139705002096
:103B3000938585214101028389476399F500B7E7A1
:103B4000040083A7070B8545829771D9B2402244B0
:103B5000410182808280797122D452CC2E842A8ABB
:103B600097D501009385C5B517D501001305C5B7D5
:103B700006D63AC626D24AD0B68432894ECE97B0FF
:103B80000100E780E008A68517D501001305C5B63A
:103B900097B00100E780C007294597B00100E78092
:103BA000000C8347840093F70702E1E78349040090
:103BB0008947054532476396F908544083C7160084
:103BC00083C60600A207D58FC166138616FE638CD6
:103BD000C7028D16638FD7068D669386269029457A
:103BE0006391D706B7E70400A285225403A34714C4
:103BF000B250F249A6864A86925402595285624AC8
:103C00008547456102832D450DEF93070002354539
:103C100063E99702B7E70400FC4748441306000233
:103C2000CA8582978149970700209387A7129C43F2
:103C3000014581CB9C4391C74E852686CA858297D4
:103C40000145B250225492540259F249624A4561E8
:103C500082802D457DF79307700F3545E3E397FE8E
:103C6000B7E70400FC4748441306700FCA858297E3
:103C70005DBF2145F9B7411122C437E40400832711
:103C8000841326C2AA84416506C697050020938541
:103C9000A50B7D1582978327C40A1705000013051D
:103CA000E5E68588829795C0032304132244B24039
:103CB000924497060020938626A04146C5451705E5
:103CC00000201305658E41010283B24022449244D4
:103CD00001454101828019C59707002023ACA70642
:103CE00001458280454582801147636AA70A97D6BD
:103CF00001009386A69B0A0536951841411106C618
:103D00003697AE87B2850287130700026145639D2F
:103D1000E700B7E70400FC47130600021705002080
:103D20001305C5E882970145B240410182800547ED
:103D30006145E39BE7FEB7E70400FC47054617052E
:103D400000201305A5E8F9BF1307700F6145E39D37
:103D5000E7FCB7E70400FC471306700F17050020C7
:103D6000130505E7C1B7130700086145E39EE7FAAD
:103D7000B7E70400FC4713060008170500201305E9
:103D8000A5F44DB715476145E390E7FAB7E704009E
:103D9000FC47154617050020130545FB61B709458B
:103DA0008280411126C2B7E4040083A7C41322C451
:103DB0004AC006C62E84970500209385E5F82A8917
:103DC0008297058905C597F7FF1F9387E77D83D7FE
:103DD000A70BA28503A3440D2310F4002244B24094
:103DE00092444A850249014641010283B24022447D
:103DF00092440249494541018280114517F3FFFF72
:103E0000670083C8411193962500AA852D4506C6F3
:103E100097F0FF1FE78020EEB2400145410182800C
:103E2000011122CC06CE3714004026CA4AC84EC61D
:103E300052C483447405034AB40583498405034985
:103E4000940597F0FFFFE780209A8347A40593F439
:103E5000F40F137AFA0F93E71700230DF40493F984
:103E6000F90F1379F90FB717004003C7A705058BA2
:103E70006DFF03D5C705A38D4705238C3705A38C9C
:103E80002705A38B9704F2406244D2444249B249C9
:103E9000224A0561828041119397050122C406C61A
:103EA00026C2C1872E8463D00702B7E40400FC5405
:103EB000829719C1BC5482972165218DB24022445A
:103EC00092444101828093F7150013C51500FDF758
:103ED0009397250163D80702B7E4040083A7C41EA3
:103EE000829797000000E78080F1BC4C37F6020013
:103EF000130606E0896517050020034525E682972D
:103F0000096565BF939715010145E3D907FA17D5F0
:103F100001001305658697B00100E78040E7B7E729
:103F20000400BC4F1306006491651705002003458B
:103F3000E5E28297116551B72D71232A9110FD7426
:103F4000E98C232C811023282111232631112A8466
:103F5000AE893289930600100A86A6852D45232E48
:103F6000111097F0FF1FE78000D913154401B7E740
:103F70000400FC4751810A0513962900CA850A9559
:103F80008297A68585660146254597F0FF1FE78045
:103F900080D60A86A68593060010294597F0FF1F54
:103FA000E78060D58320C11103248111832441114E
:103FB000032901118329C11015618280B7F7070019
:103FC00003C70701411106C622C426C24AC0A5473D
:103FD000631DF70097000000E78040F6B2402244DE
:103FE0009244024901454101828013942500AA842C
:103FF0003289A286AA850146254597F0FF1FE780F2
:1040000080CFA2864A86A685294597F0FF1FE780C4
:1040100080CEE9B71D71A6CAB7E40400DC5CC858BD
:1040200086CEA2CC494697C50100938565708297DC
:1040300011E917C501001305E57097B00100E7808D
:1040400000D501A037F700E0795610CBFD5654CBD0
:10405000B7E700E0056423A087109306F00214C3BD
:1040600023A0871801000100370700201847130616
:10407000000481459706002023A0E6CE4157A38A7D
:10408000E740BC4408088297970700209387C769D8
:104090003EC89D673ECCB7070104938707103ECE0C
:1040A0009307B00F2310F10285472301F102970710
:1040B0000000938767D5BEC297070000938747F03B
:1040C000BEC4930750112312F10297F7FFFF9387A5
:1040D000675E3ED8970700009387C7D43EDCB7F5EC
:1040E000070097070000938787D13EDE8146970738
:1040F00000009387471E3000E10519453EDA231A78
:10410000810097F0FF1FE78000BF1808814799469C
:1041100030003E960346060085070507A30BC7003F
:10412000E398D7FEC24791C7035741018567637380
:10413000F70001A0B7E7040083A7470A08088297A1
:10414000AA8511C917C501001305056197B00100C3
:10415000E78000AC01A0F6406644D6442561828029
:10416000411126C2B7E4040083A7040806C622C48E
:1041700017050000130565D2829717040020130469
:10418000E4BD2300A40097000000E780000797002B
:104190000000E780E02203450400224403A38405D5
:1041A000B2409244130600328965410102834111F5
:1041B00093078008F3B7078093F787083EC601008E
:1041C0000100B7170040130770052380E7041307A9
:1041D00080FA2380E70401000100C8DB2380070484
:1041E000B247F3A70780010001009707002023A929
:1041F00007B641018280797106D622D41307800860
:10420000F337078093F787083EC201000100B71714
:104210000040930570052380B704130680FA2380BD
:10422000C7040100010083C6F70293F6A60FA38717
:10423000D702238007049246F3A6068001000100FE
:1042400073370780137787083AC401000100238081
:10425000B7042380C7040100010003C7F7021367F6
:104260002700A387E70223800704A247F3A707805C
:1042700001000100054597E0FFFFE780005F970020
:104280000000E780C0B70147814681470546854564
:104290001305407E97E0FFFFE780006237E40400EB
:1042A0003C446800514681458297B707C0A83EC884
:1042B000B787E803938707D03ECA97E7FF1F938726
:1042C00047633EC67C5868008297B25022544561CD
:1042D0008280011126CA06CE22CCAA849730000023
:1042E000E780E0FD71C9930730031384D4FC63E7D2
:1042F00097003704C0A81304D4FC2694680097F0F4
:10430000FFFFE780203897E0FF1FE780C0D8B307A2
:10431000A4406376A400B707C0A8A297898F374747
:10432000F6A68117130707C6637DF700324597F09D
:10433000FFFFE780E0360945F2406244D244056160
:104340008280228597000000E780A0E6324597F042
:10435000FFFFE780E034373700408347574093F74B
:104360000704A9CB97300000E78080FB9707002067
:104370009387079F9C43A9E31165690597E0FF1F99
:10438000E78000EA054597E0FFFFE7802049054503
:1043900097F0FFFFE780E01897E0FF1FE780A0CFCE
:1043A0002AC497E0FF1FE78000CFA247E30BF5FE8A
:1043B000014559B7010055B70D45BDBF011106CEE6
:1043C00022CC13078008F337078093F787083EC491
:1043D00001000100B7170040930570052380B70462
:1043E000130680FA2380C7040100010083C6E7009A
:1043F00093E696012387D70023800704A246F3A6FD
:1044000006800100010073370780137787083AC6DA
:10441000010001002380B7042380C70401000100CC
:1044200003C7170313670702A388E7022380070463
:10443000B247F3A7078001000100B707001037E477
:1044400000E02320F4108545414597F0FFFFE78009
:1044500040FA8945414597F0FFFFE780E003B70741
:1044600004002320F410F24062440561828041116F
:1044700097D501009385859617C501001305C526BC
:1044800006C697A00100E780A07817D501001305A4
:10449000A5AD97A00100E780A077B2402945410172
:1044A00017A301006700A37B411197D501009385F5
:1044B000259417C501001305252306C697A0010002
:1044C000E780007517D501001305C5A897A0010066
:1044D000E7800074B2402945410117A3010067003D
:1044E0000378411122C406C6834705002A849DC76C
:1044F00097D501009385859517C501001305C51E45
:1045000097A00100E780C0704C4017D5010013054B
:10451000E5B997A00100E780A06F3DA058410DEFDD
:1045200097D501009385859217C501001305C51B1A
:1045300097A00100E780C06D17D50100130585B86D
:1045400097A00100E780C06C2244B2402945410198
:1045500017A301006700A370A1679386D7036313B5
:10456000D70297D501009385658E17C50100130505
:10457000A51797A00100E780A06917D501001305D2
:1045800065B57DBFED0797D501009385258C17C5CF
:10459000010013056515631BF70097A00100E78074
:1045A000206717D50100130525B459BF97A0010056
:1045B000E78000664C4017D501001305E5B491BFB4
:1045C000411197D501009385E58317C501001305B7
:1045D000A51106C697A00100E7808063B240294577
:1045E000410117A3010067008367797122D426D2A5
:1045F0004AD02E842A898145B2844800714606D665
:1046000097E0FFFFE780E00197F7FF1F9387872B75
:10461000DC4783D70700231421012313F1009750AF
:104620000000E78000819547A305F1009307401F34
:104630003EC6FD572305A100230AF1009750000054
:10464000E78060932686A285480097500000E780A7
:104650002081B250225492540259456182809717AA
:1046600000202396071C97170020238F070AB7E71F
:104670000400BC47411106C641468145170500208C
:10468000130505F9829797200000E780E05D9720E9
:104690000000E7802039014597500000E780202086
:1046A000170700200347C7F89307F00A6315F702BE
:1046B0009307F0F8894517050020130565F71707DC
:1046C00000202307F7F697070020A38307F69750EB
:1046D0000000E780C04C97500000E780A05E814555
:1046E000370504009707002023A207F29707002050
:1046F000239C07F097070020238907F097070020E5
:10470000239A07E897070020239807E697070020D9
:10471000239B07EE97070020239407F097300000B3
:10472000E78020C4014597500000E780405097C5BE
:1047300001009385A56F17C501001305E5FA97A041
:104740000100E780E04C17D50100130525A297A0D2
:104750000100E780E04BB2402945410117A3010069
:104760006700E34F411122C406C626C293F7150025
:104770002E84638F0710814617F6FF1F1306C6119C
:104780008545170500200355E5DE97C00000E7804A
:10479000E0B915C997C501009385056A17C50100E1
:1047A000130585F497A00100E780804617C5010036
:1047B0001305450B97A00100E7808045294597A088
:1047C0000100E780C04997C501009385E56617C5DC
:1047D0000100130565F197A00100E780604317C54C
:1047E00001001305650997A00100E7806042294593
:1047F00097A00100E780A04617F5FF1F1305850C61
:104800005C4505472390E70097300100E780606A28
:1048100097C501009385456217C501001305C5ECD6
:1048200097A00100E780C03E17C5010013050506EB
:1048300097A00100E780C03D294597A00100E780CF
:104840000042930710F8170700202303F7DE9707AD
:10485000002083D7E7D117070020A30BF7DC17054B
:1048600000201305E5DCA1839145170700202302F2
:10487000F7DC97070020A38E07DA97500000E78047
:10488000003213451400B240224492444101828018
:1048900093F72500E1C3170700200357E7D645CB60
:1048A00097060020938686D6944297D70100938777
:1048B000E78D17060020034646D5814517050020E1
:1048C000130505D597700000E780A0C5AA8441C1F3
:1048D00097C501009385055D17C501001305C5E067
:1048E00097A00100E780C032A68517C50100130517
:1048F00065FB97A00100E780A031294597A0010042
:10490000E780E03597070020239007D0930710F841
:1049100017070020230EF7D09707002083D747C53D
:1049200017070020A306F7D0A18317070020230252
:10493000F7D091458D4717050020130565CF170760
:104940000020A308F7CE97500000E78040251345CC
:10495000240015BF93F74500D1C397C50100938587
:10496000655417C50100130525D897A00100E780FD
:10497000202A17C501001305A5F497A00100E780C0
:104980002029294597A00100E780602D930720F892
:1049900017070020230EF7C89707002083D787BF8B
:1049A00017070020A306F7C8A183170700202302DA
:1049B000F7C8854717070020A30DF7C697400000EA
:1049C000E780605B17050020130585C69145975069
:1049D0000000E780C01C1345440075B593F78500BF
:1049E000A9C797C501009385E54B17C501001305BD
:1049F000A5CF97A00100E780A02117C501001305EE
:104A000065ED97A00100E780A020294597A001004F
:104A1000E780E02497070020239807BE97700000E6
:104A2000E78000C013458400B9BD93F70501D1C3E9
:104A30008545170500200355E5B597500100E7802F
:104A4000207297C501009385E54517C50100130540
:104A5000A5C997A00100E780A01B17C50100130599
:104A6000A5E897A00100E780A01A294597A00100BA
:104A7000E780E01E930730F817070020230AF7BAF3
:104A80009707002083D707B117070020A302F7BAC2
:104A9000170500201305C5B9A1838D451707002010
:104AA0002309F7B897500000E780600F1345040111
:104AB000D9BB93F70502D1C797C501009385853E01
:104AC00017C50100130545C297A00100E7804014F7
:104AD00017C50100130585E397A00100E780401387
:104AE000294597A00100E7808017930740F8170732
:104AF0000020230FF7B29707002083D7E7A71707F7
:104B00000020A307F7B2A183170700202303F7B201
:104B1000854717070020A30EF7B097070020239DB5
:104B200007A497400000E780004517050020130503
:104B300025B0914597500000E780600613450402B8
:104B400099B393F70504FDC397C501009385853597
:104B500017C50100130545B997A00100E780400B78
:104B600017C50100130505DC97A00100E780400A86
:104B7000294597A00100E780800E9707002083C792
:104B800027AB1307700A6386E7061307800A638C56
:104B9000E7081307600A6393E704930760F81707B1
:104BA00000202307F7A89707002083D7C7A517077A
:104BB0000020A30FF7A6A18317070020230BF7A659
:104BC000854717070020A30AF7A6B145170500205F
:104BD000130505A697500000E78060FC9740000091
:104BE000E78060391345040497070020239D07A040
:104BF00059B9930770F817070020230BF7A29707FE
:104C0000002083D747A017070020A303F7A2A183A2
:104C100017070020230FF7A0854717070020A30BD5
:104C2000F7A0994565B7930780F8F1B793F70508A2
:104C30000145E38A07C497C501009385A52617C5DA
:104C40000100130565AA97A00100E78060FC17C565
:104C500001001305A5CE97A00100E78060FB294560
:104C600097A00100E780A0FF9307A0F81707002096
:104C70002300F79C9707002083D7879A1707002007
:104C8000A308F79AA183170700202304F79A854702
:104C900017070020A30FF798970700202392079883
:104CA00097400000E780202D170500201305459848
:104CB000914597500000E78080EE13450408E1B667
:104CC000411122C497C50100938585192A8417C50F
:104CD0000100130565A106C697A00100E78040F317
:104CE0004C4017C501001305E53997A00100E78086
:104CF00020F2294597A00100E78060F603470400F1
:104D00009307F00F631FF70297C5010093854515C0
:104D100017C501001305459D97A00100E78040EFEE
:104D20004C4017C501001305E53697A00100E78048
:104D300020EE2244B2402945410117A3010067003B
:104D400003F2B240224441018280B1C1411122C428
:104D500017C50100130545992E8497C50100938559
:104D6000250B06C697A00100E78080EAA28517C53B
:104D700001001305653D97A00100E78060E922442A
:104D8000B2402945410117A30100670043ED82802D
:104D9000411122C426C22E84AA8497C5010093859E
:104DA000E50717C501001305259406C697A0010065
:104DB000E78000E617C501001305C53997A001007B
:104DC000E78000E5294597A00100E78040E997C505
:104DD00001009385A50497F7FF1F239D977817C5BA
:104DE000010013056590854497F7FF1F239287788C
:104DF00097F7FF1F239F977697170020239987A285
:104E000097A00100E780C0E09715002083D525A278
:104E100017C501001305853497A00100E78040DF26
:104E2000294597A00100E78080E397170020238D94
:104E3000978E97200000E780E0BE22859750000003
:104E4000E780E0A5054597500000E78040DE97F732
:104E5000FF1F938727A7DC4703D70700C167FD170C
:104E60006312F7022244B7E70400B240924403A35E
:104E7000870517F5FF1F0345E5EE1306000A854574
:104E800041010283B24022449244410182800111D7
:104E900022CC37E404005C5C06CE26CA354697C5B2
:104EA00001009385A50D17D50100130525D2829722
:104EB00011E917C501001305E58897A00100E780F7
:104EC00000ED01A097F7FF1F938787EA3EC4B7F56F
:104ED0000700856793870780814617F6FF1F130633
:104EE000A6E8E10519453EC697E0FF1FE780A0E070
:104EF0007C44194697F5FF1F938505E717F5FF1FBB
:104F0000130585698297340017F6FF1F1306C6E55F
:104F100097C501009385855E17C501001305855F60
:104F200097600000E780E034AA8421C197C50100A2
:104F3000938545F617B501001305057B97A0010081
:104F4000E78000CDA68517C501001305250497A0AD
:104F50000100E780E0CB294597A00100E78020D041
:104F6000F2406244D2440561828097E00000E7800D
:104F7000209717C50100130565F897500000E780DA
:104F8000002997A00000E78060EB97500100E780C0
:104F9000E04F17F5FF1F1305658F97500100E7805D
:104FA000803817C50100130565F697500100E780AA
:104FB0006050AA8497600000E780408F970001004E
:104FC000E780C02797800100E780E0C0977000006D
:104FD000E78080E797600000E78040059730010098
:104FE000E78020E997C501009385C5EA17B5010060
:104FF0001305856F99C897A00100E78060C1A68559
:1050000017C501001305C5FA99B797A00100E780FD
:1050100020C017C501001305E5FB97A00100E7803C
:1050200020BF294597A00100E78060C397300100A9
:10503000E78000C597F00000E780C0E3630F05102C
:1050400085453705040097200000E780803197C52B
:105050000100938525E417B501001305E56897A0C5
:105060000100E780E0BA17C50100130525F897A0F5
:105070000100E780E0B9294597A00100E78020BE44
:1050800097E7FF1F9387C77383D707001707002091
:10509000231FF7788547170700202307F768972015
:1050A0000000E780E0B697200000E780A097170592
:1050B00000200355C57797400000E780407E97F7B2
:1050C000FF1F83C73766ADEBA30301008327441797
:1050D00013067100854513055030829797C501006E
:1050E000938545DB17B501001305056097A0010006
:1050F000E78000B217C50100130585F197A00100F4
:10510000E78000B1294597A00100E78040B597C529
:105110000100938525D817B501001305E55C97A01C
:105120000100E780E0AE17C50100130565F497A004
:105130000100E780E0AD05B597C50100938585D5F1
:1051400017B501001305455A97A00100E78040AC50
:1051500017C50100130545EF55B797C501009385A5
:1051600065D317B501001305255897A00100E78006
:1051700020AA17C50100130565FF97A00100E7806D
:1051800020A9294597A00100E78060AD014597500F
:105190000000E780C0A9A5BF411122C437E4040084
:1051A0008327041A06C6829797400000E78040785C
:1051B0008327040817F5FFFF1305055B829797F710
:1051C000FF1F2381A7BA17E5FF1F1305A56F97409F
:1051D0000000E780E00C2244B240410117030000C8
:1051E000670023CBB7E70400FC471171A2DDCAD9E1
:1051F00086DFA6DBCED72E8432892E86AA8517F5C8
:10520000FF1F1305E542829717F7FF1F1307474259
:1052100083470700930680029387E70793F7F70F0A
:10522000E3ECF610BA898A0717B701001307075590
:10523000BA979C43BA9782878D4797C5010093859B
:10524000A5C717B501001305254A630FF40097A001
:105250000100E780E09B17C501001305A58497A016
:105260000100E780E09ABDA497A00100E780409A82
:1052700017C501001305858497A00100E7804099B8
:10528000294597A00100E780809D930720F81146EB
:1052900097F5FF1F9385C5394A8517F7FF1F230927
:1052A000F73897F7FF1FA386073897F0FFFFE780CF
:1052B00000342A841DC997C501009385E5BF17B541
:1052C00001001305654297A00100E7806094A28564
:1052D00017C501001305458297A00100E7804093A0
:1052E000294597A00100E780809797C50100938525
:1052F000A5BC17B501001305253F97A00100E78065
:10530000209117C501001305658097A00100E78073
:105310002090294597A00100E7806094416593079C
:1053200030FA054697F5FF1F938585307D1517F7F1
:10533000FF1F230FF72E97F0FFFFE780402B2A84F3
:105340001DC997C50100938525B717B50100130541
:10535000A53997A00100E780A08BA28517B50100B1
:105360001305857997A00100E780808A294597A0D9
:105370000100E780C08EB7E70400BC4F0566130646
:1053800006C8A14517F5FF1F0345C59D8297FE502E
:105390006E54DE544E59BE591161828091476303A9
:1053A000F40297C50100938525B117B501001305D7
:1053B000A53397A00100E780A08517B5010013056C
:1053C000257871BDB7E70400FC4F914517F5FF1F25
:1053D00003454599829797C501009385E5AD17B5BB
:1053E00001001305653097A00100E780608217B5C2
:1053F00001001305A57697A00100E780608129458B
:1054000097A00100E780A08597400000E780A0B644
:10541000914535A485476303F40297C50100938540
:10542000A5A917B501001305252C97900100E78069
:10543000207E17B501001305E57315B597F7FF1F1B
:10544000239A2715B7E704000566BC4F130606C864
:10545000C1450DBF8D476303F40297C501009385D5
:10546000A5A517B501001305252897900100E78031
:10547000207A17B501001305A571D5B3930740F83D
:10548000114697F5FF1F9385A51A4A8517F7FF1F49
:105490002300F71A97F7FF1FA38D071897F0FFFF58
:1054A000E780E0142A84E30405EE97C501009385A4
:1054B000A5A017B501001305252397900100E780EB
:1054C0002075A28517B501001305056397900100AB
:1054D000E7800074294597900100E780407845BD3A
:1054E0009147E31CF4F6B7E70400FC4F9305000274
:1054F00017F5FF1F03450587829797C50100938520
:10550000A59B17B501001305251E97900100E780A4
:10551000207017B5010013052569F1BD894763E3C4
:10552000870297C501009385259917B501001305DA
:10553000A51B97900100E780A06D17B5010013052A
:10554000E56731BB97F4FF1F83C4A40E97F7FF1FD5
:1055500083C7170E97C5010093850596A20417B55A
:10556000010013056518DD8C97900100E780406A03
:10557000A28517B501001305A56597900100E78086
:105580002069C204294597900100E780406DC184DD
:105590009305D4FF93960401C1824A8693F5F50FD3
:1055A00017F5FF1F1305F50897200000E78020DF9F
:1055B000E35F90DC930750F817F7FF1F230AF70605
:1055C00083C73900228697F5FF1F938565068507F7
:1055D0004A8517F7FF1FA30EF70497F0FFFFE78038
:1055E00000012A84E30505DA97C501009385C58C7F
:1055F00017B501001305450F97900100E780406142
:10560000A28517C50100130525B3C9B5894763E312
:10561000870297C501009385258A17B501001305F8
:10562000A50C97900100E780A05E17B50100130557
:10563000E55B35B197400000E780E093A28517F560
:10564000FF1F1305E5FE97400000E780405581B33A
:105650008D476303F40297C501009385E58517B56F
:1056600001001305650897900100E780605A17B59F
:10567000010013056559E5B6B76602000146B77526
:105680000200054597D0FF1FE780E066930760F8AA
:1056900017F7FF1F230EF7F897F7FF1FA38B07F8E5
:1056A0009307000617F7FF1F2306F7F8894717F738
:1056B000FF1FA301F7F897F7FF1F238E07F697F751
:1056C000FF1FA38A07F6C14717F7FF1F2306F7F648
:1056D000930720F917F7FF1FA300F7F6314697F756
:1056E000FF1FA38CA7F497F5FF1F938565F44A85E8
:1056F00097F7FF1F238307F497F0FFFFE78020EF62
:105700002A84E30605C897B501009385E57A17B5A5
:105710000100130565FD97900100E780604FA285A9
:1057200017B501001305C54F55B3B1476303F40224
:1057300097B501009385457817B501001305C5FAA3
:1057400097900100E780C04C17B501001305054F85
:1057500039B6B7E70400FC4F9305000417E5FF1FB7
:1057600003454560829797400000E780C080B145BF
:10577000F9B5914763E3870297B501009385C57337
:1057800017B50100130545F697900100E7804048E2
:1057900017B501001305454CD9B497F4FF1F83C416
:1057A00064E997F7FF1F83C7D7E8A204DD8C8E0456
:1057B000B77702006D14BE942286A68517B5010046
:1057C0001305C54A97900100E7808044B7E70400BD
:1057D000FC47228697F5FF1F9385D5E52800829721
:1057E00093160401C1823000A685094597D0FF1F9A
:1057F000E78060502A8409C917B501001305C54820
:1058000097900100E780A058930770F8194697F524
:10581000FF1F9385E5E14A8517F7FF1F230AF7E08D
:1058200097F7FF1FA38887E097F0FFFFE78020DC52
:105830002A84E30E05B497B501009385E56717B593
:105840000100130565EA97900100E780603CA2859E
:1058500017B501001305454495B99947630BF41238
:1058600097B501009385456517B501001305C5E798
:1058700097900100E780C03917B501001305454333
:10588000F9BA914763E3870297B501009385C56232
:1058900017B50100130545E597900100E7804037F3
:1058A00017B50100130545425DBA97F4FF1F83C485
:1058B00064D897F7FF1F83C7D7D7A204DD8C8E0467
:1058C000B77702006D14BE942286A68517B5010035
:1058D0001305C54097900100E7808033B7E70400C7
:1058E000FC47228697F5FF1F9385D5D42800829721
:1058F00093160401C1823000A6850D4597D0FF1F85
:10590000E780603F2A8409C917B501001305C53E29
:1059100097900100E780A047930780F8194697F514
:10592000FF1F9385E5D04A8517F7FF1F2302F7D0A5
:1059300097F7FF1FA38087D097F0FFFFE78020CB6A
:105940002A84E30605A497B501009385E55617B5AB
:105950000100130565D997900100E780602BA285AF
:1059600017B501001305853A95B699476303F4020C
:1059700097B501009385455417B501001305C5D6A9
:1059800097900100E780C02817B5010013058539FD
:10599000F9B0B7E70400FC4F9305000417E5FF1FBB
:1059A0000345453C829797300000E780C05C9945ED
:1059B00079B18D476303F40297B501009385C54F14
:1059C00017B50100130545D297900100E7804024E8
:1059D00017B501001305853659B017B50100130539
:1059E000E53697900100E780803A1305C01297D002
:1059F000FF1FE78020E8014597E0FFFFE78080C8B0
:105A00000D4597100000E780009F294597D0FF1FA4
:105A1000E78040E697D0FF1FE780A0D68DBA994770
:105A20006303F40297B501009385054917B501009A
:105A3000130585CB97900100E780801D17B5010005
:105A40001305853129B817F7FF1F0347B7BE97F72E
:105A5000FF1F83C727BE22075D8F9166BA96C206D5
:105A60001166C1821306F6EF8D476365D60297E78C
:105A7000FF1F938727E59C4B17F6FF1F034676BB56
:105A80009386C7002DC203D6070069CA8907E39C25
:105A9000D7FE89471307A0F8114697F5FF1F938596
:105AA00025B94A8597F6FF1F2384E6B817F7FF1F2D
:105AB000A301F7B897F0FFFFE78060B32A84E308FB
:105AC000058C97B501009385253F17B50100130597
:105AD000A5C197900100E780A013A28517B501002A
:105AE0001305C528E5B203D60700630EE60A890749
:105AF000E39BF6FE8D4779BF91476304F40297B5A7
:105B000001009385653B17B501001305E5BD97902E
:105B10000100E780E00F17B501001305A5266FF01F
:105B20000FF4B7E70400FC4F9305000817E5FF1FCB
:105B3000034545238297C9B897B501009385C537BA
:105B400017B50100130545BA97900100E780400C96
:105B500017B50100130585246FF06FF02390E7005F
:105B600017E5FF1F130505D697200100E780C03613
:105B700097B501009385453417B501001305C5B6E7
:105B800097900100E780C00817B5010013050522B2
:105B900097900100E780C007294597900100E780B2
:105BA000000C8147C5BD2390070017E5FF1F1305B3
:105BB00065D197200100E780203297B501009385D9
:105BC000A52F17B50100130525B297900100E780B6
:105BD000200417B501001305E51E5DBF411122C465
:105BE00006C6834705002A849DC797B501009385A3
:105BF000652817B50100130525AF97900100E780D0
:105C000020014C4017B5010013054559979001003C
:105C1000E7800000E1A05841B707CF009387777D68
:105C2000631DF70697B501009385C52417B50100DC
:105C3000130585AB97900100E78080FD1C448356D7
:105C4000E4008355C40003C6070017B5010013051F
:105C5000655697900100E780A0FB294597900100C9
:105C6000E780E0FF0357E4009707002083D727BCB5
:105C70006309F7008355C400084497E0FFFFE780FD
:105C800000B50356E4008355C40008442244B240E2
:105C9000410117F3FFFF67002355B707CC00938737
:105CA000777D6315F70497B501009385A51C17B59B
:105CB0000100130565A397900100E78060F51C447F
:105CC0008356E4008355C40003C6070017B50100DE
:105CD0001305454E97900100E78080F32244B240BF
:105CE0002945410117930100670063F7B707CE000C
:105CF0009387777D6304F70297B501009385851735
:105D000017B501001305459E97900100E78040F00C
:105D10004C4017B501001305253FCDBDB2402244CC
:105D200041018280B7E70400FC4741112E8606C678
:105D300022C426C24AC02E842A89AA8517F5FF1FCD
:105D40001305058F829797B501009385A51817B5A0
:105D500001001305659997900100E78060EB97F5C6
:105D6000FF1F83C5E58C17B501001305A5BE9790ED
:105D70000100E780E0E9294597900100E78020EEE7
:105D800097F4FF1F9384C48A83C704004147938715
:105D9000070693F7F70F636AF75C17B7010013075D
:105DA00027A88A07BA979C43BA9782879D476307BB
:105DB000F40297B501009385E51117B501001305AD
:105DC000A59297900100E780A0E417B501001305A4
:105DD000E5B897900100E780A0E3ADAC97F7FF1F0F
:105DE00083C71785DDCB17F7FF1F0347978497F706
:105DF000FF1F83C7078422075D8F97F7FF1F83C7A5
:105E00006783C2075D8F97F7FF1F83C7B782E207DB
:105E1000D98F17E7FF1F232BF77E83C7640097B541
:105E200001009385250B17B501001305E58B17E7D6
:105E3000FF1F230CF77C97900100E78060DD97E758
:105E4000FF1F9387A77C8C4317E6FF1F0346E67B63
:105E500017B50100130545B297900100E78040DBBC
:105E6000294597900100E78080DF97E7FF1FA38116
:105E7000077C2244B24092440249930700F817E796
:105E8000FF1F2307F77A9D4517E5FF1F1305457A86
:105E9000410117430000670083D097600000E7804E
:105EA000A08797E7FF1F2386A7789357850017E7FA
:105EB000FF1FA300F778935705012A8417E7FF1FF8
:105EC000230AF77693578501014517E7FF1FA303C0
:105ED000F77697600000E780E08497E7FF1F238C48
:105EE000A77497B501009385E5FE17A5010013057A
:105EF000A57F97900100E780A0D117E6FF1F03461A
:105F00008673A28517B50100130585A8B1B7CD47E3
:105F10006303F40297B501009385C5FB17A5010043
:105F20001305857C97900100E78080CE17B50100AE
:105F3000130585A779BD37E404007C44414697E505
:105F4000FF1F9385F56E17E5FF1F1305656C82979C
:105F500017E5FF1F1305C56B97100000E78060C4AD
:105F600097100000E78000AC97E7FF1F83C7676DBD
:105F700017E7FF1F0347D76CA20703238405D98FB8
:105F800017E7FF1F2312F7681306000A894522440A
:105F9000B2409244024917E5FF1F0345A5DC4101C9
:105FA00002838D476303F40297B50100938585F260
:105FB00017A501001305457397900100E78040C5C0
:105FC00017B50100130505AE29B517E4FF1F0344FB
:105FD000446697E7FF1F83C7B76597B501009385B0
:105FE00065EF220417A50100130505705D8C9790DD
:105FF0000100E780E0C1A28517B501001305459CAB
:1060000097900100E780C0C0294597900100E78084
:1060100000C50D4697E5FF1F93858561228597E0B2
:10602000FFFFE780C05CAA8421C197B5010093857A
:1060300065EA17A501001305256B97900100E7801D
:1060400020BDA68517B501001305C59897900100DE
:10605000E78000BC2244B2409244024929454101F4
:10606000179301006700A3BF97E7FF1F2394875290
:10607000B7E70400116603A38705130606E89145F8
:1060800039B78D476303F40297B50100938585E422
:1060900017A501001305456597900100E78040B7FB
:1060A00017B501001305C5AE2DB317E4FF1F034458
:1060B000445897E7FF1F83C7B75797B501009385EB
:1060C00065E1220417A50100130505625D8C979018
:1060D0000100E780E0B3A28517B501001305C59064
:1060E00097900100E780C0B2294597900100E780B2
:1060F00000B70D4697E5FF1F93858553228597E0EE
:10610000FFFFE780C04EAA841DC197B501009385AB
:1061100065DC17A501001305255D97900100E78058
:1061200020AFA68517B501001305458D05B797E784
:10613000FF1F23938744B7E70400116603A3870575
:10614000130606E89305000299B5894763E38702C1
:1061500097B50100938505D817A501001305C5580B
:1061600097900100E780C0AA17B50100130505A5A7
:106170008DB197E4FF1F83C4C44B97E7FF1F83C70C
:10618000374B97B501009385E5D4A20417A501000C
:1061900013058555DD8C97900100E78060A7A685E3
:1061A00017B501001305058797900100E78040A609
:1061B000294597900100E78080AA228697E5FF1F76
:1061C00093850547268597E0FFFFE78040422A84B4
:1061D000630E051A97B501009385C5CF17A5010079
:1061E0001305855097900100E78080A2A28517B51E
:1061F00001001305658399BD854763F987188345B9
:1062000019002244B24092440249B335B00097E7E6
:10621000FF1F238BB73817B50100130525824101F5
:10622000179301006700C39EA2852244B2409244A6
:106230004A8502494101170300006700032299477C
:106240006303F40297B501009385C5C817A5010043
:106250001305854997900100E780809B17B50100E1
:10626000130585AFBDB617E4FF1F0344843C97E7D1
:10627000FF1F83C7F73B97B501009385A5C522048F
:1062800017A50100130545465D8C97900100E78036
:106290002098A28517A501001305C57B97900100E2
:1062A000E7800097294597900100E780409B1946B9
:1062B00097E5FF1F9385C537228597E0FFFFE780AD
:1062C0000033AA841DC197B501009385A5C017A509
:1062D00001001305654197900100E7806093A68552
:1062E00017A501001305057895B397E7FF1F2399BC
:1062F0008732B7E70400116603A38705130606E893
:106300009305000869B1854797B50100938585BC61
:1063100017A501001305453D630BF400979001009C
:10632000E780008F17A50100130505755DB49790F0
:106330000100E780E08D17A50100130565759790B2
:106340000100E780E08C294597900100E7802091CB
:106350002244B2409244024997E7FF1F2396072A3E
:106360004101175300006700A32B97B501009385E7
:1063700065B617A501001305253797900100E78042
:10638000208917B50100130565A1A1B4B2402244CC
:106390009244024941018280411106C622C497E01D
:1063A000FFFFE780C0249377F50FA1C32A8497B538
:1063B00001009385A5B317A501001305E532979059
:1063C0000100E780E0849375F40F17B50100130511
:1063D000A5D697900100E780A0832244B2402945CA
:1063E00041011793010067008387B24022444101B5
:1063F0008280411122C491462A8417E6FF1F1306AA
:1064000066319D652D4506C697D0FF1FE780A08E9B
:10641000B7F7070003C70701A5476313F70001A0FB
:106420009306001001469D65254597D0FF1FE78024
:10643000808C97E7FF1F238F872C2244B240914620
:1064400017E6FF1F1306062D9D652945410117D349
:10645000FF1F6700438A5171CAD137E904008327BF
:10646000C904A2D52E8686D7A6D32E84AA8517E581
:10647000FF1F1305E51B829797E7FF1F83C7471B85
:106480001307700A6387E710636CF7001307600A4D
:106490006384E704BE502E549E540E596D61828071
:1064A0001307800A6388E7161307900AE394E7FE50
:1064B0008D476309F41C97B50100938525DB17A56B
:1064C00001001305652297800100E780607417B50D
:1064D00001001305E5D625A08D47630CF40297B59E
:1064E00001009385A5D817A501001305E51F978026
:1064F0000100E780E07117B501001305A5CD978075
:106500000100E780E070294597800100E780207551
:1065100051B7854717B50100130585CD17E7FF1F54
:106520002304F70897900100E7806086B7750200A2
:10653000B76602000146054597C0FF1FE780A07BB4
:10654000930760F817E7FF1F2304F70E97E7FF1F75
:10655000A381070E9307002617E7FF1F232CF70CD4
:10656000E5779387072117E7FF1F2317F70CB1453E
:1065700097E7FF1F2383070C97E7FF1FA38FA70A47
:1065800017E5FF1F1305C50A97300000E78020615B
:1065900011B7914763E3870297B50100938505CD55
:1065A00017A501001305451497800100E780406698
:1065B00017B501001305C5C599B797E4FF1F83C43C
:1065C000640797E7FF1F83C7D706A204DD8C8327E4
:1065D000C9046D14228697E5FF1F9385B505280031
:1065E00082978E0493160401B7750200C1823000B1
:1065F000A695094597C0FF1FE780E06F930770F8E5
:1066000017E7FF1F2306F702994597E7FF1FA383AC
:10661000A702BDB7914763E3870297B50100938551
:10662000E5C417A501001305250C97800100E7803C
:10663000205E17B50100130525BFD1B597E4FF1FF4
:1066400083C444FF97E7FF1F83C7B7FEA204DD8C16
:106650008327C9046D14228697E5FF1F938595FD56
:10666000280082978E0493160401B7750200C18238
:106670003000A6950D4597C0FF1FE780C0679307C0
:1066800080F8BDBF17B501001305C5BC9780010098
:10669000E780E06F1305C01297C0FF1FE780801DE1
:1066A000014597D0FFFFE780E0FD0D459700000012
:1066B000E78060D4294597C0FF1FE780A01B97C0E3
:1066C000FF1FE780000CF9B341114AC097F6FF1F86
:1066D00083D6E615328917D6FF1F0356C62022C47B
:1066E00026C206C62A84AE8497000000E780A05F19
:1066F00035C12DC0994763FF9704834714000347B2
:106700000400A207D98F13978700A183D98FC207EE
:106710003167C1831307C755639EE70297D7FF1FF1
:1067200083D7671CA301F400A1832302F40097F729
:10673000FF1F83D7C70F91C7A302F400A1832303D0
:10674000F400A68517B50100130545B69780010032
:10675000E780004C97F7FF1F83C707FDB9CF97D598
:10676000FF1F83D5451817B501001305E5B59780C0
:106770000100E780E0492686A28517D5FF1F035553
:10678000851697000000E78060C16301090497E760
:10679000FF1F83C727F99DCB95C897E7FF1F83C7C6
:1067A000A7E08DE722852244B2400249A6859244A3
:1067B0004101173300006700833E17B50100130540
:1067C000A5B197800100E780805CC1B7B240224448
:1067D0009244024941018280834755008345450028
:1067E00017B50100130545ABA207DD8D1783010026
:1067F0006700034217B50100130505A917830100BF
:106800006700E3588D4763FBB70A011126CA06CE1D
:1068100022CC0344350097E4FF1F83C4B4F097B53E
:106820000100938525ACB337800017E7FF1FA30B4A
:10683000F7EE09C497B50100938585AB17B5010044
:10684000130585AB97800100E780803C97E7FF1F29
:1068500083C757ED6386970097000000E7806026A6
:1068600097E7FF1F83C717EC8DC785472306F10005
:10687000B7E7040083A7471770008545130550301C
:10688000829717B50100130525A897800100E780BE
:1068900000509967938757EE2316F10068008547EB
:1068A0009145A30781002307F10097300000E7809E
:1068B000002FF2406244D244056182808280894781
:1068C00063F7B708011122CC06CE26CA83442500FF
:1068D00085472A84639DF404914763F5B704034513
:1068E00045008347340022055D8D97D7FF1F239C09
:1068F000A7FE97000000E780E0479967938767EE5F
:106900002314F1008347340023059100A305F1000F
:1069100083474400954528002306F1009730000086
:10692000E780E027F2406244D24405618280FDF8AE
:106930009967938767EE2314F10097D7FF1F83D7DA
:1069400087FAA305F10023050100A183E1B7828046
:106950000111996722CCD51717F4FF1F1304C4DC6B
:106960002314F1008347040026CA97F4FF1F938481
:1069700004EC2305F10083D7040028009545A30506
:10698000F100A18306CE2306F10097300000E780D6
:10699000002103D604008345040017B50100130548
:1069A000259897800100E780A026F2406244D244F7
:1069B000056182809D677971D9172316F10097F7D9
:1069C000FF1F83C767D606D62307F100A9C3B7E721
:1069D0000400FC47414697E5FF1F938565C31305F7
:1069E000F10082976800CD4597300000E780201BBA
:1069F00097F5FF1F83C545D317B5010013054595CE
:106A000097800100E780C020B25045618280B7E7DF
:106A10000400BC47414681451305F1008297D9B770
:106A2000B76702045D71938757AA3EC09307006061
:106A30002312F10097F7FF1F938707CF83C7070043
:106A4000A2C4A30301002303F10097F7FF1F93875C
:106A500007DE83D7070037E4040086C62314F1005D
:106A600097D7FF1F938727E883D707004146680021
:106A70002315F1007C4497E5FF1F938565B9829744
:106A8000F1450A8597000000E780E021231EA10060
:106A90007C448A850810794682973C441305E103BB
:106AA000094681458297101093050002014597D051
:106AB000FFFFE780A023B640264461618280B7C70C
:106AC000A55A01119387C7333EC497E7FF1F83C7B9
:106AD00077C53EC6B7F7070003C7070106CE22CC2D
:106AE000A5476313F70001A01164930504F0930612
:106AF00000100146254597C0FF1FE780C01F3000EA
:106B0000930504F0A146294597C0FF1FE780A01E0A
:106B100097E5FF1F83C515C117B50100130505943F
:106B200097800100E780C00EF240624405618280D8
:106B300001119165A1463000938505F02D4506CEE3
:106B400097C0FF1FE780201B2247B7C7A55A93872E
:106B5000C7336314F702B24517B501001305458327
:106B6000B335B00097E7FF1FA38EB7BA9780010037
:106B7000E780000AF24005618280814517B5010077
:106B80001305458397E7FF1FA38E07B89780010081
:106B9000E780000897000000E780A0F2E1BFB7C7D8
:106BA000A55A79719387F7353EC6B7E70400FC47CD
:106BB000AA8506D622D4414608088297B7F707006F
:106BC00003C70701A5476313F70001A011649305EC
:106BD00004E8930600100146254597C0FF1FE78093
:106BE00080117000930504E8D146294597C0FF1F26
:106BF000E780601017B501001305058A9780010032
:106C0000E780E018B2502254456182807971916525
:106C1000D1467000938505E82D4506D697C0FF1F25
:106C2000E780600D3247B7C7A55A9387F73517B588
:106C30000100130525806310F702B7E70400FC4745
:106C400017E5FF1F1305C59C41460C08829717A541
:106C500001001305257C97800100E7804013B250A6
:106C600045618280B7F7070003C70701A547631393
:106C7000F70001A09165411193060010014693852C
:106C800005E8254506C697C0FF1FE780C006B2404D
:106C900017A501001305056E410117830100670068
:106CA000030FC16769768146FD1705061397060134
:106CB00041836364B7003E8582803307D500034774
:106CC0000700B98F214713F8170085836305080073
:106CD000B18FC207C1837D171377F70F6DF7850654
:106CE000F1B741C5A547054763F2B70883471500CB
:106CF000034705003168A207D98F13978700A18346
:106D0000D98FC207C1831308C85505476390070789
:106D1000411106C622C426C203442500914763F0F0
:106D200087049307540063ECF502A301C500218298
:106D30002302C5009304340091C6A302D500A182AA
:106D40002303D5002A84A68597000000E780A0F5DC
:106D500026942300A4002181A300A4000147B2408F
:106D6000224492443A854101828005473A858280D7
:106D7000B7C7A55A01119387E7343EC42AC6B7F7AF
:106D8000070003C7070106CE22CC26CAA547631316
:106D9000F70001A091642A84938504EE9306001005
:106DA0000146254597C0FF1FE780E0F43000A1466B
:106DB000938504EE294597C0FF1FE780C0F3A285A5
:106DC00017A501001305856B97800100E78040E45B
:106DD00097000000E78000C5F2406244D24405619C
:106DE000828001119165A1463000938505EE2D4505
:106DF00006CE97C0FF1FE78000F02247B7C7A55A0D
:106E00009387E7346318F702B24517A5010013050D
:106E1000655C97D7FF1F2398B7ACC205C1819780E7
:106E20000100E780E0DE97000000E780A0BFF240AD
:106E300005618280D147D14517A501001305855B07
:106E400017D7FF1F2311F7AA97800100E78040DCC6
:106E500017D5FF1F035525A997000000E78080F193
:106E6000F9B7011126CA06CE22CC93F71500AE84DD
:106E70008DCBAD67371700409387A7AA1CC3B7E730
:106E80000400BC4F13060019854517D5FF1F0345A5
:106E900065A5829713C51400F2406244D24405618F
:106EA000828093F725006386071897A501009385D4
:106EB000A5622D46480097800100E78000CA97F53B
:106EC000FF1F83C5A596854793C4240063E5B704D7
:106ED0009DC9854517F5FF1F1305458597200000BF
:106EE000E780C0AD97E7FF1F83C7C78389CF97F5BA
:106EF000FF1F83C5A59317F5FF1F13052583973043
:106F00000000E780C0C91395040197F7FF1F238F86
:106F10000790418151B717F4FF1F0344248197F76D
:106F2000FF1F83C7B78022045D8CAD67C2059387BE
:106F3000B755C181630DF40C63E18704A96793879A
:106F4000A755630FF40C17E5FF1F1305257E972047
:106F50000000E780A0A697D7FF1F83C7A77CD1CFEB
:106F600097F5FF1F83C5858C17E5FF1F1305057C6B
:106F700097300000E780A0C249A0B1679387C7554A
:106F80006302F404B5679387D755E31EF4FA17E557
:106F9000FF1F1305A57997300000E78040C097F5E3
:106FA000FF1F83C5A588894763F9B704F915C20592
:106FB000C18117E5FF1F1305857797200000E78043
:106FC000E09F25A8054617E5FF1F1305257697F0D6
:106FD000FFFFE780A06F97E7FF1F83C7E77491EF7C
:106FE000480097800100E78040E393150501C181C7
:106FF000480097C0FFFFE780807DA28517A50100AC
:107000001305854B97800100E78080C0EDBD17E533
:10701000FF1F1305A57197F0FFFFE780207CF1BFEC
:1070200017E5FF1F1305857097F0FFFFE780C07C11
:10703000E9B793F745000145E38007E617A501008E
:107040001305C54897800100E78060D497300000A1
:10705000E78000C913C5440081B5411122C437E45B
:1070600004005C5C06C6354697A50100938505F1D2
:1070700017B50100130585B5829711E917A5010021
:107080001305454697800100E78060D001A0832763
:10709000041C82972A84054597C00000E780A083DE
:1070A00097600100E780C00897600100E780C0DDBD
:1070B00097B00000E78020952285B240224441012C
:1070C00082801567B71700401307575598C3D843F8
:1070D0009D66558FD8C3D843FD76758FD8C3D843E6
:1070E0001367F70FD8C335671307C7CC98C38280DF
:1070F00041111305800406C622C426C297B0FF1FA3
:10710000E780004E97000000E780C01A85457D5556
:1071100097C0FFFFE780802385457D5597C0FFFF1F
:10712000E780202D371400408327840A8D451305FE
:10713000002093E707202324F40A97C0FFFFE7808D
:10714000E020B7E4040097C0FFFFE780C06EC85896
:1071500097800100E780A0C317B50100130505A7BC
:1071600097800100E780A0C28327840C85454145B4
:1071700093E707082324F40C97C0FFFFE7806027FC
:107180008D451305000897C0FFFFE780802697C054
:10719000FFFFE780005C014597C0FFFFE780E05EEE
:1071A00085450545894717E7FF1F2303F76897C003
:1071B000FFFFE780205F37070004B7E700E023A068
:1071C000E71097D0FFFFE78020E597D0FFFFE7802B
:1071D00060F997000000E78080E897000000E780F2
:1071E000609597000000E78000C097E0FFFFE78010
:1071F000E0FA97000000E780601397000000E78046
:10720000A00D83A70408170500001305C5C58297C4
:1072100097C7FF1F2388A76CBC4C130600648545E5
:10722000829797000000E78000EA97B0FF1FE78091
:10723000606F01458280B7F7070003C70701A547C4
:10724000AE866316F7009397450191C301A0AA8506
:107250000146254517C3FF1F6700E3A94111B28608
:107260002E86AA852D4506C697C0FF1FE780A0A8D9
:10727000B2400145410182809307000463E8C702E0
:107280001D71A2CC2A84080886CE32C697800100E0
:10729000E780A08CB2461008A285294597C0FF1F41
:1072A000E78060A5F640664425618280395582807A
:1072B000054517C3FFFF6700C326411106C6971097
:1072C0000000E780C06EB240134515001375F50F3E
:1072D0004101828041110D658D4506C697C0FFFFB3
:1072E000E780C006B71700408D6623A6D70A17E5CA
:1072F000FF1F130525541387C70A9387870A1CC1EC
:107300005CC5856689675CC958C114C518C9B7E7EB
:107310000400B24003A3871E41010283B717004057
:107320000D6723A6E70A828097E7FF1F83C70752EE
:1073300099EF411106C697100000E7806061B240E6
:10734000854717E7FF1F2303F750410182808280A2
:1073500011C589C517C3FFFF6700634782804111CC
:1073600026C2AE848D4522C406C62A8497C0FFFF7C
:10737000E7802008B717004099C803A5C70C418DC6
:1073800023A6A70CB240224492444101828003A567
:10739000870C418D23A4A70CF5B78347050003474D
:1073A0001500A207D98FC2076177C187130727206D
:1073B000639AE700834525003705040017030000A2
:1073C000670023FA828017E6FF1F1306664881478D
:1073D000B2861303F00FA9483308F60003480800EB
:1073E00013F7F70F6307A80C630668008507E3959A
:1073F00017FF2947B387E6002380A70097E7FF1F01
:107400009387C7455DA8411113D76500134717003F
:1074100006C693F63500058B954791CA05469947F0
:107420006387C60009469D476383C600A14713F6DC
:1074300045003336C00093F68503050685C2A14595
:10744000638BB604E145638AB604930580026388C2
:10745000B604930580036393B600914697E5FF1F3A
:107460002383F56697E5FF1F238EC56497E5FF1F0D
:10747000A38AD564BE8517A5010013052510977052
:107480000100E780E078B240854717E7FF1FA30CB3
:10749000F762410182808546D1B78946C1B78D46E2
:1074A00075BF17A501001305E50F177301006700ED
:1074B000237617E7FF1F1307673ABA972380B700B1
:1074C000E147E302F5F493077002E30CF5FC8280D8
:1074D0002A8723800500814717E5FF1F13054537DD
:1074E0001308F00F2946B306F50083C6060063961D
:1074F000E60297E6FF1F93866636B69783C70700B6
:1075000005452380F5009947636EF7029D4763FDAB
:10751000E700E147630DF700828063850601850778
:10752000E393C7FC0145C5B7238005008280B737C8
:10753000004003C7370083C7050093F70704D98FBE
:107540002380F5008280797126D24AD097E4FF1F0C
:1075500083C4446917E9FF1F1309096806D622D4BA
:107560004ECE52CC56CA5AC8B307990083C70700FB
:1075700093F7F70FA5C79387140093F7F70F0D47FD
:107580006361F70C17E7FF1F230EF76497E7FF1FF0
:1075900093870765A69783C707001307100293F721
:1075A000F703638FE7286363F70A05446380872046
:1075B000E389076E09476389E71413070002E38E26
:1075C000E758B7E700E03707400023A0E7180100BD
:1075D0000100CA942380040023A0E710B78700406D
:1075E00003C76700058BE30F077897E6FF1F83C685
:1075F000865F0547E39AE67629472381E702094734
:107600002383E7022385E70297E7FF1FA38E074A3C
:1076100097E7FF1FA389075CB7870040A381070096
:1076200017E7FF1FA304074A05472383E700B2506B
:10763000225492540259F249624AD24A424B45615D
:10764000828097E7FF1F238F075889B713073002FF
:107650006386E70A63E6E71413074002638AE708D4
:1076600013070003E39FE7F497E7FF1F938707578C
:10767000A69703C70700A1471377F70FE31AF71C74
:1076800017EAFF1F130A4A1E83476A0097E6FF1F87
:107690002382F64297E7FF1F83C7771D91C7FD57E7
:1076A00097E6FF1F2388F64097E5FF1F83C5D51B8C
:1076B00097E7FF1FA380B74097E7FF1F83C7C71A4D
:1076C00093F907089306000493F707066393D752CC
:1076D0009307A009638DF51A63EAB7169307F005BF
:1076E000638AF54E930750096388F52E014479AB00
:1076F000FD5717E7FF1F230EF73AE1B5FD5717E7D0
:10770000FF1F2307F73A75BD17A50100130505FBF9
:1077100097700100E780A06797E7FF1F9387074CEA
:10772000A69703C40700814917EAFF1F130A4A2CD2
:107730001374F40F97AA0100938ACAF863C78904E7
:10774000294597700100E7808051854717E7FF1FA3
:10775000A30EF72817E7FF1F230B872817E7FF1F44
:107760002304F73637E700E0B70640002320D71898
:1077700001000100378600408347A60293F7370FC8
:107780002305F6022320D7102DBDB3073A0183C588
:1077900007005685850997700100E780604779BF2B
:1077A000854717E7FF1F2303F72421BD17A5010015
:1077B0001305C5F097700100E780605D97E7FF1F34
:1077C0009387C741A69703C40700814917EAFF1FA3
:1077D000130ACA151374F40F97AA0100938A8AEE4C
:1077E00063C58904294597700100E78040478547B4
:1077F00017E7FF1FA30AF71217E7FF1F23078712D8
:1078000017E7FF1F2302F72C37E700E0B706400019
:107810002320D71801000100378600408347660205
:1078200093F7370F2303F602B1BFB3073A0183C5BD
:1078300007005685850997700100E780603D4DB7C8
:10784000854717E7FF1F2301F70EA5BB9307400AE3
:10785000638DF5349307200B6388F5369307100A80
:10786000E396F5E883072A00014463D1074297E7CE
:10787000FF1F83C797FF93F63700638E061A0546EE
:10788000638EC62209466399C61A1D4775A217E57D
:10789000FF1F034585FDC94717EAFF1F034AFAFC8E
:1078A00097E5FF1F83C585FC17E4FF1F034414FC05
:1078B0006319F510CD476316FA1093077008639C9F
:1078C000F5021307300FB7170E006308E400130723
:1078D000900DB7B704006314E40817E7FF1F2321D6
:1078E000F71EBE8517A50100130545DE9770010040
:1078F000E7800032E5BB93078008639DF500330401
:107900008040B77746001374F40F938787CDB3D7C1
:107910008702E1B793079008639AF500330480402B
:1079200091671374F40F9387C766D5B79307A008C0
:10793000639BF50033048040B7173D001374F40FC8
:1079400093870790E9B79307B008639AF50033046B
:10795000804091671374F40F938797D04DBF93F5D0
:10796000F5078D47639BF50033048040B7975B00B4
:107970001374F40F938707D859BF8947639BF500A9
:1079800033048040B7770B001374F40F9387071B01
:10799000BDBF8547639AF50033048040DD671374EB
:1079A000F40F938767E3A5B789E9330480408D67B7
:1079B0001374F40F938777DC99BFF16793870720DF
:1079C00029BF97000000E78040A0A285528597005C
:1079D0000000E780809F19BB9305610017E5FF1F3A
:1079E0000345A5E817E4FF1F034434E897000000AF
:1079F000E78040AE93057100228597000000E78084
:107A000060AD3C0017E7FF1F2326F71C834761008A
:107A10002304F10083477100A304F100894717E7AD
:107A2000FF1F2309F7088357810017E7FF1F231D56
:107A3000F7E20944A1AC154793F64700B336D000EE
:107A400093F78703850685C32146638BC706614686
:107A5000638AC706130680026388C706130680037D
:107A60006393C700914717E6FF1F230DD60497E6DF
:107A7000FF1FA389F60497E7FF1F2386E70417E794
:107A8000FF1F0347A7DE9376070497E7FF1F83C70F
:107A9000F7DD8DEE1377770C93067008630CD70231
:107AA0001377F7078D46631ED70AB307F040B795E3
:107AB0005B0093F7F70F938505D881A81947ADBFF1
:107AC000854755B7894745B78D4771BF93067008FD
:107AD0006311D7021307300FB7150E006389E70251
:107AE0001307900DB7B504006383E702130770080E
:107AF00045BF9306800C6311D702B307F040B775FA
:107B0000460093F7F70F938585CDB3D5F50297E738
:107B1000FF1F23A7B7FAF9B39306900C631AD70097
:107B2000B307F040916593F7F70F9385C566F1BFF2
:107B30009306A00C631BD700B307F040B7153D00B8
:107B400093F7F70F93850590C9B79306B00CE31927
:107B5000D7F4B307F040916593F7F70F938595D06D
:107B60006DB78946631BD700B307F040B7750B00AC
:107B700093F7F70F9385051B49BF8546631AD70016
:107B8000B307F040DD6593F7F70F938565E3B5BF65
:107B900009EBB307F0408D6593F7F70F938575DC1C
:107BA000ADB7F165938505209DB783472A00C18B4A
:107BB00099C7854717E7FF1F2301F7F005BE97E731
:107BC000FF1F238C07EE1DB6854717E7FF1FA30C89
:107BD000F7EE29BE3C0017E7FF1F232DF7FE0947EC
:107BE000930700032314F10097E6FF1F2384E6ECBC
:107BF0002DBD639A0758A94763ECB74417A7010046
:107C0000130707958A05BA959C41BA97828717E4AE
:107C1000FF1F034494C5094A630C440F636C8A0830
:107C200085476309F40A9307F00F17E7FF1F03471F
:107C300067E863F6E70017E7FF1F230DF7E617EA8B
:107C4000FF1F034A2AE7930700041374FA0F63F433
:107C500047011304000497E7FF1F9387A7F783AA40
:107C60000700228617E5FF1F130505C0D685330AD6
:107C70008A40A29A97700100E78020EE97E7FF1FE5
:107C8000238A47E397E7FF1F23A657F597E7FF1FD0
:107C900083C757E21547639AE762B7E700E0370703
:107CA000400023A0E71801000100B78600402380B0
:107CB00086028DA58D47630CF40A9947E315F4F607
:107CC00097A701009387478F17E7FF1F2324F7F03B
:107CD000A947A1BF17E7FF1F0347E7F097E7FF1F7B
:107CE000938747DF494697A501009385E59563068D
:107CF000870097A50100938525913E859770010027
:107D0000E780A0E517E7FF1F2326A7ECC94731BF8F
:107D100097E6FF1F83C626ED054797E7FF1F93876A
:107D200067DB6394E6023E851306700297A50100A7
:107D30009385058F97700100E78020E217E7FF1F0A
:107D4000232AA7E893077002CDB53E8513063004B9
:107D500097A501009385058797700100E780E0DF14
:107D600017E7FF1F2328A7E6930730047DBD97E59B
:107D7000FF1F83C585AF17A5010013056596977092
:107D80000100E780E0E8854A17EBFF1F034BABE5F6
:107D900097E5FF1F83C565AD17A501001305459441
:107DA00063185B0B97700100E78080E697E7FF1F81
:107DB00083C7A7ABB5CBE368F4E617A401001304AF
:107DC000E48C638C670117A401001304A48C638600
:107DD000470117A401001304648D228597700100E8
:107DE000E780A0031375F50F93071500860717E7C3
:107DF000FF1F2301F7CE8D4717E7FF1FA30CF7CC1A
:107E000097E7FF1F938707CD0147BE861376F70FCD
:107E100089076365A60297E7FF1F23ADD7DA97E7C7
:107E2000FF1F83C727CB11B5979701009387077F63
:107E300017E7FF1F2320F7DA9147C5BB3306E4009D
:107E400003460600A380070005072380C7007DBF07
:107E500097700100E780C0DB97E7FF1F83C7E7A0AB
:107E6000E1D7E362F4DC179401001304247F638CF0
:107E70005701179401001304E47E638647011794A9
:107E800001001304A47F228597700100E780E0F8C9
:107E90001375F50F93071500860717E7FF1F230BD0
:107EA000F7C28D4717E7FF1FA306F7C297E7FF1F2B
:107EB000938747C20147BE861376F70F8907E37C95
:107EC000A6F43306E40003460600A3800700050776
:107ED0002380C700D5B797E5FF1F83C5059917A570
:107EE00001001305A58097700100E78060D297E735
:107EF000FF1F83C7F7BD93E7470017E7FF1FA309DD
:107F0000F7BC83472A0017E7FF1FA301F7BC6FF0F8
:107F1000EFFD179501001305A57E97700100E7801E
:107F200000E797E7FF1F938767BA83C7070017E744
:107F3000FF1F230BF79217E4FF1F0344A4B733344A
:107F40008000A9B3179501001305C57C9770010047
:107F5000E780E0E397E7FF1F83C797B793E7070141
:107F600017E7FF1FA306F7B683472A0017E7FF1F8F
:107F7000230EF7B46FF08FF7179501001305C57A3C
:107F800097700100E780A0E003470A007D8B51EF66
:107F9000B787004003C767021377C70B1367270033
:107FA0002383E70203C7A7021377C70B13672700D2
:107FB0002385E70203C7E7021377C70B1367270080
:107FC0002387E70203C727031377C70B136727002D
:107FD0002389E702854717E7FF1F2307F79417E771
:107FE000FF1F2305F7A017E7FF1F2303F7AC17E7D1
:107FF000FF1F2300F7AC97E7FF1FA387079297E7C0
:10800000FF1FA385079E97E7FF1FA38307AA97E794
:10801000FF1FA38007AA97E7FF1FA38707AA97E779
:10802000FF1FA38207BC6FF06FEC89476312F70252
:1080300097E7FF1F83C787839146638CD70863E068
:10804000F604638EE70C6369F70A05476380E70E61
:10805000FD5717E7FF1FA30FF7A437074000B7E747
:1080600000E023A0E71801000100B78600401306D6
:10807000F0FC2381C60223A0E7106FF08FD4130712
:1080800020086382E7086362F70213071008E39190
:10809000E7FC378700408347670293F7C70B93E7F6
:1080A00027002303F7026FF06FE41307300863899A
:1080B000E70213074008E39DE7F83787004083474E
:1080C000270393F7C70B93E727002309F7026FF005
:1080D000EFE1378700408347270393F73707F5B76A
:1080E000378700408347E70293F7C70B93E72700E2
:1080F0002307F7026FF08FDF378700408347E702DF
:1081000093F73707F5B7378700408347A70293F700
:10811000C70B93E727002305F7026FF02FDD3787A2
:1081200000408347A70293F73707F5B7378700402A
:108130008347670293F73707ADB71795010013051B
:10814000A55F97700100E78080C497D7FF1F238D3C
:108150000770D5B3179501001305055F97700100EF
:10816000E780E0C297D7FF1F2390077097E7FF1FB4
:108170009387479403C40700894763F38700094442
:108180001374F40F21B613070002E393E7EC63992D
:10819000090A638FF500930720026381F50817959C
:1081A00001001305E55D97700100E78060A64DB5FD
:1081B000179501001305055A97700100E78020BD4F
:1081C0000144179B0100130B2B5AA14AB3078A00E5
:1081D00083C507005A85050497700100E78040A316
:1081E000E31654FF179501001305C5B697700100FB
:1081F000E780E0B917D4FF1F0344446711E497D721
:10820000FF1F2386076459B48947E313F4E48547C5
:1082100017D7FF1F230DF7626FF04FCD17D6FF1F43
:108220000346B66497D5FF1F83C5256417950100E3
:108230001305055497700100E780809D6FF00FCB08
:10824000638FF50493071002E39BF5F497D5FF1FA6
:1082500083C5C5611795010013058553977001000B
:10826000E780009B97E7FF1F23A6479797E7FF1F2D
:1082700093870785944383D7470017E7FF1F03477A
:10828000878417D6FF1F2321D65E1D4497D6FF1F74
:10829000239EF65C97D7FF1F238BE75CC5BA97D563
:1082A000FF1F83C5A55C179501001305E54F977067
:1082B0000100E780E09597D7FF1F238A075897D7DB
:1082C000FF1F2393075A6FF0CFF62547E387E79CFC
:1082D00019476391E702B786004023808602B7E71B
:1082E00000E03707400023A0E71801000100130653
:1082F00000FC41B31307100A6391E702B786004000
:1083000023808602B7E700E03707400023A0E71884
:1083100001000100130680FCA9BB1307A009E38F2D
:10832000E7FC1307400AE38BE7FC13072002E38610
:10833000E7960547E383E796B7E700E03707400095
:1083400023A0E718E391099601000100B7860040D9
:1083500023808602130620FC29BB17D7FF1F034783
:1083600077756308F71E63E7E7029547630EF70E1C
:1083700099476308F704B786004023800602B7E7F1
:1083800000E03707400023A0E718010001001306B2
:10839000A0FCC5B19307F005630AF70093075009E5
:1083A0006306F70093071002E317F7FCB7E700E056
:1083B0003707400023A0E71801000100B7860040FE
:1083C00051BF97D9FF1F83C9E96E93070004CE8A76
:1083D00063F43701930A000497D7FF1F9387877FC1
:1083E00003AA070013F4FA0F2286D28517D5FF1FC0
:1083F0001305854797600100E7802076B3878940A1
:10840000529417D7FF1F2307F76A97D7FF1F23A39D
:10841000877C638E0902B787004023805703B7E645
:1084200000E03706400023A0C6180100010003C782
:108430002702134707042381E70203C727021377A4
:10844000C70F2381E70223A0C6106FF08F97B7866E
:10845000004023800602B7E700E03707400023A072
:10846000E71801000100FDB537870040834737005A
:1084700097D6FF1F83C6966593F70708D58FA3018C
:10848000F700B7064000B7E700E023A0D7180100C7
:1084900001001306A0FC2301C70223A0D7106FF030
:1084A0004F9297D7FF1F93876773A69783C70700DD
:1084B00093F7F70FD9CF97D7FF1F83C7C772D1EBB9
:1084C00017D7FF1F0347175F930700026313F708CF
:1084D00097D7FF1F9387473903AB070097DAFF1F32
:1084E00083CACA3817DAFF1F034A5A3897D9FF1FC1
:1084F00083C9E937D2875687CE865A8697D5FF1F1C
:1085000083C5E534179501001305852B976001009D
:10851000E780007097D7FF1F23A4675B97D7FF1FE3
:108520002382575B97D7FF1FA38E475997D7FF1F0B
:10853000238B375997D7FF1FA38A8730B7E700E00F
:108540003707400023A0E71801000100B78600406C
:10855000D1B3B7E700E03707400023A0E7180100D8
:108560000100B786004025B529472381E702094766
:108570002383E7022385E7022387E7022389E702B3
:108580006FF08F8803C76700118B6302078A83C768
:108590005700918BB5CF17D7FF1F0347C764854797
:1085A0006313F70697D7FF1FA38FE75097D7FF1FD7
:1085B000238C073697D7FF1F238A074297D7FF1FC1
:1085C0002388074E97D7FF1F2385074E97D7FF1F96
:1085D000A38C073497D7FF1FA38A074097D7FF1FA5
:1085E000A388074C97D7FF1FA385074C97D7FF1F7A
:1085F000A38C074C97D7FF1FA387075EB787004060
:1086000011476FF08F8217D7FF1FA301F72479BF9F
:10861000854717D7FF1F2309F73017D7FF1F2307F9
:10862000F73C17D7FF1F2305F74817D7FF1F230273
:10863000F74869BF854717D7FF1F2307F72E17D7BE
:10864000FF1F2305F73A17D7FF1F2303F74617D756
:10865000FF1F2300F74617D7FF1FA307072C17D7C5
:10866000FF1FA305073817D7FF1FA303074497D79A
:10867000FF1FA38007448280411106C697000000B7
:10868000E78080FBB787004023800700130740FC8A
:108690002386E7001307C004A386E70017D7FF1F50
:1086A0001307871C2398E70017D7FF1F1307C71F5F
:1086B000239AE70017D7FF1F1307472B239CE700D8
:1086C00017D7FF1F1307C736239EE70029472381CB
:1086D000E70209472383E7022385E7022387E702AE
:1086E0002389E702A3810700930600F8A380D7003F
:1086F000930690022380D700FD562383D700238161
:10870000E700B706400037E700E02320D71003C793
:10871000170013671700A380E700B24097D7FF1F29
:108720002396073A41018280411106C69700000056
:10873000E78080F0B787004023800700130700FC24
:108740002386E7003147A386E70017D7FF1F1307EB
:10875000A7112398E70017D7FF1F1307E714239AE1
:10876000E70017D7FF1F13076720239CE70029475F
:108770002381E70209472383E7022385E702A381D8
:108780000700930600F8A380D70093069002238089
:10879000D700FD562383D7002381E700B7064000AA
:1087A00037E700E02320D71003C71700136717002F
:1087B000A380E700B24097D7FF1F239907304101FC
:1087C0008280F1679387072017D7FF1F232AF72E90
:1087D000854717D7FF1F2317F72EA14717D7FF1F6E
:1087E0002303F72E97D7FF1FA38F072C97D7FF1FC1
:1087F000238C072C97D7FF1F238B070497D7FF1FC6
:10880000A3860704814717D5FF1F13056504FD558F
:1088100017D6FF1F130686042947B306F5002380E9
:10882000B600B306F600238006008507E397E7FE4F
:1088300097D7FF1F2382073A97D7FF1FA38E0738CA
:1088400097D7FF1F238B073897D7FF1FA3850726CE
:1088500097D7FF1FA383072697D7FF1F238E0724D1
:1088600097D7FF1F2389072497D7FF1F2388072443
:1088700097D7FF1FA382072497D7FF1F238F0722B5
:1088800097D7FF1FA38B0734828017D7FF1F03479B
:10889000873585476316F70017030000670003E973
:1088A00017030000670083DD411122C406C617D7F5
:1088B000FF1F0347473385472E8613F4F50FAA851C
:1088C0006317F70417D5FF1F1305450E97600100C6
:1088D000E780A02897D7FF1F238A0710B78700409B
:1088E00023848702B7E600E03706400023A0C618BD
:1088F0000100010003C7A7021377C70F2385E70212
:10890000B240224423A0C61001454101828017D500
:10891000FF1F130565FD97600100E780002497D7CE
:10892000FF1F23830700B787004023828702B7E633
:1089300000E03706400023A0C6180100010003C76D
:1089400067021377C70F2383E7025DBF411106C695
:1089500097000000E78020E7B240410117030000C4
:108960006700E3F2411106C697F0FFFFE780E0BD24
:1089700097D7FF1F83C757FB95C797D5FF1F83C5A1
:10898000C5FA89C917D5FF1F130545FA97F0FFFFF0
:10899000E780409C97D7FF1FA38807F897D7FF1F52
:1089A00023840712B2404101828017D5FF1F03457F
:1089B000E5113335A000828041C9D9C597D7FF1F83
:1089C00083C7C710D1C3011122CC4AC84EC656C2B4
:1089D0005AC006CE26CA52C42E89AA890144930AD7
:1089E0000004371B030063772403B3078940C207E1
:1089F000C183BE8463F4FA0093040004C204C180FE
:108A0000130A1BD497D7FF1F83C707F29DE37D1A74
:108A1000631C0A00F2406244D2444249B249224AED
:108A2000924A024B0561828097F0FFFFE780E0B138
:108A3000D1BF338589002694A685420497000000A3
:108A4000E780C0E6418045B7828097D7FF1F9387B4
:108A5000271D18429C4383D645000345070083C564
:108A6000C700035646006396A50083D5E700638DD3
:108A7000D502011106CE2386A7002397D700B7059C
:108A8000CF00DC4B9385757D05077D162EC2230034
:108A900001003AC42316C1002317D10099C30A85E7
:108AA0008297F240056182808280DC4DDC4B81CF71
:108AB000B7E70400904503A38705914517D5FF1F2D
:108AC00003454516028382806D713C083EC6B70798
:108AD000E500232291103EC8AA843C083285232653
:108AE00011103ECA23248110232021112E89973092
:108AF0000000E780405C2A84979501009385C5CFEC
:108B000017850100130545BE97600100E7804010FE
:108B1000A285179501001305A5DE97600100E78087
:108B2000200F294597600100E7806013B705CB004F
:108B30009385757D680097100000E7806065A285C9
:108B4000680097300000E780604901478146700067
:108B5000CA85268597200000E780E08805CD2A8415
:108B600097950100938545C9178501001305C5B781
:108B700097600100E780C009A285179501001305E1
:108B8000E5D897600100E780A008294597600100BB
:108B9000E780E00C8320C11003248110832441105E
:108BA000032901105161828097D7FF1F93874707E0
:108BB00018429C43797122D406D60348070083C823
:108BC00007012A8483D645000355460063960801B1
:108BD00083D82701638DD8022388070105072399CD
:108BE000D7003708CC00DC4B1308787D3ACC13074C
:108BF000F5FF42CA23080100231EE100231FD10014
:108C000099C7080832C62EC482973246A2452285EB
:108C100097000000E78080EBB250225445618280CB
:108C20006D713C083EC0B707E5003EC23C083EC43B
:108C300023261110232481102322911023170100D1
:108C40002318010023190100231A0100231B01002E
:108C500097B7FF1F83D787CB99E3C167FD1723160B
:108C6000F10097B7FF1F83D787CA91EB97D7FF1FF4
:108C7000938707FB9C439C43DC4783D7070017B4CB
:108C8000FF1F1304A4C8584C2317F1008357440056
:108C9000484B2318F10031E1979501009385C5BC3D
:108CA00017850100130545A497600100E78040F691
:108CB00017950100130585BC97600100E78040F51A
:108CC000294597600100E78080F98320C1100324C3
:108CD0008110832441105161828097B7FF1F83C7A1
:108CE00057C389EBB7E70400BC5782975C4C23AAB3
:108CF0000700E1BFFD1797B6FF1FA38CF6C0035610
:108D00000701834704014C470A85230BF100973084
:108D10000000E780C02997D7FF1F938767F09C4327
:108D20000147814688430A866C0097100000E7805F
:108D3000806BAA8429C1979501009385E5B21785B8
:108D400001001305659A97600100E78060ECA68535
:108D500017950100130545B397600100E78040EBCC
:108D6000294597600100E78080EF584CB7E7040081
:108D7000BC57484B9DBF97B7FF1F83C797B9F5D71F
:108D8000B7E70400BC4F1044854517D5FF1F0345C6
:108D900065E982971DBF5C4EDC4BB9CFB1CD411167
:108DA00022C417850100130525942E849795010090
:108DB0009385C5A906C697600100E78060E5A28596
:108DC00017950100130505AF97600100E78040E4A7
:108DD000294597600100E78080E8B7E70400224456
:108DE000B24003A3870517D5FF1F0345A5E313066C
:108DF00040069145410102838280411122C417B48B
:108E0000FF1F130464AE1C4C06C689C7DC4399C31C
:108E10004C488297584CB7E70400BC57484B8297A0
:108E20005C4CB240224423AA07004101828017B75C
:108E3000FF1F130767AD834707009306F00B8507F5
:108E400093F7F70F63E9F60097B6FF1F238EF6AA94
:108E5000034507008280930700F8FDB7835745005C
:108E60006386071001114AC817B9FF1F130909AA21
:108E700052C4032AC90106CE22CC03274A0126CABE
:108E80004EC656C2F15735E31307D00DFD57636E3A
:108E9000C704B7E9040083A709072A8413058600DD
:108EA00042054181B284AE8A8297232AAA00032513
:108EB000C9015C49A9E79795010093852597178516
:108EC00001001305658297600100E78060D4179563
:108ED0000100130565A697600100E78060D329456E
:108EE00097600100E780A0D7DD57F2406244D2448A
:108EF0004249B249224A924A3E850561828093875F
:108F00004400B705CF002319F5009385757D310521
:108F100097100000E780C0270325C901834564003E
:108F2000310597300000E780600B0325C9012686D4
:108F3000D685310597300000E78060077146A2852D
:108F40004A8597600100E78040C1504419CA83A751
:108F50008905854517D5FF1F0345C5CC82978147F5
:108F600069B797000000E780E0CBD5BFFD573E858D
:108F70008280411126C297B4FF1F93842499D84C54
:108F800022C437E404003C54484B06C68297DC4CAC
:108F90000323C4052244B240924423AA070017D5F4
:108FA000FF1F034525C8854541010283411126C2A3
:108FB00097D4FF1F9384C4C69C4006C622C44AC0EF
:108FC000D5C3DC43C5C35CC12300B5002A84979593
:108FD00001009385E580177501001305E570976022
:108FE0000100E780E0C2294597600100E78020C7C3
:108FF0009C4023A4070023A2070097B7FF1F938775
:10900000A78EDC4FDC4B91C7295597000000E78005
:1090100000DF97B7FF1F9387678FDC4FDC4B89C753
:1090200097000000E78020F537E904008327C90591
:10903000894517D5FF1F0345E5BE82978327C905DC
:10904000914517D5FF1F0345E5BD82979C4003A3BB
:1090500047016309030022852244B2409244024939
:1090600041010283B240224492440249410182807C
:109070000111328506CE22CC26CA2E8497300000FC
:10908000E7806003AA84978501009385A57817750A
:1090900001001305656597600100E78060B703076D
:1090A00084000356640083554400A686179501008A
:1090B0001305458297600100E78080B529459760D8
:1090C0000100E780C0B997B7FF1F83C74782639D40
:1090D0009700014597000000E78060D281450A852E
:1090E00097000000E780C0ECF2406244D244056182
:1090F00082806D7123248110232611102322911068
:1091000093F745002E84638707143C083EC0B707D9
:10911000E5003EC23C083EC42317010023180100AD
:1091200023190100231A0100231B010097A7FF1F29
:1091300083D7877B99E3C167FD172316F10097A7B3
:10914000FF1F83D7877A91EB97D7FF1F938747AD90
:109150009C439C43DC4783D7070017A7FF1F1307D7
:10916000A7782317F100544F835747002318F100C5
:10917000DC4AA1E7978501009385056E177501000C
:109180001305855697600100E78080A817850100C8
:109190001305C56E97600100E78080A72945976099
:1091A0000100E780C0AB134544008320C1100324B5
:1091B0008110832441105161828097A7FF1F83C7CC
:1091C00017732555D9C3FD1717A6FF1FA301F67204
:1091D00003D6060183470701CC460A85230BF1001D
:1091E00097300000E780A0DC97D7FF1F938747A345
:1091F0009C4317A7FF1F1307276F978601009386CD
:10920000E66A88430A866C0097100000E780A01D7C
:10921000AA8451D9978501009385056417750100CB
:109220001305854C97600100E780809EA685178511
:1092300001001305656597600100E780609D294581
:1092400097600100E780A0A1268597000000E780D5
:1092500000BB91BF93F725009DC7B7E70400BC474B
:109260004146814528088297255597000000E780F0
:1092700000B928089305F00F97000000E78040D35D
:10928000134524001DB793F71500014599DF97009A
:109290000000E78020991345140001BF5C4D411187
:1092A00006C688C317D7FF1F232CF796B7E704001D
:1092B00083A70708170500001305E5E38297B2406E
:1092C00097D7FF1F2380A796014541018280011196
:1092D0009307700F2316F10006CE97D7FF1F83C7A1
:1092E000F7958DE7B7E7040083A7870D17A6FF1F43
:1092F0000346C6646C0017D5FF1F0355659482971B
:109300003335A00097D7FF1FA38AA792F2400561CB
:10931000828041119397050122C406C626C2C187E7
:109320002E8463D40702B7E40400FC5417A5FF1F82
:109330000345C560829719C1BC5482972165218D70
:10934000B240224492444101828093F715008DC7B8
:10935000B7E7040083A7471A17A6FF1F1306065D89
:1093600097D5FF1F9385C58C17A5FF1F0345055D86
:10937000829713451400E9B793F7250099CFB7E713
:109380000400BC4F13060064894517A5FF1F034561
:10939000E55A82971345240065B793F785009DC76A
:1093A000B7E7040003A8871A1307401F97A7FF1FFA
:1093B00083C7C758914613060003E14517D5FF1F21
:1093C000035505880298134584009DBF93F7450017
:1093D0000145BDD7B7E4040083A7041817D5FF1FC4
:1093E000035505868297BC4C13060064914517A56A
:1093F000FF1F0345A55482971345440091B797D7A3
:10940000FF1F83D7E7836398A70217D7FF1F231A8D
:10941000B78217D7FF1F2317C78217D7FF1F231441
:10942000D7822E861785010013050568BE85175360
:1094300001006700E37D1785010013056568176368
:1094400001006700C39403574500011106CE22CCEA
:1094500097C7FF1F83D7C77E178501001305456691
:109460006310F706C167F91717C7FF1F232AF77C98
:1094700037E4040097C7FF1F23A6077C7C4C89456F
:1094800017A5FF1F0345854B82977C4C914517A577
:10949000FF1F0345A54A829797B7FF1F83C79728E9
:1094A00085CB8547A307F100832744171306F100F6
:1094B00085451305503082971785010013058554A3
:1094C00097600100E780A08CF240624405618280D1
:1094D00097C7FF1F83C74725178501001305455709
:1094E000E5F38547A307F100832744171306F1002E
:1094F0008545130550308297178501001305C55225
:10950000C1B77D15954763E0A71C178701001307B6
:10951000274C0A053A951C41011122CC06CE26CAD9
:10952000BA972E848287178501001305E559976045
:109530000100E780C0851DAA03C725009947631174
:10954000F7022E8597000000E78020F08345640035
:10955000178501001305455897500100E780406BBF
:1095600097B7FF1F2380071C178501001305855837
:109570007DBF03C7250095476319F702C16717C769
:10958000FF1F0357E76BF91703D5A5006309F7021F
:10959000B7E7040083A7C717829717850100130553
:1095A000655697500100E780807E854717B7FF1FFB
:1095B000230AF71617850100130545578DBF97C776
:1095C000FF1F239FA76683D7E500B7E40400096661
:1095D00017C7FF1F2317F76683D7050113060690E9
:1095E00017A5FF1F0345853517C7FF1F231CF76409
:1095F00083D72501A14517C7FF1F2316F764BC4C6D
:109600008297BC4C13060064914517A5FF1F0345C4
:10961000E53282970356E4008355A40017850100C4
:109620001305854F97500100E780805EBDBF178509
:10963000010013056550E5BD83C525009147639C76
:10964000F50285471785010013058550A307F10032
:1096500097500100E780A073B7E7040083A747177E
:109660001306F1008545130550308297F24062449D
:10967000D2440561828099476392F5022285970062
:109680000000E78080DC8345640017850100130536
:10969000A54497500100E780A057C9BF9547639F35
:1096A000F50083471400178501001305654AE39010
:1096B00007E8178501001305654B95BD1785010067
:1096C0001305454BF9B782806D7123248110232641
:1096D000111023229110328401CD8947630AF502CB
:1096E0008320C110032481108324411051618280A2
:1096F000178501001305C548AE8497500100E78027
:109700000069A285268597C0FFFFE780E061C9BF99
:10971000B7E70400FC47280082971785010013056E
:10972000E54697500100E78080668347810039C491
:109730001307000B6380E7021387A7051377F70F62
:109740008D4663EDE602A285280097D0FFFFE780F3
:10975000C0D079B78547E3F587F883459100177541
:1097600001001305A52DB335B00097B7FF1F238D5A
:10977000B7E297500100E780A0499DB703479100E9
:10978000A207D98F35671307D7556385E708636844
:10979000F7022D671307B7556387E706316713078D
:1097A000C755638AE70429671307A7556394E7023F
:1097B000A285280097D0FFFFE780000415B739671E
:1097C0009306E765638DD70663E9F6001307E7554F
:1097D0006380E706A28528003DB73D679306F755ED
:1097E0006386D7061307F766E396E7FE97D0FFFF79
:1097F000E780801CF5B50146A285280097D0FFFFC1
:10980000E780C0ECF1BDA285280097D0FFFFE7807C
:10981000E0FCF9B58947E3F587EC9305E4FFC20561
:10982000C1811305A10097A0FFFFE78040FA4DBD5D
:10983000A285280097D0FFFFE78000FD55B5A285DF
:10984000280097D0FFFFE780C00759BD97D0FFFFE2
:10985000E780401071B5411122C417A4FF1F130403
:10986000240FAA8617860100130606182285C14513
:1098700006C697500100E780C0520357440097A7DF
:10988000FF1F9387E70D2393E7000357640023949A
:10989000E700B240224441018280011106CE22CC71
:1098A00097000000E78060FB37E4040083278414FE
:1098B00017A6FF1F1306C609D545014582978327C2
:1098C00084179305F1001305503082978347F10008
:1098D000A1C7A3070100832744171306F10085459C
:1098E0001305503082978327441717A6FF1F1306CE
:1098F0002607CD451305703082978547A307F100F1
:10990000832744171306F1008545130550308297CD
:10991000F2406244056182808327441717A6FF1F27
:1099200013060604CD4513057030D5B761712324A5
:10993000811A37E40400832704082326111A2322FE
:10994000911A2320211B232E31191705000013051E
:10995000859C829717A9FF1F130949FEE14785449B
:109960002300A900231CF100978501009385C510F1
:109970009307000317750100130505D7231CF10891
:109980002308910097C9FF1F938969EA9750010046
:10999000E780002883D50900178501001305850598
:1099A00097500100E780C026294597500100E780C5
:1099B000002B03D50900856997000000E780E0E9E6
:1099C0008327441710088545130550308297832755
:1099D000441717A6FF1F1306A6F8CD4513057030D0
:1099E00082978327441717A6FF1F130666F5B54510
:1099F0001305603082978327441730088945130583
:109A00001031829783274417300989451305203187
:109A1000829783274415938509C80D45829783272C
:109A20004415938509C811458297A3059100230623
:109A300091002308910002CD230C01008327841696
:109A400030099145130570408297832784161306C9
:109A5000B100854513050040829783278416700066
:109A60008545130510408297832784163008854565
:109A70001305204082978327841610088545130517
:109A800050408297832704157D558297832744137E
:109A90007D5582977D5597A0FFFFE780001E8327A5
:109AA000440C829797A0FFFFE78040F98327841436
:109AB00017A6FF1F1306C6E9D545014582978947BA
:109AC0001306700F814528092306F1009790FFFFC8
:109AD000E78020B58D471306000881452808230C30
:109AE000F1089790FFFFE780C0B39147230CF10086
:109AF000977701009387C7B0984383C747003AC858
:109B0000230AF10097D0FFFFE780C0F17000854580
:109B1000054597A0FFFFE780601D30099305700F92
:109B2000094597A0FFFFE780601C300893050008F7
:109B30000D4597A0FFFFE780601B10089545114574
:109B400097A0FFFFE780801AC16717C7FF1F1307A1
:109B5000270FF9171CC32322070017A5FF1F1305A2
:109B6000A5DD97A0FFFFE78040178327C41D17C519
:109B7000FF1F1305650B82973C4803450900854587
:109B800082978320C11A0324811A8324411A03294E
:109B9000011A8329C1195D618280C16717C8FF1F3F
:109BA0000358080AF9176301F8083DCDB5CD011136
:109BB00026CAB7E4040083A7841222CC2E8623157C
:109BC000B10006CE2A8401478146ED454285829741
:109BD0002AC611ED17850100130505EB975001000A
:109BE000E780E01AF2406244D24405618280FC447E
:109BF0000356A100A28582972C0017C5FF1F0355AD
:109C0000250497A0FFFFE780001A69DD1785010092
:109C10001305C5E897500100E780601783A7C412B9
:109C2000ED45280082977DBF8280011106CE22CCAF
:109C30002DC9854717A7FF1FA309F7D097A7FF1FB7
:109C4000238607D037E40400832784179305F100A7
:109C50001305503082978347F100A9CBA307010079
:109C6000832744171306F10085451305503082976A
:109C70008327441717A6FF1F130686CCB545130587
:109C8000603082978547A307F100832744171306A6
:109C9000F1008545130550308297F240624405611A
:109CA000828097A7FF1FA38207CA49BF8327441753
:109CB00017A6FF1F1306C6C8B54513056030E9BFD8
:109CC000C16717C5FF1F0355A5F7F9176307F5000F
:109CD000B7E7040003A3C7170283828001118547F9
:109CE000A307010017C7FF1F230AF7F4B7E7040013
:109CF00083A7471706CE1306F1008545130550309C
:109D00008297F240056182801793FFFFE702C38CC0
:109D10002A8408452E89B28919C900C19715000007
:109D20009385A586610597300100E7808001814415
:109D30007D5A97100000E780E03963C7A40481448E
:109D400097100000E780003A63C8A40497C7FF1F7C
:109D5000938787EF9C43DC47B307F9409187230241
:109D6000F400638309048327C900B307F44095878F
:109D7000A302F4001C4C89C79C4799C32285829793
:109D80001793FFFF670083885C44139714008504D2
:109D9000BA972390470171BF1C481397140085049C
:109DA000BA972390070069BF832789000547B30747
:109DB000F4409587A302F40083570400638EE70202
:109DC0008DC309476384E7040D47E395E7FA978756
:109DD00001009387672E1CCC978701009387C72EBD
:109DE00011A8978701009387A7F41CCC97870100DF
:109DF000938707F55CC8BDBF97870100938747E04D
:109E00001CCC978701009387A7E0EDB797870100E7
:109E10009387472F1CCC978701009387A72FD9BF23
:109E200095E51783FFFFE702C37C0046184483478C
:109E3000940075839D8B6317F70097100000E780EF
:109E400060B448C41783FFFF6700E37C82801783F8
:109E5000FFFFE702637813893500C16442094111AD
:109E6000AA890144F11413590901054A2EC6971015
:109E70000000E7802026B2456348A4000145410167
:109E80001783FFFF6700837883A709001317140067
:109E9000BA9783D707006388B70063949700637409
:109EA0002A010504E1B70545D9BF1783FFFFE70283
:109EB000C371AA892E89328BB6843A8ABE8A97A04A
:109EC0000000E78020FB71C9268597200000E7800D
:109ED00020098D4763E7A7007D551783FFFF6700C3
:109EE000437283DB440097100000E780A0242A849B
:109EF00097100000E7804025930774003144330534
:109F0000850263CDA70297100000E780A02297107A
:109F10000000E78020222A8497100000E780C022FA
:109F20009307740031443305850263C3A704971077
:109F30000000E78020209307450029A89710000023
:109F4000E7808020330585021307F0179307C017B9
:109F5000E35FA7FA2D55E3C277F963040B02D686B7
:109F60005286A6854A8597200100E78020BAB5B7BA
:109F700097100000E780401D330585029307C5FF59
:109F8000D1BF832749001385C90083D527009700D7
:109F90000000E78000EC61F581B769553DBF97C7C8
:109FA000FF1F2395A7CA97C7FF1F9387E7C9904351
:109FB00081470C463307F500420741836393B7009E
:109FC00082805446139847008507C2962390E60086
:109FD000D5B797C7FF1F938727C79C4303C5870043
:109FE000828017C5FF1F035565C682801783FFFF58
:109FF000E7022360C1671387D7FF630BE502636A3B
:10A00000A700F1176300F50201451783FFFF670002
:10A0100083601387E7FF6302E502FD171D8D13358B
:10A020001500E5B797500000E780C0267D15C5BF35
:10A0300097500000E78040FBD5BF97500000E780B5
:10A0400060F9EDB71783FFFFE702A35A4111AA8415
:10A0500001442EC697100000E780C008B24563484F
:10A06000A400014541011783FFFF6700C35A9C48C4
:10A07000131514003E9583570500E385B7FE0504CC
:10A08000C9BF03485500814693F7F60F63E5070102
:10A0900081473E858280584593975600BA9703D7EB
:10A0A00027006316B70003D70700E304C7FE850641
:10A0B000E1BF8346450001479377F70F63E4D7007C
:10A0C000814711A81C45131657000507B29703D600
:10A0D0000700E313B6FE3E8582801783FFFFE70289
:10A0E000A34F93170501C18797CAFF1F938ACAB56B
:10A0F000635BF00883A70A00C0479C47035704002E
:10A10000198D420541816368F5000144228517835A
:10A11000FFFF6700A34F12052A94CDBFDC471394BD
:10A120004900014A3E94834744006341FA02014AD0
:10A13000834754006349FA028509C20993D909018A
:10A1400083A70A009847E3EBE9FCC1B71C44131945
:10A150005A00A6853E994A8597000000E780C0EE28
:10A1600005E1050AC9B75C4413195A00A6853E9952
:10A170004A8597000000E78020ED19E1050A4DBFF0
:10A18000E30C09FA61B7AA8481495DBF1783FFFF19
:10A19000E70223461C452A8481E79307C5001CC5B6
:10A1A0001C44231204001CC09307F00F63EDB7009A
:10A1B00093F5F50F228597200000E78020E21783B2
:10A1C000FFFF6700434593940501C167C18063F9B0
:10A1D000F500A685228597200000E78040E5C5B7F9
:10A1E000C18193F5F50F228597200000E78000DFFD
:10A1F000A685228597200000E78040E0C9B797C771
:10A20000FF1F938767A4884382801C4599C797C71F
:10A21000FF1F23ABA7A2014582807D55828097C78F
:10A22000FF1F938767A298438347450048479207DB
:10A230003E9582801783FFFFE702A33B61710045D3
:10A240001C183EC6B70780013EC81C183ECA83577B
:10A25000440002CE02D002CC231EF10083478400CA
:10A260002A8902D22301F1023C083ED402D697008B
:10A270000000E78000FB835705002316F10297508A
:10A280000000E78060C42307A1025C40035564001E
:10A29000F18313F717008347F10252055181F99BAF
:10A2A000D98FA307F10297100100E780807539CD9F
:10A2B000AA840355050097A00000E78080BC83D7DF
:10A2C00004002AD26800231CF10083D72400231D38
:10A2D000F1001C4803D647008C4397200000E7801C
:10A2E00000CD8347B400CA86178601001306C68ACC
:10A2F0008117A305F4006C00481097200100E78047
:10A30000E0805D611783FFFF6700E3302155D5BF13
:10A310001C45B1CF03C5A700894613576500630BE1
:10A32000D7028D46630ED70285466300D702130716
:10A3300040063305E50203C7B700418B15CB83C741
:10A34000B700BD8B3355F54082801375F5031307B5
:10A35000803EC5B709671375F50313070771D1BFB1
:10A36000372709001375F5031307077CD9B7014593
:10A3700082801783FFFFE702C32703A98500630CD0
:10A3800009048347B900AE8493F7070E85C30345DC
:10A390009900930520030D810505B305B502884496
:10A3A000610597300100E780E0A935A02E85970070
:10A3B0000000E78020F62A8419CD97000000E7808E
:10A3C000605C8325C900B307B54063FA87002E940B
:10A3D000B305A440E9F51783FFFF6700C323854554
:10A3E0007DBF1783FFFFE702C3202A8403D5050042
:10A3F000011132C636C43AC22EC002CA02CC02CE05
:10A4000097A00000E780E0A782452ACA22852ECCCB
:10A4100097000000E780E0E003570500231EE100FD
:10A4200097500000E78040AAA24632469247230F89
:10A43000A10036874C08B2862285014697000000AD
:10A44000E780E0A605611783FFFF6700C31C178341
:10A45000FFFFE702031A61711C183EC6B7078001AF
:10A460003EC81C183ECA3C0800453ED4AA8402CC13
:10A4700002CE02D002D202D697000000E78060DA56
:10A480008357050035592316F10297500000E780E5
:10A49000A0A32307A10209C48357440081EB2159DB
:10A4A0004A855D611783FFFF6700E316035564006B
:10A4B0005205518197100100E780A0542A8965D187
:10A4C0008347B40093F7070E99C7130584019730AB
:10A4D0000100E780609983574400231EF100834701
:10A4E00084002301F1025C4003550900D98313F76E
:10A4F000070883471102231CA10093F7F707D98FA0
:10A50000A300F10283572900231DF1005C40F18371
:10A5100013F717008347F102F99BD98FA307F102C4
:10A5200097A00000E780E0952AD235D983479400B0
:10A530006800139757008347B400FD8BD98FA3059C
:10A54000F4001C4803D647008C4397200000E780A6
:10A5500000A6A68717770100130707647400054655
:10A560004C10268597000000E78060942A890DD959
:10A570008347B400A685FD8BA305F4009700000077
:10A58000E78060DF31BF1783FFFFE7028306832484
:10A5900085FE2A844111268597000000E78080D738
:10A5A000834734FF93F7070E8DCB2AC62685970085
:10A5B0000000E78060C809CD834734FFB245FD8BBA
:10A5C000A309F4FE91C5228597300100E7808087BA
:10A5D00041011783FFFF670003047DD98327C4FF70
:10A5E0002685829775F5834734FF93F7070E91C749
:10A5F000228597300100E7802087032584FE97009D
:10A600000000E78000E5E9B71783FFFFE70263FB7F
:10A610009C4141112A8903C7070089472E8493561C
:10A6200067006380F6040D466388C6049307F0074D
:10A630006304F7022E8597200000E780C0A7AA8454
:10A640008149C16B130C490097B7FF1F9387C75F00
:10A650009C43984763E4E90441011783FFFF6700C7
:10A6600003FA03D745008547E3F8E7FE2E859720D8
:10A670000000E780A0A9E1B703D74500E3FEE7FCAF
:10A680002E8597200000E78000A3AA8422859720CA
:10A690000000E78060A4C204C98C5DB7DC470355A5
:10A6A000A900139A49003E9A93170501C187635D7B
:10A6B000F00083570A006397A70263E774038327B8
:10A6C000CA00034D5A002DA0A1672167A98F130767
:10A6D000F7EFE374F7FE6397090097000000E78047
:10A6E000209161FD85098DB783278A00034D4A00BB
:10A6F000835DA90003576900216A138BC7003AC61E
:10A70000814A33CA4D01631E5D0197B7FF1F9387CE
:10A7100027549C43E1DBA286628681452685829789
:10A72000D1B7A1679387F7EF930C4BFF63F2470311
:10A73000B2455A8597F0FFFFE780A0710DC103274E
:10A740008B00104709CE10436382C4023107D5BF86
:10A75000EE85668597000000E780008F71F993868B
:10A760001A0093FAF60F130B0B0271BF83564400C5
:10A770005C43E3E9F6F622853AC697100000E780CD
:10A78000807DA1679387D7042A8A035D44003247FE
:10A7900063E897008347D90093E707F8A306F90019
:10A7A0001C4766852286E2858297C1670844FD17AB
:10A7B000337AFA00529508C02312A40125B797B73F
:10A7C000FF1F938767489843814715C31447814704
:10A7D00063FFD500939745004C47BE9519C903C741
:10A7E000550081476375E600DC451606B2973E8545
:10A7F000828003C745008147E37BE6FE16069C4541
:10A80000F5B71783FFFFE70223DDAA892E8A81446B
:10A8100097BAFF1F938A4A4383A70A00984763E6C3
:10A82000E4001783FFFF670063DEDC4713944400F6
:10A8300001493E9413BB140083474400634BF90065
:10A84000014913BB140083475400634FF90085048A
:10A85000E1B70844931759005287DA860146A2856A
:10A860003E9582990509C9BF4844931759005287FC
:10A87000DA860546A2853E9582990509E9B71783D0
:10A88000FFFFE70203D7814517F5FFFF13050548D2
:10A8900097B7FF1F239C073A97000000E780A0F6B8
:10A8A0001783FFFF670023D797B7FF1F9387C73929
:10A8B0009C4395C31783FFFFE702A3D3814517F598
:10A8C000FFFF1305A54497000000E780C0F317833E
:10A8D000FFFF670043D482801783FFFFE702C3CFE7
:10A8E00037E404008327841241112315E100AE8967
:10A8F0003289368A3A8681460147ED45AA84829795
:10A900002AC621C90356A100D28597400100E780DD
:10A91000C0248327C413CE8526858297058905C95F
:10A920008327440D2314210101462C00268582979C
:10A930002A8401C9B7E7040083A7C712ED452800A0
:10A940008297228541011783FFFF670023CC49448A
:10A95000D5B76554FDB75C41FD175CC18280178394
:10A96000FFFFE70203C9B7E70400FC5F8297954742
:10A970003305F50281450D811783FFFF6700A3C9E9
:10A980001783FFFFE702E3C6B7E70400FC5F829787
:10A9900095473305F5020D811783FFFF6700A3C7B5
:10A9A0001783FFFFE702E3C4B7E7040083A7870B21
:10A9B0000355050082971783FFFF6700C3C5178300
:10A9C000FFFFE70203C3035505003287AE861796E3
:10A9D000FF1F035606FF97B5FF1F9385A527970016
:10A9E0000000E780A0EF1783FFFF6700C3C2178353
:10A9F000FFFFE70203C0B7E7040083A7C7178297EA
:10AA00001783FFFF670023C11783FFFFE70263BEC1
:10AA1000B7E7040083A7871397B5FF1F93858523A6
:10AA2000829701451783FFFF6700E3BE1783FFFF8F
:10AA3000E70223BCB7E7040083A7C71F814517952A
:10AA4000FF1F035505F482971783FFFF6700A3BC20
:10AA50001783FFFFE702E3B9B7E7040083A7871373
:10AA600097B5FF1F93850520829701451783FFFF48
:10AA7000670063BA1783FFFFE702A3B7B7E70400D5
:10AA800083A7C71F81451795FF1F035585F582973B
:10AA90001783FFFF670023B81783FFFFE70263B543
:10AAA0002E8597800000E780E0AF97800000E78068
:10AAB000E0EC1783FFFF670003B61783FFFFE70291
:10AAC00043B397800000E780E0F61783FFFF67003D
:10AAD00083B45C49E1175CC95CC583572501A107B4
:10AAE0002319F50083570501A1072318F50082807B
:10AAF000F1473305F50297B7FF1F9387A7189C43CB
:10AB00003E9582808D476315F60803D7460085473A
:10AB100063F0E7081783FFFFE702A3AD36853684AD
:10AB20002E8997100000E780005929C983574400F7
:10AB300093140501C18063E39704228597100000F8
:10AB4000E7806057FD14231294009307A00263006E
:10AB5000F5029307B0026307F50293079002631FA3
:10AB6000F500228597000100E780C08501A8014615
:10AB7000CA85228597A00000E78060B01783FFFF99
:10AB8000670063A9228597100000E780C003FDB726
:10AB9000828097B6FF1F9386260F9C42014599CF6E
:10ABA0009843D44217B6FF1F2320E60E6396D700C2
:10ABB00097B6FF1F23ACE60C1385C7FE8280178370
:10ABC000FFFFE70203A397000000E780A04B71445A
:10ABD00033058502914597900000E78020E911E553
:10ABE00065551783FFFF670003A397B7FF1F23A9CE
:10ABF000A70897000000E780E048330585029145EB
:10AC000097900000E78080E661DD97B7FF1F23ABD8
:10AC1000A70697000000E780E04697B7FF1F239B39
:10AC2000A70497000000E780E04597B7FF1F239433
:10AC3000A70497770100938767FB17B7FF1F232FA0
:10AC4000F70297070000938707E917B7FF1F23252F
:10AC5000F702014579B71783FFFFE7028399AA85B9
:10AC600017B5FF1F1305050197100000E780C05BB3
:10AC70001783FFFF6700239A1783FFFFE70263979D
:10AC800097000000E78060FD97100000E780405BC0
:10AC900097B7FF1F938747FF9C4391CF1387C7FE4A
:10ACA00019CB83D5C7FF17B5FF1F130565FE972086
:10ACB0000100E78020191783FFFF6700C395178302
:10ACC000FFFFE702039397000000E780C0EC09CD87
:10ACD000834785002A8493F7070499EB0355E50021
:10ACE00097000000E78080F91783FFFF6700A392B9
:10ACF0008347C5009304450117B9FF1F1309C9F81D
:10AD000085E3832709005CC997B7FF1F23AE97F639
:10AD100083274900F1FB97B7FF1F23A997F6E9B7EF
:10AD2000FD172306F500610597800000E780C0D677
:10AD30008307840063CB07048347840093E707F805
:10AD40002304F400B7E704009C5F82974205A947FB
:10AD500041813375F5028347840093F707FCC98F5F
:10AD60002304F4008347D4003E951C402318A4001C
:10AD700089CF984319CB8347C4005040814585074C
:10AD80003305F502420541810297832709005CC81B
:10AD900097B7FF1F23AA97EE8327490089E797B744
:10ADA000FF1F23A597EE8347C4009DDF8355040151
:10ADB00017B5FF1F1305C5ED97200100E780800838
:10ADC00025B71783FFFFE702C38297B7FF1F93875B
:10ADD00067119C4701448583858B85E3AE84B285EA
:10ADE0003A8697100000E780804B2A8419C5971097
:10ADF0000000E780C041829408CC22851783FFFFC2
:10AE0000670063811773FFFFE702037D41112E89FD
:10AE100032C6AA8997000000E780C0313247130686
:10AE20000502CA86970500009385C5CC17B5FF1F9C
:10AE3000130545E497000000E780E0F82A8425C95F
:10AE40009304C50097000000E780E0411946AA85F9
:10AE5000268597100000E780801585452685971088
:10AE60000000E7806011177501001305E5D54E95C8
:10AE700083450500268597100000E78020165C4872
:10AE800031468145A1075CC85CC483572401E117A2
:10AE90002319F40083570401E1172318F4001C4C14
:10AEA0003E859770FFFFE780C077A30425012285C8
:10AEB00041011773FFFF670063751773FFFFE70218
:10AEC00043734111AA842EC632C497100000E78054
:10AED0006036004DB2452246834784000CC050C006
:10AEE00093F7F70393E707042304F40023180400FF
:10AEF000268597100000E780803183479400A9469B
:10AF00002317A40013D7370005073307D7029D8BFB
:10AF100085072306F400A306E40083C70401D8488C
:10AF20008507230FF7FE17B7FF1F1307E7D5584311
:10AF3000232A04009307440129E317B7FF1F23279F
:10AF4000F7D417B7FF1F2321F7D417B4FF1F13043B
:10AF500024D4228597200100E78000E11C44858BE2
:10AF60005D8D19E58145228597200100E78080ED00
:10AF700041011773FFFF6700036A1CC317B7FF1F68
:10AF80002326F7D0D9B71773FFFFE702836697052B
:10AF90000000938565B7014597000000E78000B089
:10AFA00001451773FFFF670003671773FFFFE70291
:10AFB000436497000000E78080B01773FFFF6700CD
:10AFC00083658347C500A5E31773FFFFE70263624C
:10AFD0002A840355E50097000000E78000C821C1DE
:10AFE0008347840093F7F7FB2304F4001C4091C7C8
:10AFF000DC4381C74C400145829797000000E78001
:10B0000080B917B5FF1F1305A5C897200100E78079
:10B01000A0E50355E40097000000E78020C6177301
:10B02000FFFF6700435F82801773FFFFE702635CE7
:10B0300097B7FF1F938747C597050000938565C89D
:10B0400017B5FF1F1305C5C423A0070023A20700DF
:10B0500097200100E780E0CE1773FFFF6700A35B36
:10B060001C4D91CFDC4381CF1773FFFFE70263587C
:10B070008345070082971773FFFF6700C3598280DB
:10B0800097B7FF1F938707C39C4303C507008280C0
:10B0900097B7FF1F938707C29C4303C517008280A1
:10B0A00097B7FF1F938707C19C4303C52700828082
:10B0B00097B7FF1F938707C09C4303C54700828053
:10B0C00097B7FF1F938707BF9C4303C53700828054
:10B0D00097B7FF1F938707BE9C4303C55700828025
:10B0E00097B7FF1F938707BD9C4303C56700828006
:10B0F00097B7FF1F938707BC9C4303C577008280E7
:10B1000097B7FF1F938707BB9C4303C587008280C7
:10B1100097B7FF1F938707BA9C4303C597008280A8
:10B1200097B7FF1F938707B99C4303C5A700828089
:10B1300097B7FF1F938707B89C4303C5B70011E17A
:10B140001D45828097B7FF1F9387C7B69C4303C5F1
:10B15000C700828097B7FF1F9387C7B59C4303C57D
:10B16000D700828097B7FF1F9387C7B49C4303C55E
:10B17000E700828097B7FF1F9387C7B39C4303D52F
:10B180000701828097B7FF1F9387C7B29C4303C50F
:10B190002701828097B7FF1F9387C7B19C4303D5D0
:10B1A0004701828097B7FF1F9387C7B09C4303D5A1
:10B1B0006701828097B7FF1F9387C7AF9C4303D572
:10B1C0008701828097B7FF1F9387C7AE9C4303C553
:10B1D000A701828097B7FF1F9387C7AD9C4303C524
:10B1E000B701828097B7FF1F9387C7AC9C4303C505
:10B1F000C701828097B7FF1F9387C7AB9C4303C5E6
:10B20000D701828097B7FF1F9387C7AA9C438857AF
:10B21000828097B7FF1F9387E7A99C4303D5C70296
:10B22000828097B7FF1F9387E7A89C4303D5E70267
:10B2300019E11305800C828097B7FF1F938787A7BA
:10B240009C4303C50703828097B7FF1F938787A698
:10B250009C43C85B828097B7FF1F938727A58843CD
:10B26000828097B7FF1F9387A7A48843828019E144
:10B270007D558280F5DE984265DFFDD917B7FF1F47
:10B28000130747C61847AA877155058B631D072406
:10B2900003C507001547E37DA7FC03C73700130567
:10B2A000F0057D171377F70FE364E5FC03C3570040
:10B2B000E30003FC83C86700E38C08FA03C7770048
:10B2C000494579171377F70FE364E5FA03C7A70039
:10B2D00011481305F7FF1375F50FE36BA8F803CEBC
:10B2E00097000D481305FEFF1375F50FE362A8F8EC
:10B2F00003C8B7006309080065181378F80F130531
:10B30000600DE36705F703C5C70079487915137524
:10B31000F50FE36FA8F403C8D7000D457D18137827
:10B32000F80FE36705F503D80701930E401751188E
:10B33000420813580801E3ED0EF303C8E7007D1837
:10B340001378F80FE36605F303C827017D18137817
:10B35000F80FE36F05F103C88700C54E7518137821
:10B36000F80FE3E70EF103D86701856E938EBEE018
:10B370006D18420813580801E3EC0EEF03D847019B
:10B380006D18420813580801E3E40EEF03D8870153
:10B390007918420813580801E36C05ED03C8A701AA
:10B3A0007D181378F80FE36505ED03C5B7011D4857
:10B3B0007D151375F50FE36DA8EA03C5D701714834
:10B3C00079151375F50FE365A8EA03D5E7011308AE
:10B3D000E00F7D1542054181E36CA8E803C5070233
:10B3E000494879151375F50FE364A8E8C85301C9F6
:10B3F00037C834005915130858BFE36BA8E603A8F3
:10B40000870237C53400130555BF5918E36205E7B5
:10B4100017B5FF1F232EC58803C6050117B5FF1FEB
:10B42000232AF5880545E375C5E403D82501D049ED
:10B4300033760603E31E06E203C61501E30A06E2BD
:10B4400017B6FF1F2324B68683C5270001466387EE
:10B45000A50003C61700F1453306B60283C70703EC
:10B460009305C00272971A071307C70516031A97A8
:10B4700096084697B387B70241553E9732974207E1
:10B4800041836362E8061773FFFFE7028316368580
:10B4900097800000E780A06897000100E7802048BF
:10B4A0002A8497A00000E780805A2A9497F0000031
:10B4B000E78060262A9497900000E780A0812A9474
:10B4C00097F0FFFFE780E06F2A9497400000E78045
:10B4D00060932A9497700000E780A09C22951773D0
:10B4E000FFFF6700431382801773FFFFE7026310BB
:10B4F0004111A307A10097A00000E780A0C5930514
:10B50000F100170500001305E5B597F0FFFFE78090
:10B51000802F014541011773FFFF6700C30F1773A9
:10B52000FFFFE702830A17B4FF1F1304A49B03283D
:10B53000840079599368180097B4FF1F23A8149BBF
:10B540001378180063100802BA84BE89368B328AD9
:10B550002E89AA8A97F0FFFFE780E0A77D15269540
:10B5600019E531594A851773FFFF6700830997F082
:10B57000FFFFE78040A67D152695A167E353F5FE02
:10B5800097B7FF1F938707CD98433E8C814B01CB24
:10B59000014597F00000E7802044933B15004A8561
:10B5A000DA865686D28597900000E780C04D2A89BA
:10B5B00011CD1C44F99B17B7FF1F2329F79283274E
:10B5C0000C00CDD3E3800BFA829769BF268597B72D
:10B5D000FF1F23AB079097F0FFFFE780809C414659
:10B5E000CE8517B5FF1F1305659997300100E780D9
:10B5F000C05697D00000E78040990325040B97D0F0
:10B600000000E780009D054597D00000E78000A47A
:10B61000054597000000E78060EDA9B797B7FF1FC9
:10B620009387478C9C47858BEDC71773FFFFE70215
:10B6300043FC17B5FF1F1305A59297B7FF1F23A360
:10B64000078A97B7FF1F23A1078A97B7FF1F23AF6A
:10B65000078897200100E780208197500000E7804D
:10B66000E0F597100100E780A04C97100100E780FB
:10B67000A05297B7FF1F938767859C4391C70545E5
:10B6800097800000E780402097A7FF1F9387C76D32
:10B690009C4399C741657D1597700000E78040A2E3
:10B6A00097F00000E780E03D97D00000E780808FB2
:10B6B00097B7FF1F938707989C431397170163560B
:10B6C000070097F00000E78000AD97B7FF1F23A7A2
:10B6D000078A97B7FF1F23A5078A97B7FF1F23A3E2
:10B6E000078A97B7FF1F23A1078A97000000E7800A
:10B6F000008C97000000E780007297F0FFFFE78062
:10B70000401897F00000E78040D61773FFFF6700EE
:10B7100083F0828097A7FF1F9387C77C884382802E
:10B720001773FFFFE702E3EC97800000E780607586
:10B7300097800000E780C0771773FFFF6700A3EDD5
:10B740001773FFFFE70243E92A84930414020111EF
:10B750002E85B289A685214636C63A8997300100E2
:10B76000E780403D0DE9B24638082686CE851305B0
:10B77000940497500000E780604121462C084A85D8
:10B7800097300100E780003B133515000561177302
:10B79000FFFF6700A3E70145D5BF1773FFFFE7026F
:10B7A00043E59305450617A5FF1F1305E5509710C0
:10B7B0000100E78020691773FFFF6700C3E5177377
:10B7C000FFFFE70203E341112EC697F0FFFFE7807A
:10B7D000601BB24588C141011773FFFF6700A3E3F7
:10B7E0001773FFFFE70243DFAA842E8497800000CF
:10B7F000E780006CAA898545228597000000E780D4
:10B80000E07D83C7E4011389940899E31389040355
:10B81000CE85228597000000E780407C2146930575
:10B820001902228597000000E780607897A7FF1F24
:10B830009387476B8C43228597100000E780C08276
:10B84000214693858402228597000000E7802076B8
:10B850001773FFFF670083DB1773FFFFE702E3D671
:10B86000397197F00000E780E0B49305400661E984
:10B8700097800000E78000606302051497A7FF1F10
:10B8800083C7474513B7170097A6FF1F2384E644D5
:10B89000014499CFC16417A9FF1F1309A964930933
:10B8A000400EFD1497000000E780C0866342A40AA2
:10B8B00097F0FFFFE780000D4169B7290900096A89
:10B8C000FD7A2A8B81447D199389F97B130A0A71C9
:10B8D000938A8AC797000000E780C08363D7A404D7
:10B8E0001304400EB387840217A7FF1F1307875F57
:10B8F0000324070B3E948357C4016382270B18402F
:10B900003307EB4063EAE900834744008507B387C8
:10B910004703D6976365F70801468145094597F0C7
:10B92000FFFFE780604EAA8B29E597400000E78083
:10B93000808385476317F50689659385057117A58B
:10B94000FF1F1305653797100100E780A04F95A0F2
:10B95000B30734030327090BBA9703D7C70163085A
:10B96000970003C75700A38207002382E70005045E
:10B9700015BF9305C500228597000000E78080E68B
:10B980005E852286976501009385452597F0FFFF28
:10B99000E780E0525E8597100000E780608A8504AA
:10B9A00015BF97A7FF1F9387E7539C478D83858B10
:10B9B000C1F721611773FFFF6700A3C401468545E6
:10B9C000094502D002D202D402D697F0FFFFE780E9
:10B9D000A043AA8479DD97F00000E780E09C1389FA
:10B9E000C4002A8481454A8597000000E780005FF3
:10B9F0000C4041464A8597000000E780405B832960
:10BA000044006385090C4E8502D802DA02DC02DEAE
:10BA100097300100E78060402ACE141005462C08BC
:10BA200008184ECC97500000E780E00A1375F50F18
:10BA300051ED8355840093E525004A859700000069
:10BA4000E780E05E11460C104A8597000000E78011
:10BA500000560146976501009385C518268597F025
:10BA6000FFFFE780C045268597000000E780407D06
:10BA70005C40A1D3014685450D4597F0FFFFE78067
:10BA8000A038AA841DD548401389C400973001000E
:10BA9000E780A0382AC64A8597000000E780404C1E
:10BAA0003246636FC5004C404A8597000000E7802E
:10BAB000005001468145268597F0FFFFE780204032
:10BAC000268597000000E780A077E5B583558400C0
:10BAD000ADB71773FFFFE702C3B197A7FF1F9387A7
:10BAE00067409C471DC193E7870017A5FF1F1305FB
:10BAF000A51C17A7FF1F232BF73E97100100E78017
:10BB000040321773FFFF670003B1DD9B17A7FF1FCC
:10BB1000232EF73C97300000E780E0647DF117A505
:10BB2000FF1F1305651997100100E780E033D1BFAF
:10BB30001773FFFFE70263A94169AA892E8AB28AB7
:10BB4000368BBA8B814417ACFF1F130CAC39930CA6
:10BB5000400E7D1997F0FFFFE780C05B63C4A4002F
:10BB600001443DA03384940383270C0B3E948357F8
:10BB7000C401638627055A87D6865286CE8513056B
:10BB8000040397000000E780E0BB01C923800B009D
:10BB900022851773FFFF6700C3A68347F40185C39F
:10BBA0005A87D6865286CE851305940897000000E2
:10BBB000E78040B909C585472380FB00D1BF8504D4
:10BBC00051BF835745006380071E1773FFFFE702CD
:10BBD000A3A001112A8497000000E780C04D09C985
:10BBE00085476309F50605611773FFFF670003A228
:10BBF00097E00000E780007C7DF5835744004947CB
:10BC0000ED9BE392E7FEC145228597000000E780A7
:10BC10004033AA84228597000000E780204F035715
:10BC2000440002CE91472A89631AF70022859700C3
:10BC30000000E780A0513C082ACC3ECE97E00000EF
:10BC4000E78080765C55C5D374084A86A68505458D
:10BC5000829751BF03574400D147E3F6E7F8032A20
:10BC60000400C169014997AAFF1F938AAA27130BF1
:10BC7000400EFD1997F0FFFFE780C049634FA90E02
:10BC80002285032A040097000000E780C042A145F6
:10BC90002A89228597000000E780A02AAA842285AD
:10BCA00097000000E780804A14402A86AA89780815
:10BCB0002685CA8597000000E780C0E7AA8405D5DD
:10BCC00003C7F40189476315F7008347C10181DF8A
:10BCD0005546D2851385640097300100E780E0E780
:10BCE000014597800000E780C01901C583D7C401D2
:10BCF000A5E797A7FF1F9387E71E9C479355190059
:10BD0000858913D73700058B01CF8983858B63998C
:10BD1000B70001452EC697000000E780C0DBB245A2
:10BD20004E8597800000E780601F0346C1012A848A
:10BD300093751900268597900000E780E03935C19A
:10BD4000268597800000E780E018268511C0014510
:10BD500097800000E780004C97300000E780A0400B
:10BD60008547E312F5E883C754001307F00FE38C0F
:10BD7000E7E68507A382F400BDB5B304690383A792
:10BD80000A0BBE9483D7C401638B37015546D28515
:10BD90001385640097300100E780C0D955DD05099F
:10BDA000D1BD5DD86DB782801773FFFFE702C382F4
:10BDB00097800000E780000C05C1C164014417A909
:10BDC000FF1F130929129309400EFD1497F0FFFF7E
:10BDD000E7804034634EA40017A5FF1F1305C5ED8F
:10BDE00097100100E780E0031773FFFF67000382ED
:10BDF000330534038327090B3E958357C5016388B8
:10BE000097002312050097800000E780A00C05042E
:10BE100075BF97A7FF1F9387E70C9C478D83858B82
:10BE20008DE31763FFFFE702C37C17A5FF1F130510
:10BE3000A5E897100100E78020031763FFFF670064
:10BE4000837D82801763FFFFE702A37A97050000D6
:10BE50009385C5A017A5FF1F130505E697100100E0
:10BE6000E78020EE1763FFFF6700E37A1763FFFFA9
:10BE7000E70223788841B7E70400BC5B050542056B
:10BE80004181829709C585472300F50005051763A1
:10BE9000FFFF6700437883C7F5FF2E858507A38FD3
:10BEA000F5FE828083C7F5FFFD1793F7F70FA38F89
:10BEB000F5FE99EF1763FFFFE702A373B7E70400EE
:10BEC000BC571385F5FF82971763FFFF6700A374C4
:10BED00082801C41035745008D8FBA951CC12312E7
:10BEE000B5003E85828093D78500A2051441DD8D83
:10BEF000835745001387E6FF18C189072312F50011
:10BF000013D685004111238FB6FEA38FC6FE4101D3
:10BF1000828018419307F7FF1CC1835745008507AE
:10BF20002312F500A30FB7FE8280835745008D8F43
:10BF30002312F5001C41BE950CC12E858280AA8774
:10BF400003D7470008410D8FAA952392E7008CC3C1
:10BF50008280184108453305A740828083574500F9
:10BF6000035765001D8F1C4108453385A7403305E5
:10BF7000A74082801763FFFFE702A36741112EC627
:10BF80002A8497000000E780A0FDB2456373B500E6
:10BF900001A0835744000840BE952312B4003E958B
:10BFA00041011763FFFF670003671763FFFFE702A5
:10BFB000436441112E84B28532C697000000E780A9
:10BFC000A0FB3246A28597300100E78000B941010D
:10BFD0001763FFFF670023641763FFFFE7026361D6
:10BFE0002E84854597000000E78000F92300850036
:10BFF0001763FFFF670023621763FFFFE702635FBA
:10C0000041112317B100894597000000E780C0F671
:10C010008347E1002300F5008347F100A300F5000A
:10C0200041011763FFFF6700035F1763FFFFE7022C
:10C03000435C93D78500A2054111DD8D2317B10024
:10C04000894597000000E78020F38347E100230043
:10C05000F5008347F100A300F50041011763FFFFDE
:10C060006700635B1763FFFFE702A358139785011F
:10C0700093D78501C166938606F0D98F13D78500C3
:10C08000758FD98FA2053707FF00F98D4111DD8D1E
:10C090002EC6914597000000E78000EE6C00114627
:10C0A00097300100E78060AB41011763FFFF670035
:10C0B00083561763FFFFE702C3531C41854503C442
:10C0C000070097000000E78080E622851763FFFFE6
:10C0D000670063541763FFFFE702A3511C4141113E
:10C0E000894503C7070083C717002307E100A3079B
:10C0F000F10097000000E78080E30355E100410173
:10C100001763FFFF670023511763FFFFE702634ECA
:10C110001C414111894503C7070083C71700230746
:10C12000E100A307F10097000000E78040E083579B
:10C13000E100410113D58700A2075D8D42054181D1
:10C140001763FFFF6700234D1763FFFFE702634A92
:10C150000C4141112A841146680097300100E780A4
:10C16000C09F9145228597000000E78040DCB247E0
:10C17000C166938606F01397870113D58701598D01
:10C1800013D78700758F598DA2073707FF00F98FE6
:10C190005D8D41011763FFFF6700E3471C45BE95B6
:10C1A0000CC18280AE87944391E6584101EF0CC1E7
:10C1B0005CC1828003C7570013671700A382E700A2
:10C1C000B687D5B70CC3EDB7AA87084119CD18417A
:10C1D000D44398C36313D500D8C32A8703465700B6
:10C1E0009376160081E6232007008280944381CA5B
:10C1F0008C4203A847008CC363930601CCC3799A91
:10C2000014C3A302C7003687D1BF1C45DC471D8D70
:10C21000B777DBB6938777DB09853305F5024205EF
:10C2200041818280F147B385F50248452E95828091
:10C230008347450085072302F50082801763FFFFCF
:10C24000E702233B2A8409E41763FFFF6700A33C4E
:10C2500083474400F5DBFD1793F7F70F2302F40043
:10C26000E5F71C4403D7270005072391E700DC43CB
:10C2700099C3228582974C4889CD83475400898B86
:10C2800099E71C4422859C479C439C478297232A1C
:10C2900004000040232004007DB71763FFFFE7027E
:10C2A00043358357250041112EC681EB0144228579
:10C2B00041011763FFFF67000336035705008147FD
:10C2C000F146E305F7FEB385D702404585072E9476
:10C2D0008345440008C4F5F5B247AA8481E7232AC0
:10C2E000040009A81C456C0022859C439C4382974E
:10C2F00048C84DDD85472312F400B24723200400CF
:10C30000231804002319F4005C485CC483D724007C
:10C31000FD172391F40061BF1763FFFFE702632D50
:10C3200097A7FF1F9387479B884323260500232455
:10C330000500410597100100E78000B31763FFFF78
:10C340006700632D1763FFFFE702A32A17A4FF1FEF
:10C35000130484981C40411199CF9C472300B500D9
:10C360002AC65CC197000000E78040FB1C40DC430C
:10C3700099C33245829741011763FFFF6700A329E4
:10C380000347450029E3584DAA877D551DCF176304
:10C39000FFFFE70203261CC3DC4797A6FF1F23AD60
:10C3A000E692F156130507012390D7009705000088
:10C3B0009385050297100100E780A0980145176357
:10C3C000FFFF670043257D55828082801763FFFF52
:10C3D000E702232201116146814528009760FFFF93
:10C3E000E780202497A7FF1F9387078F9C4328008F
:10C3F0009305F00FDC473EC697000000E780C0F4CD
:10C4000005611763FFFF6700032197A7FF1F93874D
:10C41000A78C9C43D847A1679387C702631EF70A7E
:10C42000397106DE22DC26DA80004AD84ED652D494
:10C4300056D23285B28497000000E780C0C7AA892F
:10C44000268597000000E78020C92318A4FC2685D4
:10C4500097000000E78040C82319A4FC26859700B8
:10C460000000E78060C783D744000A8A231AA4FC2F
:10C47000858393F7F70F230EF4FC8607BD0793F728
:10C48000073F3301F1408A8A01498347C4FD63674E
:10C49000F902CE85130584FC232C54FD970000007F
:10C4A000E78080EA5281130104FCF2506254D254B6
:10C4B0004259B259225A925A2161828026859700A8
:10C4C0000000E78060C193171900D69705092390F3
:10C4D000A7001379F90F55BF82809797FF1F9387A5
:10C4E000A77F9C43D847A1679387A702631AF70ADF
:10C4F000397106DE22DC26DA80004AD84ED652D4C4
:10C5000056D23285B28497000000E780C0BAAA896B
:10C51000268597000000E78020BCFD572318A4FC67
:10C5200026852319F4FC97000000E780E0BA83D742
:10C5300044000A8A231AA4FC858393F7F70F230E7D
:10C54000F4FC8607BD0793F7073F3301F1408A8A61
:10C5500001498347C4FD6367F902CE85130584FC56
:10C56000232C54FD97000000E78000DE5281130168
:10C5700004FCF2506254D2544259B259225A925A8F
:10C5800021618280268597000000E780E0B4931740
:10C590001900D69705092390A7001379F90F55BF05
:10C5A00082809797FF1F938727739C43D847A16783
:10C5B00089076310F70A397106DE22DC26DA80006B
:10C5C0004AD84ED652D456D23285328997000000CE
:10C5D000E78060AEAA894A8597000000E780C0AF77
:10C5E000835749000A8A2318A4FC858393F7F70F21
:10C5F000230CF4FC8607BD0793F7073F3301F14096
:10C600008A8A8144834784FD63E7F402CE8513055B
:10C6100084FC232A54FD97000000E780E0D2528179
:10C62000130104FCF2506254D2544259B259225AB6
:10C63000925A216182804A8597000000E780C0A954
:10C6400093971400D69785042390A70093F4F40FD2
:10C6500055BF82809797FF1F938707689C43D847F1
:10C66000A1679387E704631EF70A397106DE22DCAF
:10C6700026DA80004AD84ED652D456D23285B284B9
:10C6800097000000E78020A3AA8926859700000074
:10C69000E78080A42318A4FC268597000000E7808B
:10C6A000A0A3231AA4FC268597000000E780C0A25F
:10C6B00083D744000A8A2319A4FC858393F7F70FD4
:10C6C000230EF4FC8607BD0793F7073F3301F140C3
:10C6D0008A8A01498347C4FD6367F902CE85130541
:10C6E00084FC232C54FD97000000E780E0C55281B4
:10C6F000130104FCF2506254D2544259B259225AE6
:10C70000925A21618280268597000000E780C09CB4
:10C7100093171900D69705092390A7001379F90FED
:10C7200055BF82809797FF1F9387075B9C43D8472D
:10C73000A1679387C704631AF70A397106DE22DC02
:10C7400026DA80004AD84ED652D456D23285B284E8
:10C7500097000000E7802096AA89268597000000B0
:10C76000E7808097FD572318A4FC2685231AF4FC44
:10C7700097000000E780409683D744000A8A231977
:10C78000A4FC858393F7F70F230EF4FC8607BD07FF
:10C7900093F7073F3301F1408A8A01498347C4FD7B
:10C7A0006367F902CE85130584FC232C54FD9700A2
:10C7B0000000E78060B95281130104FCF25062541A
:10C7C000D2544259B259225A925A21618280268506
:10C7D00097000000E780409093171900D69705094D
:10C7E0002390A7001379F90F55BF82809797FF1FF9
:10C7F0009387874E9C43D847A167DD076317F704EB
:10C800001763FFFFE702E3DE797132853284970018
:10C810000000E780408A2AC6228597000000E78052
:10C82000A08B2311A102228597000000E780A08839
:10C83000B2452300A102280897000000E780C0B09D
:10C8400045611763FFFF670003DD82809797FF1F35
:10C85000938787489C43D847A167938787046317CA
:10C86000F7041763FFFFE702C3D87971328532847A
:10C8700097000000E78020842AC6228597000000E8
:10C88000E78080852311A102228597000000E780C0
:10C890008082B2452300A102280897000000E780AB
:10C8A000A0AA45611763FFFF6700E3D682809797D0
:10C8B000FF1F938767429C43D847A1679387A704CC
:10C8C0006312F7021763FFFFE702A3D201112800EA
:10C8D000814597000000E78020A705611763FFFFEF
:10C8E000670063D382809797FF1F9387E73E9C433F
:10C8F000D847A167938757026319F7021763FFFFB1
:10C90000E70223CF0111328597F0FFFFE780A07A7D
:10C910002308A1008145280097000000E780C0A2FD
:10C9200005611763FFFF670003CF82809797FF1FA2
:10C930009387873A9C43D847A1679387E702631B95
:10C94000F7041763FFFFE702C3CA0111328532847F
:10C9500097F0FFFFE7804078AA84228597F0FFFFD9
:10C96000E7808077854709E9228597F0FFFFE78018
:10C9700080744205B337A000280081452318910038
:10C980003ECA97000000E780209C05611763FFFF07
:10C99000670063C882809797FF1F9387E7339C43A4
:10C9A000D84799476313F7081763FFFFE70263C48B
:10C9B00079713285328497F0FFFFE780C06F2AC615
:10C9C000228597F0FFFFE78020712310A1022285C6
:10C9D00097F0FFFFE780206E2301A102228597F0E8
:10C9E000FFFFE780406DA301A102228597F0FFFFC2
:10C9F000E780606C2302A102228597F0FFFFE780A9
:10CA0000806B2313A102228597F0FFFFE780A06AC5
:10CA1000B2452314A102280897000000E780C092C5
:10CA200045611763FFFF670003BF82809797FF1F71
:10CA30009387872A9C43D847A1679387C7036313CB
:10CA4000F7081763FFFFE702C3BA797132853284B2
:10CA500097F0FFFFE78020662AC6228597F0FFFF48
:10CA6000E78080672310A102228597F0FFFFE7800F
:10CA7000A0662311A102228597F0FFFFE780A06343
:10CA80002302A102228597F0FFFFE780C062A30284
:10CA9000A102228597F0FFFFE780E0612303A10256
:10CAA000228597F0FFFFE7800061B245A303A10252
:10CAB000280897000000E780208945611763FFFF81
:10CAC000670063B582801763FFFFE70283B201113D
:10CAD0002A8497F0FFFFE780005EAA84228597F002
:10CAE000FFFFE780605F228597F0FFFFE780C05E71
:10CAF000035744008D4763F7E700228597F0FFFF57
:10CB0000E780805D228597F0FFFFE780E05C2800EA
:10CB1000A68597000000E780208305611763FFFF6B
:10CB2000670063AF9797FF1F9387071B9C43D84706
:10CB3000A167FD07631FF7001763FFFFE70263AB01
:10CB4000328597000000E78040F81763FFFF670019
:10CB500083AC82809797FF1F938707189C43D84721
:10CB6000A167E5076315F7081763FFFFE70263A8EE
:10CB700079713285328497F0FFFFE780C0532AC66F
:10CB8000228597F0FFFFE7802055228597F0FFFF71
:10CB9000E78080542310A102228597F0FFFFE780F1
:10CBA000A053520551812311A102228523020102C3
:10CBB00097F0FFFFE7802050A302A102228597F0A3
:10CBC000FFFFE780404F2303A102228597F0FFFF7C
:10CBD000E780604EB245A303A102280897F0FFFF4B
:10CBE000E780807645611763FFFF6700C3A28280FC
:10CBF0009797FF1F9387470E9C43D847A16793875A
:10CC0000E703631FF7001763FFFFE702839E328588
:10CC100097000000E78060EB1763FFFF6700A39FAA
:10CC200082809797FF1F9387270B9C43D847A16764
:10CC300093874704631EF7021763FFFFE702639BB6
:10CC400079713285328497F0FFFFE780C0462AC6AB
:10CC5000228597F0FFFFE7802048B245280897F02B
:10CC6000FFFFE780606E45611763FFFF6700A39ACF
:10CC700082809797FF1F938727069C43D847A16719
:10CC8000938787026310F7041763FFFFE702639639
:10CC900079713285328497F0FFFFE780C0412AC660
:10CCA000228597F0FFFFE7800041B2452300A102F3
:10CCB000280897F0FFFFE780206945611763FFFFB1
:10CCC0006700639582801763FFFFE702839201117B
:10CCD00097F0FFFFE780203EAA85280097F0FFFF2E
:10CCE000E780806605611763FFFF6700C39297972F
:10CCF000FF1F938767FE9C43D847A167D107631F37
:10CD0000F7001763FFFFE702C38E3285970000002C
:10CD1000E780A0FB1763FFFF6700E38F8280979790
:10CD2000FF1F938767FB9C43D847A167C507631F15
:10CD3000F7001763FFFFE702C38B328597000000FF
:10CD4000E780A0F81763FFFF6700E38C8280979766
:10CD5000FF1F938767F89C43D847A167B907631FF4
:10CD6000F7001763FFFFE702C388328597000000D2
:10CD7000E780A0F51763FFFF6700E389828097973C
:10CD8000FF1F938767F59C43D847A167AD07631FD3
:10CD9000F7001763FFFFE702C385328597000000A5
:10CDA000E780A0F21763FFFF6700E3868280979712
:10CDB000FF1F938767F29C43D84789476318F702A0
:10CDC0001763FFFFE702E3820111328532C897F053
:10CDD000FFFFE780402EAA85280097F0FFFFE7803D
:10CDE000A05605611763FFFF6700E3828280979773
:10CDF000FF1F938767EE9C43D847A1678D07631198
:10CE0000F7041753FFFFE702C37E01113285328416
:10CE100097F0FFFFE780202A13066100AA844C00E8
:10CE2000228597300000E780C0232800A68597F070
:10CE3000FFFFE780605105611753FFFF6700A37D87
:10CE400082809797FF1F938767E99C4381CFDC43DC
:10CE500091CB1753FFFFE702C37982971753FFFF68
:10CE60006700637B82801753FFFFE7028378797145
:10CE70003C08AE843ED2A165B7070A002A843ED49E
:10CE800048103C08DD053ED636C432C63AC297D0BB
:10CE9000FFFFE780E02F12474810BA8597F0FFFFA9
:10CEA000E780C01332464810B28597F0FFFFE78055
:10CEB000E014A2464810B68597F0FFFFE780001205
:10CEC000501001478146A685228597D0FFFFE78055
:10CED000805145611753FFFF6700E3731753FFFF4E
:10CEE000E702237101117C000329C501AE843ECA0B
:10CEF000A165B70707002A843ECC48087C00C50519
:10CF00003ECE97D0FFFFE780A0288345D900480890
:10CF100097F0FFFFE780800C500801478146A68507
:10CF2000228597D0FFFFE780004C05611753FFFF74
:10CF30006700636E1753FFFFE702A36B83C795007B
:10CF400093F7F707A384F50097000000E78040F906
:10CF50001753FFFF6700236C1753FFFFE702636956
:10CF600079713C08AE843ED2A165B70709002A84D6
:10CF70003ED448103C08938545043ED632C636C49C
:10CF800097D0FFFFE780C020A2464810B68597F0F3
:10CF9000FFFFE780A00432464810B28597F0FFFFFC
:10CFA000E780C005501001478146A685228597D0AD
:10CFB000FFFFE780404345611753FFFF6700A3650C
:10CFC0001753FFFFE702E36283C7950041112A84EC
:10CFD00093F7F707A384F50032852EC697F0FFFF7D
:10CFE000E780800F85672AC46370F50297700000A0
:10CFF000E78020E92246B24509ED114781462285A6
:10D0000097000000E78060E641011753FFFF6700CB
:10D01000836001478346F501DDB71753FFFFE70241
:10D02000A35B01113C003ECAB7070A003ECC3C009E
:10D030003ECE83C79500AA89328593F7F707A3846C
:10D04000F5002E8497F0FFFFE78000098567637D78
:10D05000F504A165AA8493858504480897D0FFFF4D
:10D06000E7800013268597700000E78080E12A8919
:10D0700029E19145480897F0FFFFE78020F6A68553
:10D08000480897F0FFFFE78060F7CA85480897F0E7
:10D09000FFFFE780A0F4014781465008A2854E8536
:10D0A00097D0FFFFE780203405611753FFFF67002B
:10D0B000E3558145480897F0FFFFE78020F20349D8
:10D0C000090275BF1753FFFFE702035179711C1066
:10D0D0003ECAB7070F003ECC404D1C10AA84AE8953
:10D0E0004808994532C636893ECE97D0FFFFE78083
:10D0F000200A32464808B28597F0FFFFE78000EE2D
:10D10000630C0902A545480897F0FFFFE780C0E6D9
:10D110002546CA8597200100E78020A450080147D2
:10D120008146CE85268597D0FFFFE780C02B4561DD
:10D130001753FFFF6700834D8355C402480897F0DB
:10D14000FFFFE780A0EB0355E402814505C5854755
:10D1500085456301F502C167FD179305F00F630B69
:10D16000F5007D1597700000E780208E930515006F
:10D1700093F5F50F480897F0FFFFE78020E6834519
:10D180000403480897F0FFFFE78040E58345140358
:10D19000480897F0FFFFE78060E4835524034808C0
:10D1A00097F0FFFFE78080E583554403480897F038
:10D1B000FFFFE780A0E49DB71753FFFFE70263433B
:10D1C00083C795008146014693F7F707A384F500CE
:10D1D00097000000E78040EF1753FFFF6700A3436D
:10D1E0001753FFFFE702E34079713E841C103ECAEB
:10D1F0002E89B7070F00A1653ECCFD051C10AA843F
:10D20000480842C03AC23ECE36C432C697D0FFFF6D
:10D21000E78000F832464808B28597F0FFFFE780C4
:10D22000E0DBA2464808B68597F0FFFFE78000DD07
:10D2300012474808BA8597F0FFFFE78020DC0248D4
:10D24000630C08029145480897F0FFFFE780C0D2C1
:10D250001146A28597200100E780209050080147E1
:10D260008146CA85268597D0FFFFE780C0174561B4
:10D270001753FFFF6700233A8945480897F0FFFFDF
:10D28000E78080CF834704002300F5008347140024
:10D29000A300F500E1B71753FFFFE702E33383C7AD
:10D2A000950001112A8A93F7F707A384F5003285C8
:10D2B000AE8432C697F0FFFFE78000E232462A894B
:10D2C000328597F0FFFFE78000DF85676373F9021F
:10D2D000AA894A8597700000E780A0BA2A8419EDD0
:10D2E000114781464A86A685528597000000E7804F
:10D2F000C0B705611753FFFF670043319387E9FF0C
:10D3000093F7F70F0547E366F7FE8347F50195EBC3
:10D310008947E380F9FE8346F401528501474A8636
:10D32000A68597000000E78040B4A167D9074808A8
:10D330003ECC230A010002CE97000000E780A0B097
:10D340004DBF639EE7008947639EF9009307102055
:10D35000231FF50097700000E780C0B76DBF094735
:10D36000E39BE7FA8D47E398F9FA2285977000006E
:10D37000E78080DF9797FF1F938747B59C4399E726
:10D380009797FF1F9387479E9C4399C703D5040037
:10D3900097800000E780A0CE231F040022855DBF98
:10D3A0001753FFFFE702E32401113C003ECAB70711
:10D3B0000B003ECC3C003ECE83C795002A893285C7
:10D3C00093F7F707A384F500AE8497F0FFFFE7809B
:10D3D000A0D093170501C187635AF006A1652A847E
:10D3E0009385E502480897D0FFFFE78060DAA285C1
:10D3F000480897F0FFFFE78060C09797FF1F93876B
:10D40000A7969C43A9EB01449375F40F480897F045
:10D41000FFFFE780A0BC9355844093F5F50F4808C3
:10D4200097F0FFFFE78080BB9355044193F5F50F1C
:10D43000480897F0FFFFE78060BA0147814650082F
:10D44000A6854A8597D0FFFFE780E0F9056117536D
:10D45000FFFF6700431C416585460546A2857D1593
:10D4600097500000E78060BD59DD5105970001002D
:10D47000E780808F130440063344850271B7175349
:10D48000FFFFE70203170111B70706003EC683C777
:10D49000950021642A8993F7F707A384F500AE84E9
:10D4A00028009305A4040AC40AC897D0FFFFE780A8
:10D4B00020CE300001478146A6854A8597D0FFFFE0
:10D4C000E78060F297E0FFFFE78080151304940483
:10D4D000480822CC230A010002CE97000000E78012
:10D4E000809605611753FFFF6700E3121753FFFF94
:10D4F000E702830EC1642A8901449799FF1F93892B
:10D50000699E130A8002FD1497E0FFFFE78080C147
:10D510006347A40001451753FFFF6700230FB307BC
:10D52000440303A7C90ABA9703D707006306970005
:10D5300083D72700638427010504F9B70545E1BFB8
:10D540001753FFFFE70243092A8A2E8999C123A0B6
:10D55000050081498144978AFF1F938A6A78614B4D
:10D5600097E0FFFFE78040C263C7A4004E851753D2
:10D57000FFFF6700A3093384640383A70A003E9476
:10D580008357040099E76304090023208900850478
:10D59000C1BF4146D2851305440097100100E780C2
:10D5A000605975F5A289E5B71753FFFFE702C3027B
:10D5B00039717C083ED4B7070A003ED67C083ED8B5
:10D5C00083C795002A8A328593F7F707A384F5006D
:10D5D0002E8932C697F0FFFFE78000B0856763733E
:10D5E000F5083246AA84328597F0FFFFE780A0ACA9
:10D5F0008547AA8963E8A706A16593858504281055
:10D6000097D0FFFFE780C0B8268597700000E780BD
:10D6100040872A8429ED9145281097F0FFFFE78085
:10D62000E09BA685281097F0FFFFE780209DCE8520
:10D63000281097F0FFFFE780609A0147814630107D
:10D64000CA85528597D0FFFFE780E0D9A16793870D
:10D65000770448183EDC230A010202DE97F0FFFF40
:10D66000E780607E21611753FFFF670023FA814541
:10D67000281097F0FFFFE7806096A685281097F0A6
:10D68000FFFFE780A0979797FF1F938767BC9C4396
:10D6900081CB22856389090097D00000E780402470
:10D6A0008345040271B797D00000E780C022CDBF48
:10D6B0001753FFFFE70243F283C795004111AA8980
:10D6C00093F7F707A384F5003285AE84328A97F08A
:10D6D000FFFFE78060A08567637FF5022A89976076
:10D6E0000000E780007A2A84914631C58347F5011E
:10D6F00005476387E70291C70D476366F704AD46A8
:10D700001DA89305050303250A0041469710010053
:10D71000E78040420DE941011753FFFF670003EF27
:10D720009305950803250A00414697100100E780FC
:10D730006040814669F54A86A6854E8597000000BF
:10D74000E780C081C9BF83250A001305940897703C
:10D750000000E780A02919C1C146F1BF9787FF1FCC
:10D760009387C7769C4399E79787FF1F9387C75F87
:10D770009C4399C7228597800000E780208A69FD35
:10D780008547A30FF400228597B00000E7806084EE
:10D79000228597600000E780E0734E8581464A86C7
:10D7A000A68597F0FFFFE780607BA167938757040A
:10D7B00048003EC42302010002C697F0FFFFE78045
:10D7C000806891BF1753FFFFE70223E083C79500EE
:10D7D0004111AA8993F7F707A384F50032852E89B2
:10D7E000B28A97F0FFFFE780208F85676374F50E9C
:10D7F000AA8497600000E780C0682A840DED416B21
:10D80000014A978BFF1F938BEB6D130C400E7D1B12
:10D8100019A833048A0383A70B0B3E948357C401D2
:10D8200063836705050A97E0FFFFE780A08EE34268
:10D83000AAFE95460DA08357C501639697029305EE
:10D84000050303A50A00414697100100E780802EDA
:10D85000994611E181462686CA854E8597F0FFFFDD
:10D86000E780C06F85A883A50A001305040397709D
:10D870000000E780A017C14679FD2285231E940091
:10D8800097A00000E780E074228597600000E780A1
:10D8900060649797FF1F9387A79B9C43A9C32300AE
:10D8A0000402228597D00000E78040F04E85814633
:10D8B0002686CA8597F0FFFFE780406AA1679387B5
:10D8C000070448003EC42302010002C697F0FFFF90
:10D8D000E780605741011753FFFF670083D28947F4
:10D8E0002300F402E1B7397106DE22DC4AD8800059
:10D8F00052D456D25AD026DA4ED65ECE2E8A3289ED
:10D900002A8B97D0FFFFE780E07D060571054199DE
:10D910008A8A3301A140232224FC231404FC97D0DB
:10D92000FFFFE780207C83479A000605350593F7C3
:10D93000F7072315A4FCA304FA004A85232624FC38
:10D9400097E0FFFFE780407993170501C1876340A7
:10D95000F0025681130104FCF2506254D254425931
:10D96000B259225A925A025BF24B21618280AA84F8
:10D970004A8597E0FFFFE7802076AA894A8597E0ED
:10D98000FFFFE7806075A1659385C5022A891305AD
:10D9900044FC97C0FFFFE780A07F268597C0FFFF6C
:10D9A000E780E073854511C94A86CE8597C0FFFFA1
:10D9B000E780606DAA8B21E98945130544FC97E057
:10D9C000FFFFE780A061A685130544FC97E0FFFFF9
:10D9D000E780C062CE85130544FC97E0FFFFE78037
:10D9E000E061CA85130544FC97E0FFFFE780006112
:10D9F00001478146130644FCD2855A8597D0FFFF24
:10DA0000E780609EB9B78145130544FC97E0FFFFAE
:10DA1000E780C05CA685130544FC97E0FFFFE78024
:10DA2000E05DCE85130544FC97E0FFFFE780005DD5
:10DA3000CA85130544FC97E0FFFFE780205C814422
:10DA400097D0FFFFE780006AE3D4A4FA83A70B0115
:10DA500013971400BA9783D5070099C5130544FCA2
:10DA600097E0FFFFE78080598504D9BF797106D61A
:10DA700022D44AD000184ECE52CC56CA26D25AC80A
:10DA8000AE893289AA8A97D0FFFFE780A065060594
:10DA9000690541990A8A3301A140232A24FC231CE9
:10DAA00004FC97D0FFFFE780E06383C79900060579
:10DAB0002D0593F7F707231DA4FCA384F9004A85DD
:10DAC000232E24FC97E0FFFFE780006193170501F8
:10DAD000C187634FF0005281130104FDB2502254FC
:10DAE00092540259F249624AD24A424B45618280BD
:10DAF000AA844A8597E0FFFFE780005EA1659385D1
:10DB0000A5022A89130544FD97C0FFFFE7804068FE
:10DB1000268597C0FFFFE780805C854509C9CA85D7
:10DB200097C0FFFFE78020592A8B29E1894513051B
:10DB300044FD97E0FFFFE780604AA685130544FD9A
:10DB400097E0FFFFE780804BCA85130544FD97E00F
:10DB5000FFFFE780A04A01478146130644FDCE85BA
:10DB6000568597D0FFFFE7800088B5B7814513053C
:10DB700044FD97E0FFFFE7806046A685130544FD5E
:10DB800097E0FFFFE7808047CA85130544FD97E0D3
:10DB9000FFFFE780A046814497D0FFFFE7808054D5
:10DBA000E3DBA4FA83270B0113971400BA9783D5FC
:10DBB000070099C5130544FD97E0FFFFE780004487
:10DBC0008504D9BF1753FFFFE702A3A2834745008F
:10DBD000404DD5EFFD575DC483469400094763630C
:10DBE000D70A0346B400854663EEC6088306E40000
:10DBF00063CA06085C45F9562390D7009787FF1F34
:10DC000083C7470E99E3A304E4009787FF1F938718
:10DC1000A7159C4381E78947A306F4009787FF1F58
:10DC2000938707639C4381E789472306F4009705A0
:10DC3000000093854506AA841305040197F00000AF
:10DC4000E7802010FD57231AF40281471CDC0148AD
:10DC50009787FF1F23A487089787FF1F938747088D
:10DC6000232E040304C0804397D0FFFFE780C051F8
:10DC700061463306C502814522859750FFFFE78044
:10DC8000409A81473E851753FFFF6700C398FD57B1
:10DC9000D5BF1753FFFFE702C3952A8403554502FA
:10DCA00097600000E780E01D19E5231E040017536C
:10DCB000FFFF670043968357E401F5DB930504FFFC
:10DCC000174501001305C52B97E00000E780E0141D
:10DCD000F9BF1753FFFFE702C3912E89A1654111D8
:10DCE0009385E5032A8436C432C6BE843AC297C0FF
:10DCF000FFFFE780E04912472285BA8597E0FFFFE2
:10DD0000E780C02D32462285B28597E0FFFFE7808D
:10DD1000E02EA2462285B68597E0FFFFE780002E21
:10DD2000630309029145228597E0FFFFE780C02445
:10DD30001146A68597100100E78020E241011753A4
:10DD4000FFFF6700438D8945228597E0FFFFE7804D
:10DD5000A02283C704002300F50083C71400A3009A
:10DD6000F500E9BF1753FFFFE702A38883C79500BB
:10DD7000444D054793F7F707A384F5001C42411172
:10DD800083C707006367F7062E842A89B1C003C7DB
:10DD9000D400630FF7021787FF1F1307E7FC184330
:10DDA00005C3A386F40097A00000E780404A83C71C
:10DDB000D40099E741657D1597400000E780403029
:10DDC00083D72403918B89C797E00000E780C013B5
:10DDD0004A85A28597F0FFFFE7808010A167C10701
:10DDE00048003EC42302010002C697F0FFFFE7800F
:10DDF000800541011753FFFF6700E3811743FFFFD1
:10DE0000E702237F03D745008D47AA8441112E8462
:10DE100032892E8563E3E70297E0FFFFE780C02B9E
:10DE2000AA8523000900268597C0FFFFE780A02868
:10DE300041011743FFFF6700037E97E0FFFFE78084
:10DE4000A0292AC6228597E0FFFFE780E028B24597
:10DE500085472A862300F900268597C0FFFFE780C3
:10DE60008022F9B7397106DE22DC26DA80004ED630
:10DE700052D456D24AD85AD05ECEAE89B284AA8A3B
:10DE800097D0FFFFE780002506051305250241997D
:10DE90000A8A3301A140232224FC231404FC97D0D6
:10DEA000FFFFE780202383C7990006054D0593F700
:10DEB000F7072315A4FCA384F9002685232624FC58
:10DEC00097E0FFFFE780402193170501C18763407A
:10DED000F0025281130104FCF2506254D2544259B0
:10DEE000B259225A925A025BF24B21618280AA8B6C
:10DEF00003AB040097C0FFFFE780601E51E583D7A6
:10DF0000440001498544F11793B71700A301F4FCBD
:10DF1000834734FCA165C9C79385E504130544FC18
:10DF200097C0FFFFE780C026A685130544FC97E055
:10DF3000FFFFE780A00ADE85130544FC97E0FFFFA2
:10DF4000E780C00B834734FC114691E30946DA852C
:10DF5000130544FC97E0FFFFE78060058144630AF6
:10DF60000900416B7D1B97D0FFFFE780A01663CCB3
:10DF7000A40201478146130644FCCE85568597C00E
:10DF8000FFFFE7804046B1B7A685130634FC970033
:10DF90000000E780E0E6933415002A8986048DBFEF
:10DFA0009385C504A5BF8327C90013971400BA97AA
:10DFB00083D5070063886501130544FC97E0FFFFE4
:10DFC000E780C003850445B71743FFFFE702E35F1F
:10DFD00079711C103EC4B7070F003EC61C103EC826
:10DFE00083C79500AA8A328593F7F707A384F500C3
:10DFF000AE89328497E0FFFFE780000E931705019A
:10E00000C187635AF0062A8A228597E0FFFFE780DE
:10E01000A00C2A895285032B040097C0FFFFE780DC
:10E02000000C39ED8357440081440544F11793B740
:10E030001700A303F10083457100DA872287CA869F
:10E040005286280097000000E780E0C8014781461B
:10E050003000CE85568597C0FFFFE780C038A167A6
:10E060009387D70348083ECC230A810026CE97F039
:10E07000FFFFE78040DD45611743FFFF67006358FE
:10E08000A2851306710097000000E78060D7AA847C
:10E09000094455D13544E30055FB4A8597F0FFFF0D
:10E0A000E78000450D4441D9014497D0FFFFE78048
:10E0B0006002634DA400C16B0144FD1B97D0FFFFBC
:10E0C000E7804001634EA4001544B5B7DC44131744
:10E0D0001400BA9783D70700638327030504F1B7B9
:10E0E000D84493171400BA9703D70700631B77012E
:10E0F00023902701268597A00000E78080DB01445C
:10E100001DBF050465BF1743FFFFE702E34C83C74C
:10E11000950041112A8A93F7F707A384F500328509
:10E120002E89328497E0FFFFE78000FB93170501FB
:10E13000C1876353F006AA89228597E0FFFFE78035
:10E14000A0F92311A1004E85832A040097C0FFFF88
:10E15000E780E0F839E58357440085440144F1172E
:10E1600093B71700A300F1000348110003572100E3
:10E17000D6875285CE862686CA8597F0FFFFE78030
:10E180006006A167F10748003EC42302910022C641
:10E1900097F0FFFFE78020CB41011743FFFF6700A7
:10E1A000E346A2851306110097000000E78040C5F2
:10E1B0002A84894455D98357210011678544BA9729
:10E1C000C2071167C1831307F7EFE36FF7F897876B
:10E1D000FF1F9387A7CF9C4381CB85451305210063
:10E1E00097500000E78020758355210022858144E7
:10E1F00097C0FFFFE78040E525D923100500228561
:10E2000097A00000E78040CD85B71743FFFFE702E6
:10E21000C33B83C7950041112A8B93F7F707A3846B
:10E22000F50032852E8A328497E0FFFFE780C0EA4E
:10E2300093170501C1876351F006AA8A228597E0EA
:10E24000FFFFE78060E92A895685832B040097C089
:10E25000FFFFE780C0E831E583574400814405446F
:10E26000F11793B71700A301F10003483100DE87CF
:10E270005A854A87D6862286D28597F0FFFFE780A7
:10E2800060F6A167ED0748003EC42302810026C660
:10E2900097F0FFFFE78020BB41011743FFFF6700B6
:10E2A0004336A2851306310097000000E78040B591
:10E2B000AA8409445DD99167CA97C2071167C183CF
:10E2C0001307F7EF0544E362F7FACA8597C0FFFF2B
:10E2D000E78080D7014451F9814997D0FFFFE7805B
:10E2E00060E063DBA900984893971900BA9703D7B9
:10E2F000070005EF2390270197D0FFFFE78080DE1E
:10E300001544E384A9F6268597A00000E780C0BCE9
:10E310009787FF1F938787BB9C430144B9D74A85E2
:10E3200097500000E780C05889B785097DB717432B
:10E33000FFFFE702632A79713E847C083EC82E8A7B
:10E34000B7071400A1653ECAE5057C08AA8908083C
:10E3500036C4428932C6BA8AC6843ECC97C0FFFF13
:10E36000E78000E3CA85080897E0FFFFE78000C761
:10E3700032460808B28597E0FFFFE78020C8A24632
:10E38000630A09049D45080897E0FFFFE780C0BEC7
:10E390001D4681459740FFFFE780A02863890A0852
:10E3A0009145080897E0FFFFE78000BD1146A6856C
:10E3B00097000100E780607A100801478146D28506
:10E3C0004E8597C0FFFFE780000245611743FFFFBE
:10E3D0006700C323B685080897E0FFFFE78000C207
:10E3E0001C400808D8439355C701858912075183FB
:10E3F000B205D98D97E0FFFFE78040C01C400808B8
:10E4000083C5870097E0FFFFE78040BD1C400808F8
:10E4100083C5A70097E0FFFFE78040BC1C400808C9
:10E4200083C5970097E0FFFFE78040BB85BF894524
:10E43000080897E0FFFFE78020B483C704002300AB
:10E44000F50083C71400A300F500BDB71743FFFF15
:10E45000E702831883C795004111AA8993F7F7074C
:10E46000A384F5003285AE84328497E0FFFFE78015
:10E47000A0C693170501C187635DF0042A89032AAA
:10E48000040097C0FFFFE78080C519E98357440067
:10E490000548F11793B71700A307F100814631A88B
:10E4A0001306F100A28597000000E78060951DC566
:10E4B0001C459DC783D6470001480347F1009307D9
:10E4C0008500D2884A86A6854E8597000000E780A1
:10E4D00040E641011743FFFF6700431309487DBF32
:10E4E0001D486DBF1743FFFFE702030F65715C080E
:10E4F0003EC4B7077B013EC65C083EC883C7950093
:10E500002A8A328593F7F707A384F500AE8997E04E
:10E51000FFFFE78040BA8357E100E1C78945280043
:10E5200097C0FFFFE780C0C68145280097E0FFFF46
:10E53000E780C0AA97C0FFFFE780A0CC9787FF1FA6
:10E54000938707D19C431774FF1F0344A479AA84BF
:10E550003334800099C3136424009787FF1F938787
:10E56000A7809C4399C3136444009787FF1F938738
:10E57000E7959C4399C31364840083D50400280065
:10E58000014997E0FFFFE78060A783D524002800BA
:10E5900097E0FFFFE78080A683D54400280097E03E
:10E5A000FFFFE780A0A597D0FFFFE780A0AE9315FF
:10E5B0000501C181280097E0FFFFE78020A4A28524
:10E5C000280097E0FFFFE78060A39C446360F902A6
:10E5D000014781463000CE85528597C0FFFFE78016
:10E5E00080E059611743FFFF67004302DC441314C6
:10E5F000490028003E9497E0FFFFE780609683473C
:10E6000044000347540089070607BA978607E36A60
:10E61000F5FC835524002800814A97E0FFFFE7803E
:10E62000E09D83454400280097E0FFFFE780009BC2
:10E6300083455400280097E0FFFFE780209A834736
:10E64000440063C9FA00814A8347540063C1FA0257
:10E650000509A5BF1C4413975A002800BA9783D513
:10E660000700850A97E0FFFFE7804099C9BF032BA9
:10E67000C40093975A0028003E9B83552B00850ABF
:10E6800097E0FFFFE780809783550B00280097E015
:10E69000FFFFE780A0964DBF1743FFFFE70263F53A
:10E6A0005C4993E717005CC997A00000E78020B69B
:10E6B0001743FFFF670023F61743FFFFE70263F3EB
:10E6C0002E84814597F0FFFFE780C0E705C583579B
:10E6D0000500FD172310F50009C4835725002310FA
:10E6E000F40097000000E78060FB01451743FFFF3F
:10E6F000670063F231457DD823100400C5BF17437E
:10E70000FFFFE70263ED83C7950041112A8A93F763
:10E71000F707A384F50032852E89328497E0FFFF46
:10E72000E780809B93170501C1876356F006AA898D
:10E73000C145228597E0FFFFE780A0802A8B4E85A8
:10E74000832A040097C0FFFFE780609931E983576F
:10E750004400231101000544F11793B71700A300EB
:10E76000F10081440348110003572100D6875285E8
:10E77000CE862286CA8597F0FFFFE780A0A6A16714
:10E780009387170248003EC42302810026C697E003
:10E79000FFFFE780406B41011743FFFF670003E77E
:10E7A00013061100A28597F0FFFFE7806065AA8439
:10E7B00009E523110100094475B7930521005A8525
:10E7C00097000000E78080EF835721002A84D9DB7F
:10E7D0009777FF1F9387876F9C4381CB85451305F0
:10E7E000210097500000E780001583552100268501
:10E7F000314497C0FFFFE78020852DD52310050009
:10E80000268597900000E780206D0144A1BF174343
:10E81000FFFFE70203DE41112E896C00AA8402C6C5
:10E8200097F0FFFFE78000D20DC1035705000507F1
:10E830002310E50097000000E78040E681473E8511
:10E8400041011743FFFF670003DD3247954765DB52
:10E85000CA85268597300000E780400DC147E34018
:10E8600005FE3244854741462310F40083570900D2
:10E87000A685130544002311F40097000100E780EA
:10E88000C02D228545BF1743FFFFE702E3D483C7AE
:10E8900095004111AA8A93F7F707A384F500328502
:10E8A000AE89328497E0FFFFE7800083931705016C
:10E8B000C1876356F0062A8AC145228597D0FFFF9B
:10E8C000E7802068AA845285032B040097C0FFFFCD
:10E8D000E780E08031E9835744002311010085443B
:10E8E000F11793B71700A300F1000144034811008A
:10E8F00003572100DA875685D2862686CE8597F083
:10E90000FFFFE780208EA1679387070248003EC47F
:10E910002302910022C697E0FFFFE780C052410129
:10E920001743FFFF670083CEA2851306110097F0FF
:10E93000FFFFE780E04C2A8409E5231101008944A8
:10E9400075B726859305210097000000E78060ECED
:10E95000AA8449FD83552100228597B0FFFFE780F7
:10E96000A06E49F5014997C0FFFFE780A077635D7E
:10E97000A900184893171900BA9703D707000DEF9D
:10E98000035721002390E70097C0FFFFE7808075C1
:10E99000630625039777FF1F938747539C4399C7C7
:10E9A0000355210097500000E78080F02285979062
:10E9B0000000E78060521DBF050975B795443DB75B
:10E9C00005C19307F00F630FF500C547630CF50011
:10E9D0009307F5FF05453315F50042054181828017
:10E9E0000145828041657D158280B9E91743FFFFAB
:10E9F000E70223C003450603328497000000E78046
:10EA000060FC9305803EB305B502C205C18181CD8E
:10EA10000357E402854763F8E7001305040197E014
:10EA20000000E78020428357E40241677D17638539
:10EA3000E700FD172317F4021743FFFF6700A3BD8C
:10EA400082801743FFFFE70243B8004283C7950067
:10EA5000444D0349140093F7F707A384F500834757
:10EA60000400220911673369F900A167B347F9006F
:10EA700041112A8BAE8A63ECE70E8347240013070B
:10EA8000C00EB91793F7F70F6373F71003473400FD
:10EA9000C14763EEE70E834744001307E00793C7BF
:10EAA00007086371F70C8349840083477400A20947
:10EAB000B3E9F900856763F7F90A034A64008347FD
:10EAC00054004E85220A336AFA0097500000E7800E
:10EAD000403B61C123962403834B3400137AFA0030
:10EAE000239A3403238874032399440393890401EC
:10EAF000631C090023A60402239804024E8597E0B4
:10EB00000000E78060363DA0034924004A85970055
:10EB10000000E78020EB2397A402834744004E8542
:10EB2000A388F402E38D0BFCE30B09FC97E00000E3
:10EB3000E780202F97900000E78000738146014610
:10EB4000D6855A8597E0FFFFE7800058A167938735
:10EB500097033EC423020100480002C697E0FFFF6E
:10EB6000E780602E41011743FFFF670083A98544BA
:10EB7000A2862686D6855A8597E0FFFFE780C05497
:10EB8000A167938797033EC423029100F1B7BD4468
:10EB9000C5B79144F1BF1743FFFFE702E3A301119B
:10EBA0001C08404D3EC2B7070F003EC41C083EC6BD
:10EBB0002A89AE8997C0FFFFE780A0DA585C1C5C09
:10EBC0006346B70E6394E50063E2A70E3385A74062
:10EBD000B3B7A700B305B7401306803E81469D8DAD
:10EBE00097000100E78080B793140501C180A165FB
:10EBF0009385C503480097B0FFFFE78060598145C2
:10EC0000480097D0FFFFE780603D8355040448002B
:10EC100097D0FFFFE780803E83552404480097D0BB
:10EC2000FFFFE780A03D814589CCC167FD179305B3
:10EC3000F00F6388F400268597500000E780E0E03D
:10EC4000AA85480097D0FFFFE78040390355440468
:10EC5000814501CDC167FD179305F00F6307F500EE
:10EC600097500000E78060DEAA85480097D0FFFF3C
:10EC7000E780C03683456404480097D0FFFFE780F3
:10EC8000E03583457404480097D0FFFFE7800035E6
:10EC9000500001478146CE854A8597B0FFFFE78047
:10ECA000807405611743FFFF67004396814481B775
:10ECB0001743FFFFE702E39383C7950093F7F70736
:10ECC000A384F50097000000E78020ED1743FFFFC5
:10ECD000670063941743FFFFE702039083C7950023
:10ECE0004111404D93F7F707A384F5002A8A328536
:10ECF000B284AE8997D0FFFFE780003E2A8B26853D
:10ED000097D0FFFFE780403D2A89268597D0FFFFF7
:10ED1000E780603A93170B0163CA0702E177CA974D
:10ED2000C207C183116763E3E70293070910C207B3
:10ED3000C1831307B00F637BF70093170901C187E5
:10ED4000AA8A634AF000C54763FE57014101174391
:10ED5000FFFF6700A38B97B0FFFFE780C028E31792
:10ED600025FFD5B763080B02630609028144638956
:10ED70000A02B7077F0023106405231124057CC015
:10ED8000568597000000E780E0C39304803EB304FB
:10ED9000950239A0B7077F00232004047CC081447A
:10EDA0000355240497E00000E780A0A3A1C497C006
:10EDB000FFFFE78000BB269593D7F44133379500DA
:10EDC000AE97BA9708DC5CDCCE85528597000000D0
:10EDD000E780A0DC99E023220404A1679387B703AE
:10EDE00048003EC42302010002C697E0FFFFE7800F
:10EDF0008005A9BF814701481CDC232E0403E9B725
:10EE00001733FFFFE702E37E97C0FFFFE780C037BD
:10EE1000E1473305F502914597500000E78000C5B2
:10EE2000E55711C59777FF1F23ACA7EA81473E85B9
:10EE30001733FFFF6700237E85471777FF1F2303E4
:10EE4000F7EA82801733FFFFE702A37A9777FF1F65
:10EE50009387C7E880433DC0835704046390A706A7
:10EE600083572404639CB7043689B28497C0FFFF9C
:10EE7000E78020AF5C5C63C3B7046395B7001C5C9C
:10EE800063EEA7028347640463F3F400A6872303B9
:10EE9000F4048347740463F39700A687A303F40480
:10EEA0008357440441677D176385E7008507231274
:10EEB000F4043C4481C7CA85268582971733FFFF37
:10EEC000670063759777FF1F938747E19C43014570
:10EED00099C303C5870082801733FFFFE702637180
:10EEE0000111B70707003EC683C79500584D0AC4F5
:10EEF00093F7F7070AC8A384F5002A89AE8411CBDB
:10EF00001C4283C707002304F70097900000E780A6
:10EF10000034216493055402280097B0FFFFE78076
:10EF2000202797000000E78020FAAA85280097D0C4
:10EF3000FFFFE780A00A300001478146A6854A8589
:10EF400097B0FFFFE780204A13044402480822CC10
:10EF5000230A010002CE97E0FFFFE780C0EE0561C3
:10EF60001733FFFF6700236B1733FFFFE702636868
:10EF700001117C003ECAB70707003ECC7C003ECEA4
:10EF800083C795002E84AA8493F7F707A384F5001E
:10EF9000A16593855502480897B0FFFFE780401FA1
:10EFA00097000000E78040F2AA85480897D0FFFF4D
:10EFB000E780C002500801478146A285268597B0A8
:10EFC000FFFFE780404205611733FFFF6700A3643E
:10EFD0009777FF1F938787D09C43094599C303C543
:10EFE000970082809777FF1F938747CF9C430945FF
:10EFF00099C303C5D70082809777FF1F938707CEF9
:10F000009C43014599C303C5A70082801733FFFFC6
:10F01000E702835C0111B70708003EC683C795006D
:10F02000404D0AC493F7F7070AC8A384F5002A895C
:10F03000AE8429C41442854703C7060063E0E70A8B
:10F0400083479400094681496380C702B307F740AC
:10F05000A304E400B339F00083C716002305F400CD
:10F0600097900000E780A01E03572403058B19C763
:10F070006386090097D00000E78000E921649305CA
:10F080008402280097B0FFFFE780801097000000FF
:10F09000E78040F4AA85280097D0FFFFE78000F4BE
:10F0A00097000000E78080F5AA85280097D0FFFF31
:10F0B000E780C0F2014781463000A6854A8597B0B7
:10F0C000FFFFE780403213047402480822CC230A71
:10F0D000010002CE97E0FFFFE780E0D6056117331D
:10F0E000FFFF6700A3521733FFFFE70283500111B0
:10F0F0007C003ECAB70708003ECC7C003ECE83C7EA
:10F1000095002E84AA8493F7F707A384F500A165E0
:10F1100093858502480897B0FFFFE7806007970056
:10F120000000E78020EBAA85480897D0FFFFE78022
:10F13000E0EA97000000E78060ECAA85480897D0D5
:10F14000FFFFE780A0E9500801478146A285268598
:10F1500097B0FFFFE780202905611733FFFF6700A5
:10F16000834B9777FF1F938767B79C43014599C3EC
:10F1700003C5B70082801733FFFFE7028347011101
:10F18000B70707003EC683C79500404D0AC493F7F2
:10F19000F7070AC8A384F5002A89AE8405C81C4273
:10F1A000054783C707006368F7060347B400630F8A
:10F1B000F700A305F40097900000E780400983471B
:10F1C000B400B9CF97D0FFFFE78040BE216493051C
:10F1D000B400280097B0FFFFE78080FB9700000095
:10F1E000E78060F8AA85280097D0FFFFE78000DF5E
:10F1F000014781463000A6854A8597B0FFFFE7802A
:10F20000801E2904480822CC230A010002CE97E080
:10F21000FFFFE78040C305611733FFFF6700A33F8F
:10F2200097D0FFFFE78020BF55B71733FFFFE702F6
:10F23000433C01117C003ECAB70707003ECC7C006E
:10F240003ECE83C795002E84AA8493F7F707A38444
:10F25000F500A165AD05480897B0FFFFE78040F3D2
:10F2600097000000E78020F0AA85480897D0FFFFAC
:10F27000E780C0D6500801478146A285268597B011
:10F28000FFFFE780401605611733FFFF6700A338D3
:10F290009777FF1F938787A49C43094599C303C5AC
:10F2A000C70082801733FFFFE702A33401117C00FF
:10F2B000AE843ECAA165B70707002A843ECCD105BB
:10F2C0007C0048083ECE97B0FFFFE78060EC9700D7
:10F2D0000000E78020FCAA85480897D0FFFFE78060
:10F2E000E0CF500801478146A685228597B0FFFFF1
:10F2F000E780600F05611733FFFF6700C3311733E5
:10F30000FFFFE702032F83C7950093F7F707A38456
:10F31000F50097000000E78020F91733FFFF670032
:10F32000832F1733FFFFE702232B83C795000329A1
:10F33000C501411193F7F707A384F5001C4283C967
:10F340000700854763E637079777FF1F938747F0E6
:10F350009C432E84AA8485CF97000000E78080F329
:10F3600089476306F502630409028347C900638085
:10F3700037032306390197900000E78040ED83575B
:10F380002903898B89C797D00000E780E0B72685DD
:10F39000A28597000000E78020F1A167CD07480013
:10F3A0003EC42302010002C697E0FFFFE780A0A948
:10F3B00041011733FFFF670063259777FF1F93878E
:10F3C000E7919C431D4599C303C5E700828017332D
:10F3D000FFFFE70203220111B70707003EC683C7FC
:10F3E0009500584D0AC493F7F7070AC8A384F5009F
:10F3F0002A89AE8415C71C4283C7070093968701EC
:10F40000E18663C4060685466381D7068346E70026
:10F410006388F6002307F70097900000E78020E359
:10F4200021649305E400280097B0FFFFE78040D6F1
:10F4300097000000E780A0F8AA85280097D0FFFF7A
:10F44000E780C0B9014781463000A6854A8597B05C
:10F45000FFFFE78040F93504480822CC230A010069
:10F4600002CE97E0FFFFE780009E05611733FFFFA4
:10F470006700631A1733FFFFE702A31701117C002F
:10F480003ECAB70707003ECC7C003ECE83C795003E
:10F490002E84AA8493F7F707A384F500A165B90524
:10F4A000480897B0FFFFE780A0CE97000000E780F4
:10F4B00000F1AA85480897D0FFFFE78020B25008E6
:10F4C00001478146A285268597B0FFFFE780A0F11E
:10F4D00005611733FFFF670003141733FFFFE702CF
:10F4E000A30FAA8401441769FF1F1309697FE1492B
:10F4F00097C0FFFFE78040C96344A400014519A8F5
:10F5000033053403832709003E958357250063970D
:10F51000970011051733FFFF6700430F0504C9BFAC
:10F52000032E8500630A0E121773FF1F1303039A3D
:10F53000032303006315030029436390061203238A
:10F540004E01631503001D43639907101733FFFF36
:10F55000E702A307C689428A3E89BA8AB684328BFB
:10F56000AE8B2A84B5E103554E0019E501431A8597
:10F570001733FFFF6700E308A167A98F116763FBDB
:10F58000E70097000000E78080F5814597F0FFFFD6
:10F59000E780C0120844B70700E05841F98F1845CA
:10F5A0005CC1B707001FF98F1CC55C4991C7610595
:10F5B00097E00000E780408BE38A09FA2285979064
:10F5C0000000E78060C65DB7328597C00000E78025
:10F5D00040430D4349DD1C44116703D54700A16733
:10F5E000A98F63FBE70097000000E78040EF8145AB
:10F5F00097F0FFFFE780800C0323840093164B01F4
:10F60000D1828347B300035663008588FD8BA30531
:10F61000F300FD777D8E558EFD76FD16B204F18EDA
:10F6200083274301C58E231273012313D3002304C0
:10F63000530123052301A3044301BDDF228597B0B5
:10F64000FFFFE78020CDAA850844B5D1610597D09A
:10F650000000E780207F8DB71D431A858280173315
:10F66000FFFFE70263F70569AA84AE89328A014485
:10F67000FD5A7D1997C0FFFFE780C0A56347A4002E
:10F6800001451733FFFF670063F8D8449317140050
:10F69000BA9703D70700631F370323905701630707
:10F6A0000A00268597900000E780A0809C449DC3B7
:10F6B00083D76700B3F72701639E3701D2880148DB
:10F6C0008147014781460146814526859700000014
:10F6D000E78040E5050479BF1733FFFFE702C3EF7A
:10F6E00079711C103EC4B7070F003EC61C103EC8FF
:10F6F00083C79500AA8A328593F7F707A384F5009C
:10F700002E89328497D0FFFFE780009D9317050173
:10F71000C187635AF006AA89228597D0FFFFE78048
:10F72000A09B2A8A4E85032B040097B0FFFFE78039
:10F73000009B39ED8357440081440544F11793B78A
:10F740001700A303F10083457100DA872287D28670
:10F750004E86280097E0FFFFE780E057014781468B
:10F760003000CA85568597B0FFFFE780C0C7A16704
:10F770009387F70348083ECC230A810026CE97D012
:10F78000FFFFE780406C45611733FFFF670003E828
:10F79000A2851306710097E0FFFFE7806066AA84E8
:10F7A000094455D1528597E0FFFFE78060D40D44AE
:10F7B00059D90546D285268597000000E78060EA82
:10F7C0002A8451B71733FFFFE702A3E283550700EE
:10F7D0000346270041112A842E8532C62EC497E0A5
:10F7E000FFFFE780E0D001C93246A245228597009D
:10F7F0000000E78000E741011733FFFF6700A3E146
:10F800001733FFFFE70263DC83C795004111AA8A23
:10F8100093F7F707A384F5003285AE89328497D039
:10F82000FFFFE780608B93170501C1876357F00ADC
:10F83000C1452A8A228597C0FFFFE78080702A8D04
:10F84000228597D0FFFFE78020892A89228597D0DB
:10F85000FFFFE7804086930705F893F7F70F13073C
:10F86000E007AA8B637BF706228597D0FFFFE7802E
:10F8700080842A8C228597D0FFFFE780C083AA8CE2
:10F880005285032B040097B0FFFFE780408539E9DC
:10F8900083574400231101008144F11793B71700E7
:10F8A000A300F1000544034711008356210093870C
:10F8B00084005685DA8822885286CE8597F0FFFF2D
:10F8C000E78020A7A167E90748003EC42302810022
:10F8D00026C697D0FFFFE780005741011733FFFF8F
:10F8E000670023D213061100A28597E0FFFFE7808F
:10F8F0002051AA8409E52311010009446DB793053D
:10F9000021006A8597F0FFFFE780A0F02A8441FD7F
:10F91000835521009356C90013164901854866880E
:10F92000E2875E87858A5182268597000000E780FE
:10F9300060BF2A848DBF1733FFFFE70203C983C767
:10F94000950041112A8B93F7F707A384F5003285C0
:10F95000AE89328497C0FFFFE780007893170501D6
:10F96000C1876352F00A2A8A228597C0FFFFE78089
:10F97000A076AA8A228597C0FFFFE780E0752A89D2
:10F98000228597C0FFFFE7800073930705F893F780
:10F99000F70F1307E0072A8C6377F706228597C0D5
:10F9A000FFFFE7804071AA8C228597C0FFFFE780A8
:10F9B00080702A8D5285832B040097A0FFFFE7807B
:10F9C000007239E58357440085440144F11793B729
:10F9D0001700A301F10003473100930784005A8503
:10F9E000DE882688D6865286CE8597F0FFFFE78090
:10F9F00040948D4748003EC42302910022C697D010
:10FA0000FFFFE780404441011733FFFF670063BFFA
:10FA1000A2851306310097E0FFFFE780603E2A844D
:10FA2000894455D99356C9001316490185486A88F7
:10FA3000E6876287858A5182D68597000000E78035
:10FA400060AEAA8449BF1733FFFFE702E3B82A89F3
:10FA500081440144617A916A176BFF1F130B0B47B6
:10FA600097B0FFFFE780006863C7A40022851733C3
:10FA7000FFFF6700A3B98327090093991400CE976D
:10FA800003D50700330745014207418363645703E9
:10FA900005C103270B0019C785453E859740000027
:10FAA000E78060E9832709000504CE9723900700CB
:10FAB00085047DB797000000E78060A283270900D6
:10FAC0000504CE972390070065D5814597F0FFFF89
:10FAD000E780C0BEF1BF1733FFFFE702E3AF83C784
:10FAE000950041112A8A93F7F707A384F500328520
:10FAF0002E89328497C0FFFFE780005E93170501CF
:10FB0000C187635AF004AA89832A040097A0FFFFE3
:10FB1000E780E05C31E58357440085440144F117F8
:10FB200093B71700A301F10003483100D68752852F
:10FB30000147CE862686CA8597D0FFFFE780806A78
:10FB4000A167F50748003EC42302910022C697D062
:10FB5000FFFFE780402F41011733FFFF670003AB32
:10FB6000A2851306310097E0FFFFE78060292A8411
:10FB700089445DD99767FF1F938747359C4381CFA1
:10FB8000044997B0FFFFE780E055AA852685974096
:10FB90000000E78040DA1305040197000000E780C9
:10FBA000C0EA228597800000E78000338144ADBF22
:10FBB0001733FFFFE70263A183C795004111AA8AAB
:10FBC00093F7F707A384F5003285AE8932842311B9
:10FBD000010097C0FFFFE780205093170501C18700
:10FBE0006354F0062A8AC145228597C0FFFFE7804B
:10FBF0004035AA8B5285032B040097A0FFFFE780B6
:10FC0000004E21E98357440085440144F11793B71E
:10FC10001700A300F1000348110003572100DA8701
:10FC20005685D2862686CE8597D0FFFFE780805BFB
:10FC3000A1679387270248003EC42302910022C691
:10FC400097D0FFFFE780202041011733FFFF6700B7
:10FC5000439BA2851306110097E0FFFFE780401A3F
:10FC60002A8489444DD99767FF1F93872726984395
:10FC70003E8901CF044997B0FFFFE780A046AA85DF
:10FC8000268597400000E78000CB1305040197000C
:10FC90000000E78080DB97B0FFFFE780A044954439
:10FCA0003DD9930521005E8597F0FFFFE78060B6A0
:10FCB000AA8435F11C480357210022852390E700D0
:10FCC00097800000E780402183270900A9D70355CA
:10FCD000210097400000E780A0BD35BF1733FFFF2C
:10FCE000E702A38E83C795004111AA8A93F7F7070D
:10FCF000A384F5003285AE89328497C0FFFFE78088
:10FD0000A03D93170501C1876351F0062A8A228519
:10FD100097C0FFFFE780403C2A895285032B0400EF
:10FD200097A0FFFFE780A03B31E58357440085445F
:10FD30000144F11793B71700A301F1000348310004
:10FD4000DA8756854A87D2862686CE8597D0FFFFEA
:10FD5000E7804049A167F90748003EC423029100AB
:10FD600022C697D0FFFFE780000E41011733FFFF47
:10FD700067002389A2851306310097E0FFFFE78023
:10FD800020082A8489445DD99167CA97C207116700
:10FD9000C1831307F7EF8544E362F7FA9767FF1F04
:10FDA0009387C7129843BE8B01CF044997B0FFFFDA
:10FDB000E7804033AA85268597400000E780A0B7FA
:10FDC0001305040197000000E78020C897B0FFFFEB
:10FDD000E780403195443DD11C48228581442390E1
:10FDE000270197800000E780200F83A70B00B9D779
:10FDF0004A8597400000E780A0AB89B71723FFFF33
:10FE0000E702237F2A844105B28497000000E7803F
:10FE1000C0C311C5228597800000E780E00B8146B2
:10FE20000146A685228597800000E780C04E1C4CC5
:10FE300089C7DC4799C3228582971723FFFF670094
:10FE4000837D9767FF1F938767E99C43014599C3AB
:10FE50001385070182809767FF1F938727E88843F0
:10FE600082801723FFFFE702C3789317C600DD8D5A
:10FE7000C2054111C1812A8432C697C0FFFFE780C5
:10FE8000E0173246228511829375F60F97C0FFFF67
:10FE9000E780C01441011723FFFF6700C3771723D2
:10FEA000FFFFE702637379713C083ED2B7070C008D
:10FEB0003ED43C083ED683C79500AE842A8993F78A
:10FEC000F707A384F500A16593853504481097A032
:10FED000FFFFE780E02BC165FD150144176AFF1F96
:10FEE000130A4A00930A400EAE892E8B2EC697B095
:10FEF000FFFFE78020224205931704014181C1835F
:10FF0000B24563E9A702C167FD176387F500481092
:10FF100097C0FFFFE780800E501001478146A685FD
:10FF20004A8597A0FFFFE780004C45611723FFFF3C
:10FF30006700C36D3307540383270A0BBA9703D6B0
:10FF4000C701630A3601638A350148109700000033
:10FF5000E78060F1DA85050451BFB285EDBF172354
:10FF6000FFFFE702836679717C083EC8B70711007E
:10FF70003ECA7C083ECC83C79500AA89328593F798
:10FF8000F707A384F5002E8997C0FFFFE780C01410
:10FF900085676378F504A165AA848905080897A098
:10FFA000FFFFE780E01E268597400000E78060EDB8
:10FFB000133415000A04A285080897C0FFFFE780E4
:10FFC000E001A685080897C0FFFFE780200325CC45
:10FFD000014781461008CA854E8597A0FFFFE7803C
:10FFE000804045611723FFFF6700A361B3075403F7
:10FFF0000327CA0ABA9703D70700631C970003D6E2
:020000040001F9
:10000000270063806505080897000000E780A0E5E9
:10001000DE8505042EC697B0FFFFE780A0104205DD
:10002000931704014181C183B245E3E1A7FCC16795
:10003000FD17E38FF5F8080897C0FFFFE78000FC85
:1000400041BFB285F9B7C165FD150144176AFF1FAD
:10005000130A4AE9930A80022E8BAE8B65BF1723E1
:10006000FFFFE70203591841834717008346070043
:10007000A207D58FD207D1832390F50083472700AD
:10008000034717008D45A207D98F91832310F600EF
:1000900097C0FFFFE780A0E91723FFFF6700A35782
:1000A0001723FFFFE7024353C16401441769FF1F91
:1000B000130949E393098002FD1497B0FFFFE7801D
:1000C00060066347A40001451723FFFF6700035440
:1000D000330534038327C90A3E9583570500E3851A
:1000E00097FE0504D9BF1723FFFFE702E34E2A8AD4
:1000F000AE89B284B68A97400000E78080D819E5BF
:1001000091473E851723FFFF670043502A894E859C
:1001100097C00000E780E08E2A84638E0A048D4732
:100120006DD103570500C547E31D47FD0347F9019E
:100130008546AD47E317D7FC8347450081CF41464D
:10014000A6855D0597F00000E780C09E814755D9E0
:10015000AD4745BF130965012302E500CA85268521
:1001600097100000E780606231C1A547E38B0AF871
:100170002302040079B705C183570500E39247F9CC
:100180004146A685190597F00000E780A09A8147AF
:100190002DD99947BDB74E8597000000E78080F0C4
:1001A0002A84954739DD130955004DBF4146A68580
:1001B00023104401231134011305190097F00000A6
:1001C000E780A099228597800000E780A0EA814718
:1001D0000DBF1723FFFFE702C34179717C003ECCBE
:1001E000B7070A003ECE7C003ED083C79500B2849C
:1001F0002E8493F7F707A384F5001306A1002A893C
:100200002C00268597000000E780A0E5A16528085E
:100210008D0597A0FFFFE780A0F790408355A100D0
:1002200003558100854697000000E78000ECAA8412
:10023000AA85280897C0FFFFE78040DA0356A1008F
:1002400083558100280897000000E780C0C130086E
:1002500001478146A2854A8597A0FFFFE780A01845
:10026000854748103ED42302910202D697D0FFFF63
:10027000E78060BD45611723FFFF6700C33917237F
:10028000FFFFE702033779717C003ECCB7070A0015
:100290003ECE7C003ED083C79500B2842E8493F777
:1002A000F707A384F5001306A1002A892C002685F0
:1002B00097000000E780E0DAA16528088D0597A087
:1002C000FFFFE780E0EC90408355A10003558100DB
:1002D000814697000000E78040E1AA84AA852808AB
:1002E00097C0FFFFE78080CF0356A10083558100B0
:1002F000280897000000E78000B7300801478146D2
:10030000A2854A8597A0FFFFE780E00D48102302F1
:10031000910202D402D697D0FFFFE780C0B24561B8
:100320001723FFFF6700232F1723FFFFE702632C2C
:1003300097000000E78060DB1723FFFF6700A32D15
:100340009767FF1F9387C799884382801723FFFF12
:10035000E702232A835725004111AE842A8423070C
:10036000B10017F5FFFF130525466C002316F100B9
:1003700097A0FFFFE780204991C422859780000065
:10038000E780E0D6FD572310F400130620028145D4
:10039000130554009720FFFFE780A0284101172391
:1003A000FFFF670043271723FFFFE702E32279716E
:1003B0007C003ECCB7070A003ECE7C003ED083C70F
:1003C0009500AA89AE8493F7F7073285A384F500D8
:1003D0001306A1002C0097000000E78080C8035599
:1003E0008100114497400000E780A0A915C503557E
:1003F000A100014497B00000E780A06011CD035731
:1004000005008357810045446318F7008545970030
:100410000000E780E0F301442169930539002808D2
:1004200097A0FFFFE780C0D6A285280897C0FFFFEE
:10043000E780C0BA0356A1008355810028089700C1
:100440000000E78040A2300801478146A6854E851E
:1004500097A0FFFFE78020F948104AD423028102C9
:1004600002D697D0FFFFE780009E45611723FFFF6C
:100470006700C3191723FFFFE70203169767FF1FE3
:100480009387C7852A8488432E8915C5035745035A
:100490008357C4016311F7022326050223180502BE
:1004A000410597D00000E780209C630609009780F3
:1004B0000000E78060DB81449769FF1F938989A270
:1004C000130A800297B0FFFFE780C0C563C4A4048D
:1004D0009767FF1F938747899C4399C70355C401BA
:1004E00097200000E780C0BD630709002285978040
:1004F0000000E780C0A01306400E814522859720AA
:10050000FFFFE7800012FD57231EF4001723FFFFB3
:100510006700C30F3385440383A7C90A3E95035779
:1005200005008357C4016317F700CA8597000000D0
:10053000E78000E2850479B71723FFFFE702C309CC
:1005400083C795004111AA8993F7F707A384F500A3
:100550003285AE8497C0FFFFE78000B88567637877
:10056000F5042A8997400000E780A091014401CD5D
:1005700083D7040031446388270185459700000034
:10058000E78080EF01444E85A2864A86A68597D0F3
:10059000FFFFE780A09CA1679387170448003EC433
:1005A0002302810002C697D0FFFFE780C089410186
:1005B0001723FFFF670083051723FFFFE702C3012F
:1005C0009757FF1F93878771804329C4014597C0C0
:1005D0000000E780002181470148C1641CDC232E14
:1005E0000403232004041769FF1F1309A98F014482
:1005F0009309400EFD1497B0FFFFE780A0B1634F51
:10060000A400814517F5FFFF1305857F97A0FFFF25
:10061000E780601F1723FFFF670043FF33053403A4
:100620008327090B3E958357C5016387970085454E
:1006300097000000E78040E4050475BF935705016B
:1006400013D78700A380F50093170501C183A18309
:100650002380E5002381F500A381A5008280172374
:10066000FFFFE70203F92300050083C71500A3007D
:10067000F50083C725002301F50083C73500A301DA
:10068000F50083C745002302F50083C75500A30288
:10069000F50083C7650093059500A30305002303B8
:1006A000F50023040500328597000000E78040F93B
:1006B0001723FFFF670023F61723FFFFE702C3F1AD
:1006C0004111E9540DCD85CD93F9C5FF2E842A89BA
:1006D000AA84338AA900B7EA040063189A020D8835
:1006E000854411CCB7E704009C5F82972AC6228616
:1006F0006C003305390197E00000E780004626854D
:1007000041011723FFFF670063F083A78A03910469
:10071000829793170501C183A183A38EF4FE93579B
:100720000501238FF4FEA183238EA4FEA38FF4FE84
:100730006DB763E6D5021723FFFFE70283EBB287AD
:1007400041113686BE8536C697E00000E780E0405E
:10075000B246410136851723FFFF6700C3EB814690
:1007600036858280838705001387F5003D05FD8768
:1007700093F77708834607007D158606B58FA3009B
:10078000F5006307B7007D17834717009D83DDB72A
:1007900082801723FFFFE702C3E5B7E7040083A7C2
:1007A000070932872A863A85829713351500172361
:1007B000FFFF670043E615C181478DC11723FFFF87
:1007C000E70223E3414697E00000E78000398547D0
:1007D0003E851723FFFF670003E481473E85828043
:1007E0001DCD1723FFFFE702C3E0414681452A8460
:1007F0009720FFFFE780E0E24146814513050403AF
:100800009720FFFFE780E0E10147C167232204044E
:1008100038C87CC805451723FFFF6700C3DF0145C3
:10082000828081473DCDB5CD1723FFFFE70263DC12
:10083000B2842E891306800581452A849720FFFF04
:10084000E78020DECA8524C4268597000000E78063
:10085000C0F64146814522859720FFFFE78060DC96
:100860003044A285228597000000E780C0F29304FF
:100870000401A285268597000000E780E0EEA685AA
:100880001305040297000000E78000EE2285970020
:100890000000E78020F585473E851723FFFF6700AE
:1008A00083D73E8582801723FFFFE702E3D2411101
:1008B000E9540DCD85CD93F9C5FF2E842A89AA84EC
:1008C000338AA900B7EA0400639844030D88814481
:1008D00011CCB7E704009C5F82972AC622866C0081
:1008E0003305390197E00000E78020272685410184
:1008F0001723FFFF670083D183A78A0391048297A0
:1009000093170501C183A183A38EF4FE93570501BC
:10091000238FF4FEA183238EA4FEA38FF4FE6DB774
:1009200065CD1723FFFFE70223CBB28411E605450F
:100930001723FFFF670083CD2A842E890145EDD957
:100940003C487848B3E6E700E5D69386F7FFB3B7AF
:10095000F6007D17032A4404BA9734C87CC863059F
:100960000A06C14913050A03B38949412295637DEB
:100970003601B2862E86A68597000000E780A0DBB0
:100980007C40BE9464C065B7CE862E86CE85970027
:100990000000E78040DAC114D2944E992322040467
:1009A000A2879306040103C7070003C60703850750
:1009B000318FA38FE7FEE398F6FE3044A2852285AF
:1009C00097000000E78020DD2699C1493306994051
:1009D00063EC9900A9DCA686A6851305040397009D
:1009E0000000E78040D579BF8147B306F4003307A4
:1009F000F6000347070083C5060085072D8F238077
:100A0000E600E39437FF3044A2852285970000007A
:100A1000E78060D8C1145DBF014582800DC11723F6
:100A2000FFFFE70203BD1306800581459720FFFF06
:100A3000E78020BF05451723FFFF6700C3BD0145C1
:100A40008280814749C5C1C51723FFFFE70263BA0A
:100A5000FC4141462E84AA846399C704138605018C
:100A6000A2878146C14503C7070003C50703850761
:100A7000298F3305D600034505008506298FA38FEE
:100A8000E7FEE392B6FE3044A2852685970000007B
:100A9000E78060D0228597000000E78060F88547F6
:100AA0003E851723FFFF670003B7138507031D8EDD
:100AB000814522959720FFFFE780A0B67C40130771
:100AC00000F813060402A2972388E70251BF3E856F
:100AD00082801723FFFFE702C3B16D712E84B284B9
:100AE000AA8590102800368997000000E780A0D3DF
:100AF00009EDD55725A050400C4028009700000074
:100B0000E78040E27DD5FD142104F5F42C004A85F0
:100B100097000000E78020F3814761DD3E85516149
:100B20001723FFFF670023AF1723FFFFE70263AC24
:100B300041112EC432C62C00054697000000E78004
:100B400080F941011723FFFF6700E3AC1723FFFF84
:100B5000E70223AA01112A842EC602C802CA02CCC7
:100B600002CE97E00000E780402BB2462A86A2859D
:100B7000080897000000E78060FB1375F50F05611A
:100B80001723FFFF670023A91723FFFFE70263A6D0
:100B90007971B2872A8421462308B1001305110117
:100BA000BE853AC436C697E00000E78000FBB24637
:100BB00093059101368597000000E78060A82285A3
:100BC000141035460C0897000000E78020F62A84B0
:100BD000224701E921460C103A8597E00000E780A2
:100BE000C0F7228545611723FFFF6700C3A21723C3
:100BF000FFFFE70203A07171AE84AA850A853284E3
:100C000097000000E78060BB11C90A86A68522858F
:100C100097000000E78020B8814711E1C5473E8575
:100C20004D611723FFFF6700039F1723FFFFE702B4
:100C300043991D712A8AB289BE84354685471305BA
:100C400011012E8CB68A3A8BC28C468D2308F10096
:100C500097E00000E78060F010100C085285231F19
:100C6000010097000000E780C0F82A843DEDA1470D
:100C70006313FD089307900591E0E5473546E2854B
:100C80001305110113990A012308F10013590901F1
:100C900097E00000E78060EC1357890093978A0083
:100CA000D98F90080C085285231FF100970000008F
:100CB000E78020F42A8415E9A1E49387FA00918360
:100CC0001379F9003EC6631309004149668B8144DC
:100CD000C14B854DB247639F970C6A868C00338564
:100CE0005C0197E00000E78040E72285256117233B
:100CF000FFFF6700C39093079004C9F0A547BDBFED
:100D0000834701050947C14B2308F10083471105BB
:100D1000A58FA308F10093872400814463E1FB04BD
:100D2000014714083386E6008C08B386E400BA95C0
:100D3000DA9683C6060083C505000507AD8E23003D
:100D4000D600E390E7FE4147639CE70490080C0857
:100D5000528597000000E780C0E925D181A0B30645
:100D60009B00BA871008B305F60090083E9603C5AD
:100D700006000346060085078506298E2380C500E8
:100D8000E39277FF998F90080C085285BE949700E4
:100D90000000E78000E68947014749D12A84B1B7BE
:100DA00090083E96034606001408BE962380C600AF
:100DB000850759BFB2478504638797148147180890
:100DC000B306F70098083E973386F90003470700FB
:100DD000034606008507318F2380E600E39177FF05
:100DE00090080C08528597000000E78080E05DF5D0
:100DF0003546E285130511012308B10197E0000093
:100E0000E780A0D513970401418393978400218341
:100E1000D98F10180C085285231FF100970000008D
:100E2000E78020DD25FD814710183387F9003E96C5
:100E30000347070003460600B306FB008507318F12
:100E40002380E600E39277FF65A81808B306F70051
:100E500098083E973386F9000347070003460600CB
:100E60008507318F2380E600E3E127FFCA87639E71
:100E7000770990080C08528597000000E78060D73A
:100E800011FD81479800B306F700900818103E97AF
:100E90003E9603470700034606008507318F2380EF
:100EA000E600E39177FF3546E2851305110123083B
:100EB000B10197E00000E78040CA13970401418325
:100EC000939784002183D98F10180C085285231F13
:100ED000F10097000000E780C0D1E31105EC8147E5
:100EE00010183387F9003E960347070003460600B3
:100EF000B306FB008507318F2380E600E3E227FF7E
:100F0000C109410BC1BB814785B79408BE9683C612
:100F1000060018083E972300D700850789BF638025
:100F200006321713FFFFE702C36959712A84BE898D
:100F3000B28B85473546130511022E8B468C4289AC
:100F4000BA8A368A2300F10297E00000E780E0C009
:100F500010180C1022852317010297000000E7806B
:100F600040C963180512A147631FFC06930790054B
:100F700063930900E5473546DA851305110293149A
:100F80000A012300F102C18097E00000E780E0BC85
:100F900093178A0013D78400D98F90080C102285EC
:100FA0002317F10297000000E780A0C47DE163925F
:100FB00009049307FA00BD88918391E0C144C207F8
:100FC000C183DE8C814A3EC6414DB24763E2FA0ED0
:100FD0006286B3854B01881097E00000E78080B5FA
:100FE0004DC93D557DA093079004E39609F8A547A8
:100FF00059B7834701050947C14C2300F1028347D4
:101000001105B3C7F900A300F102938729008149B4
:1010100063E1FC04814618103306D7008C0833873F
:10102000D900B69556970347070083C50500850686
:101030002D8F2300E600E390D7FE41476390E7063B
:1010400090080C10228597000000E78080BA35D107
:1010500089A0B3863A01BA871010B305F60090084C
:101060003E9603C506000346060085078506298EC1
:101070002380C500E39297FF3387EC4090080C1063
:101080002285BA9997000000E780A0B689470147FA
:1010900041D165611713FFFF6700635690083E96C4
:1010A000034606001410BE962380C600850779B754
:1010B000B247850A93990A01939D8A0093D9090141
:1010C0006391570F85473546DA85130511022300D2
:1010D000F10293D9890097E00000E78000A8B3ED02
:1010E0003D0190000C1022852317B10397000000EA
:1010F000E78020B059FD8147A68963EA97062686D6
:101100000C084A8597E00000E78020A58147181069
:10111000B306F700100898083E973E96034707006D
:10112000034606008507318F2380E600E3E197FE42
:10113000639FA90590080C10228597000000E780A6
:1011400040AB21F981479810B306F70090081818B2
:101150003E973E9603470700034606008507318FFA
:101160002380E600E391A7FF4109C10CB9BD18082F
:101170009000B306F7003E963387FC000347070054
:10118000034606008507318F2380E600B5B798082F
:101190004E97034707001C10CE972380E700850970
:1011A00041BF85473546DA85130511022300F10258
:1011B00093D9890097E00000E780209AB3ED3D01C4
:1011C00090000C1022852317B10397000000E780E0
:1011D00040A2E31005EC814718089000B306F70021
:1011E0003E963387FC000347070003460600850749
:1011F000318F2380E600E391A7FF41460C084A8522
:1012000097E00000E780609581471810B306F7006B
:10121000100898083E973E960347070003460600CD
:101220008507318F2380E600E391A7FF90080C101B
:10123000228597000000E780C09B1DD599BD7D5594
:1012400082801713FFFFE702C33A01112A842E851B
:1012500093055100328902C002C202C402C693043F
:10126000740097F0FFFFE780A03D1D46A68513059B
:10127000910097E00000E780408E10088A854A853B
:1012800097000000E780E09619ED93071400180816
:1012900083C607000346070085070507B18EA38FA5
:1012A000D7FEE397F4FE05611713FFFF6700A3362F
:1012B0001713FFFFE70243322E848C414111AA89A4
:1012C000838715003289914463D30700A14497575F
:1012D000FF1F9387E7F79C43A1C7C1CA8D4723101F
:1012E000F10083C725004A852301F10083C735003B
:1012F000A301F10083C745002302F10083C7550015
:10130000A302F10083C7650093059100A3030100C8
:101310002303F1002304010097F0FFFFE780403230
:101320000C404A860A8597F0FFFFE7808033032848
:10133000040083564400A6881D0881470147E5162E
:1013400042868A854E8597000000E780408E2A8974
:1013500019E5A685228597B0FFFFE780E0C14A85A1
:1013600041011713FFFF6700632A4A860A8597F039
:10137000FFFFE780002F6DB71713FFFFE702C325BC
:101380002E848C414111AA898387150032899144AA
:1013900063D30700A1449757FF1F938767EB9C43D4
:1013A000A1C7C1C68D472310F10083C725004A8518
:1013B0002301F10083C73500A301F10083C7450075
:1013C0002302F10083C75500A302F10083C7650023
:1013D00093059100A30301002303F10023040100FE
:1013E00097F0FFFFE780C0250C404A860A8597F0FA
:1013F000FFFFE780002783564400032804008A8506
:10140000858EC2061D08C1822312D400A68881479A
:101410000147E51642864E8597000000E78060B0E0
:1014200041011713FFFF6700631E4A860A8597F084
:10143000FFFFE78000234DBF1713FFFFE702631B89
:10144000B335B000011185052A891315F6013365FE
:1014500015012308B1009305110136843AC632C044
:101460003EC442C297F0FFFFE780801DA2471248AA
:10147000425593D68700230BF100930591019357B2
:101480008800A30AD100A30BF100230C010197F0FF
:10149000FFFFE780E01A3247024603280400B33713
:1014A000E000835644009207914411C2A1444A854A
:1014B000A68842860C0897F0FFFFE78040772A89CC
:1014C00019E5A685228597B0FFFFE780E0AA4A8547
:1014D00005611713FFFF670003141713FFFFE702EF
:1014E000A30F01113EC68647B335B0008505AA8912
:1014F0001315F6015D8D2308B100930511013684A3
:101500003A89B28442C446C297F0FFFFE780401395
:1015100022489248164593578800A30AF100930584
:10152000910193D78800230B0101A30BF100230C39
:10153000110197F0FFFFE780A0103247104083565B
:101540004400B337E000920703280900914891C096
:10155000A1480C084E8597000000E780809CAA8473
:1015600001E9835544004A8597B0FFFFE780C0A09A
:10157000268505611713FFFF67004309AA959307A6
:10158000F00F17170100130727A36317B50013C542
:10159000F7FF1375F50F828005058346F5FFB58FBC
:1015A000BA9783C70700D5B703574500144193077F
:1015B000F00F17160100130626A036974207418345
:1015C000139506014181631BE500AD8FB29703C5FA
:1015D0000700130515F3133515008280850603C532
:1015E000F6FFA98FB29783C70700D9BF1713FFFF74
:1015F000E7022300B28736842E86BA86AA853E8506
:10160000BA8497F0FFFFE7806052634F05002285A0
:1016100097E00000E78060802A86A686A28526855E
:1016200097F0FFFFE78080501713FFFF6700A3FECE
:101630001713FFFFE70243FA5D712A8BAE8A171575
:1016400001001305E5942C00B284368ABA893E89DC
:1016500097F0FFFFE780C04F2A845DE134104146D8
:10166000DA85280097F0FFFFE780404C2A8449E99B
:101670008547A303F100A6C2930771002408BEC4E6
:10168000A68685470D462C18281002DC02DED6C03F
:10169000BEC697F0FFFFE78000442A8435E1834708
:1016A0007102A6860D4693F7F7072300FA00C1479B
:1016B0003EDE2C188947281026DCA303F10097F0A2
:1016C000FFFFE78040412A8405ED4146A6854E850F
:1016D00097D00000E78060488D47A6860D462C18FD
:1016E0002810A303F10097F0FFFFE780C03E2A8493
:1016F00001E94146A6854A8597D00000E780E0458C
:10170000228561611713FFFF670043F01713FFFF86
:10171000E70223EE97F70000938707EF984383C70C
:10172000470079712A89AE84171501001305C58613
:101730000C083AC42306F10097F0FFFFE780404110
:101740002A8405ED14104146CA85080897F0FFFF6A
:10175000E780C03D2A8415E1140815462C000810C6
:1017600097F0FFFFE780803C2A8401E921462C089E
:10177000268597D00000E780403E228545611713FB
:10178000FFFF670043E91713FFFFE70283E697F7C0
:101790000000938767E79C477971AA842E84170518
:1017A00001001305E57F0C083EC697F0FFFFE780B8
:1017B000203A0DE914104146A685080897F0FFFF6E
:1017C000E780C03605E1140811466C00081097F058
:1017D000FFFFE780A03519E58347F10193F7F70391
:1017E0002300F40045611713FFFF6700C3E21713DE
:1017F000FFFFE70203E03688A14881470147E5463D
:1018000097F0FFFFE780A0421713FFFF6700A3E0F8
:101810001713FFFFE702E3DD3688A1488147014740
:10182000E54697F0FFFFE780C06F1713FFFF6700E3
:1018300083DE1713FFFFE702C3DB01112A842E8525
:101840000C0832C697F0FFFFE780803009ED324781
:1018500097060100938646731008C14522859700BC
:101860000000E780E0D805611713FFFF6700A3DAE7
:101870001713FFFFE702E3D74111C1472EC032C45F
:101880008A8509463EC23EC697F0FFFFE780A02446
:1018900041011713FFFF670003D81713FFFFE7028B
:1018A00043D54111AE8613061009AA850A8502C0E8
:1018B00002C202C402C697F0FFFFE7802027410161
:1018C0001713FFFF670023D51713FFFFE70263D24B
:1018D0003287970601009386266D2E8693050002B7
:1018E00097000000E780C0D01713FFFF6700A3D266
:1018F0001713FFFFE702E3CF7971C1472ACC2ED03F
:1019000032D42C080D4628003ECE3ED23ED602C42C
:1019100002C602C802CA97F0FFFFE780C01B4561FC
:101920001713FFFF670023CF1713FFFFE70263CCF6
:101930000111AA842E8417050100130565678A85A5
:1019400097F0FFFFE780C02015E514084146A68503
:101950000A8597F0FFFFE780601D09ED8347E101ED
:101960000347F101A207D98FCA07C9836177D98FCD
:101970002310F40005611713FFFF6700C3C915CDDD
:101980001713FFFFE702E3C69747FF1F9387C73987
:1019900090439745FF1F938565391745FF1F130532
:1019A000A53497D00000E78000C51745FF1F130539
:1019B000A5331713FFFF670003C61745FF1F130565
:1019C000A53282808DCD1713FFFFE70283C29747B0
:1019D000FF1F93876735944301112E840A8697452C
:1019E000FF1F9385A53497D00000E78040C60A8585
:1019F0000294014505611713FFFF6700C3C17D55C0
:101A000082801713FFFFE702C3BE97D00000E78074
:101A100080D19747FF1F23A9A73017F5FFFF1305B4
:101A2000E5C997B00000E780C0741713FFFF670097
:101A300083BE1747FF1F130767319317150008432D
:101A40003E95FD572310F50082801713FFFFE70234
:101A500043BA2A84084009E51713FFFF6700A3BBB8
:101A60001C4158401CC06313E5005CC0834755000F
:101A700023200500F99BA302F50097A0FFFFE78054
:101A8000207CC9BF1713FFFFE70203B59747FF1F6D
:101A90009387C72D98432A8411CB8347350093F74A
:101AA000070289C7035505008945029713054401BC
:101AB00097B00000E780403B835504000355E400E5
:101AC00097300000E780A00C485819C597A0FFFF89
:101AD000E7800077232A040213058403970000009F
:101AE000E780E0F68144B1499790FFFFE780C06D41
:101AF00063CBA402834734002320040493F727FC1C
:101B0000A301F40000489790FFFFE780E06C1316F4
:101B10001500814522859710FFFFE78080B01713DD
:101B2000FFFF6700A3AEB3873403032904038504D2
:101B30003E994A8597000000E78060F12304090080
:101B400065B78347350093F7070299E30145828023
:101B50008357E500E39CB7FEC167FD176316F600E7
:101B600005458280054599A81713FFFFE70263A882
:101B700093170601C187B2842A8401496359F00290
:101B8000835705009DCB01456367F600034584003C
:101B90003E953325A6001375F50F0DA01C481317AD
:101BA0001900BA9783D70700E38E97FA0509979033
:101BB000FFFFE7806062E343A9FE01451713FFFFC3
:101BC000670063A51713FFFFE70203A1AE89AA848C
:101BD0009790FFFFE78000562A8497D0FFFFE780A9
:101BE000A02EAA860147130684019705000093855D
:101BF00085E41745FF1F1305A5159790FFFFE780A4
:101C0000801C2A8925C98C441304C50022859E05A1
:101C100093F5050897A0FFFFE780403CCC40838701
:101C20007400E18163DD070493E50508228597A030
:101C3000FFFFE780A03A0D4693854400228597A0D8
:101C4000FFFFE780C03683D50400228597A0FFFF01
:101C5000E780E03D83D52400228597A0FFFFE78041
:101C6000003D03D6490083A50900228597A0FFFF08
:101C7000E780E0334A851713FFFF6700239993F548
:101C8000F5076DB71713FFFFE702A39601112A842A
:101C9000328532C697A0FFFFE780E0279780FFFFDD
:101CA000E7806034835704001747FF1F130787231B
:101CB0003246231BF100930700F8A30DF1001C47E7
:101CC0001843231AA1008983858BB307F740B28597
:101CD00048083ECE231C0100230D010097000000A0
:101CE000E78080EE05611713FFFF6700C3921713AB
:101CF000FFFFE702638E004101453DC49304C40029
:101D000026853289AE8997A0FFFFE780C0249545DC
:101D10002A8A2685035B040197A0FFFFE780202124
:101D2000268597A0FFFFE780603E8D45AA8A26851D
:101D300097A0FFFFE780A01F268597A0FFFFE78001
:101D4000E03C5C48420A135A0A01D2975CC423184B
:101D50006401814763983A0146054D813306254168
:101D60009337160013F5F70F1713FFFF6700038A69
:101D70001713FFFFE702638589692A8BAE8B328ACE
:101D8000B68A81440144314CFD199790FFFFE780EA
:101D9000A04363CDA4009790FFFFE780E045018D4D
:101DA00033B5AA001713FFFF6700A38533898403A7
:101DB00083270B003E9963170A0083478900850437
:101DC0003E94E1B703560A00DE854A8533F6C90022
:101DD00097000000E780E0F16DD10545E1B71713EA
:101DE000FFFFE702038101112A847C000355E5000F
:101DF0003ECAB70707003ECC7C003ECE97200000CD
:101E0000E78020082A898545480897A0FFFFE780DA
:101E100020399945480897A0FFFFE780E015AA847C
:101E20004A8597200000E780A0082380A4009747F8
:101E3000FF1F9387270B9C434166130606F093967A
:101E4000870113D78701558F93D68700F18E558F61
:101E5000A207B706FF00F58FD98F11462C00138516
:101E600014003EC497D00000E78020CF5008A38222
:101E700004008945228597000000E780E0E019C949
:101E8000AA851305840397A0FFFFE780E0313C405B
:101E900085073CC005611703FFFF6700C377170381
:101EA000FFFFE70203759790FFFFE780E0342A8485
:101EB00005049790FFFFE78020333305A402F14724
:101EC00091453305F50297200000E78020BA11E51F
:101ED00065551703FFFF670003749747FF1F23AF84
:101EE000A7E69790FFFFE78020312A8405049790AA
:101EF000FFFFE780602F3305A40289450605972080
:101F00000000E780A0B669D59747FF1F23A0A7E48C
:101F10009790FFFFE780402E2A8405049790FFFFEB
:101F2000E780802C3304A4029747FF1F239287E2A7
:101F30009790FFFFE780402C2A849790FFFFE7806F
:101F4000A02A930714003385A7029747FF1F239207
:101F5000A7E097070100938767C91747FF1F232D45
:101F6000F7DE0145BDB71703FFFFE702E366AA846A
:101F70002E8901449749FF1F9389C9F6130A8006E9
:101F80009790FFFFE78040266347A40001451703B1
:101F9000FFFF6700A3673305440383A709024A864E
:101FA000A6853E9597000000E780E0B919E1050499
:101FB000C1BF0545E9BF1703FFFFE7020361AA8A16
:101FC0002E8BB28B368C3A8A814401448149974CDE
:101FD000FF1F938C2CF1130D80069790FFFFE78075
:101FE000A02063C9A40011E085494E851703FFFFB7
:101FF000670023613389A40383A70C025E86D6851C
:102000003E994A8597000000E780E0B31DC1979094
:10201000FFFFE780601E0544636D4501D28662863E
:10202000DA851305090397000000E780A0D411C1E9
:10203000854985045DB71703FFFFE702E359C164D3
:1020400041112A8901449749FF1F9389A9E9130A7D
:102050008006FD1436C632C42EC29790FFFFE7807B
:10206000A01892452246B2466348A40001454101AA
:102070001703FFFF670083593305440383A7090251
:102080003E9509C683473500C18B9DC791C68347DE
:10209000350093F707028DC3630699008357E50067
:1020A000639C27010357050001CB63E7E5008347E5
:1020B0008500BA97E3CDF5FA050469BF1703FFFF62
:1020C000E7028351C1642A8901449749FF1F93891C
:1020D00069E1130A8006FD149790FFFFE780C010A6
:1020E0006346A4001703FFFF670043523305440310
:1020F00083A709023E958357E500638A970063042E
:1021000099006396270197000000E780E097050497
:10211000E1B71703FFFFE702C34A89692A8AAE8A3B
:10212000328BB68B8144174CFF1F130CACDB930C26
:102130008006314DFD199790FFFFE780E00A63C6E6
:10214000A4001703FFFF6700834B338994038327A1
:102150000C028355CA015A863E994A8597000000B1
:10216000E780609E31C1814D15A03384AD03832784
:10217000090303D60B00D68533F6C9003E942285A9
:1021800097000000E780E0B609E9850D9790FFFF12
:10219000E7808003E3CBADFC01A822859700000017
:1021A000E780E08A23040400850471B71703FFFF6A
:1021B000E702A3414169AA8A014A174BFF1F130B8B
:1021C0006BD27D19C14B054C9790FFFFE780C00192
:1021D0006346AA001703FFFF6700A3429309800626
:1021E000B3073A0383290B02BE9983D7E900638EB4
:1021F000270163842A01639A570103A4890301E834
:102200004E8597000000E780C0BD050A75BF835763
:102210000401639977099304C400268597A0FFFF02
:10222000E78060D385452A8D2685835C040197A0CD
:10223000FFFFE780C0CF268597A0FFFFE780A0E7DC
:1022400062056185635905048D45268597A0FFFFCA
:10225000E780E0CD8945268597A0FFFFE78020CD68
:102260008945268597A0FFFFE78060CC85452685B8
:1022700097A0FFFFE780E0CC83470500094793F76D
:10228000F707639AE7009945268597A0FFFFE78047
:1022900040CBA30285014848337D2D0123189401CA
:1022A0006A9548C40040A1BF1703FFFFE7026334EB
:1022B00037E404008327041D82979747FF1F83C7D5
:1022C00067AF1715FF1F13052577A300F5008327B8
:1022D000441C82978327841C81461306F00F814596
:1022E000014582971703FFFF6700E3321747FF1F7F
:1022F0001307479C18439745FF1F83C5A5AB974716
:10230000FF1F9387A7A98346870303469703639715
:10231000D5009747FF1F238FC7A8828083C58701F9
:102320000347A7036317B6009747FF1F2384E7A857
:10233000828003C687016317C7009747FF1F238B5F
:10234000D7A6828083C68701130750026319D7007E
:10235000930760021747FF1F230EF7A4828083C6EE
:102360008701130660026315D60093077002DDB77C
:1023700083C7870155BF9747FF1F938727A2D44B79
:102380000947638DE6081703FFFFE7028326174915
:10239000FF1F1309E99D3E8483470900918B9DCF60
:1023A000B7E4040083A7041D829783A7441C174544
:1023B000FF1F1305659C829783A7841C81461746DF
:1023C000FF1F0346669D81450145829721C58347CE
:1023D0000900ED9B1747FF1F230CF7988347040064
:1023E00093F7F70F85CB91471747FF1F2322F79CE1
:1023F00097000000E78080EB97000000E78040EF47
:10240000B7E70400BC4F414691451745FF1F034500
:10241000659982971703FFFF6700E31F8280170308
:10242000FFFFE702031D8D4741116306F504C54711
:102430006308F50285476310F5029747FF1F238D58
:10244000A796B7E70400BC4B930500101745FF1F84
:1024500003454595829741011703FFFF6700A31BC2
:1024600085471747FF1F2309F794B7E70400BC4BC4
:1024700093050020E1BF9747FF1F93872792D44B16
:102480001147638DE600B7E7040083A7071D829715
:10249000B7E70400BC4B930500044DBF054917473F
:1024A000FF1F2327279183C7070032C62E8493F787
:1024B000F70FD5D3B7E4040083A7041D7D1413746C
:1024C000F40F8297E37689FCB245994703C615005D
:1024D000E3F0C7FCFC4409061745FF1F1305058EF2
:1024E0008297BC48930500081745FF1F0345858B5D
:1024F000829779BF1703FFFFE702A30F1747FF1F5C
:102500001307C7894047184B1C409746FF1F23AD50
:10251000F6886316E4001747FF1F2329F788130581
:1025200084FE9790FFFFE78000AA035564FF978021
:10253000FFFFE780807297A0FFFFE78060D017035E
:10254000FFFF6700430D1703FFFFE702830A97476A
:10255000FF1F9387A784D84BDC4789C797000000EB
:10256000E78080F985471747FF1F2323F7849737B4
:10257000FF1F938727749C43930500021745FF1F95
:102580000345458283C787031747FF1F2304F7824C
:10259000B7E70400BC4B82971703FFFF6700A30750
:1025A0009737FF1F23AEA77E82801703FFFFE70246
:1025B000A30237E404007C4CA1451735FF1F0345F7
:1025C000657E82977C48A1451735FF1F0345857DB1
:1025D0009734FF1F9384847C8297DC4489EB9700B7
:1025E0000000E78080D91703FFFF6700230203D5AF
:1025F00067FF9780FFFFE7804066AA896DD1D848C2
:1026000091476310F7027C4C91451735FF1F034536
:10261000657982977C4891451735FF1F034585787A
:10262000829703A9490103D409018947B7E9040046
:102630001737FF1F232EF77683A7091D21044204B5
:10264000829783C784011715FF1F1305E53E6119A3
:102650001717FF1FA302F73E83A7491C41808297EB
:102660009737FF1F238A077483A7C91C8146094631
:102670009375F40F4A85829711E99747FF1F83C727
:10268000E78389C79710FF1FE78000A8B7E704001A
:10269000BC4F2146A1451735FF1F0345A570829702
:1026A00099B71703FFFFE702C3F493F70520011161
:1026B0002E8481CF97000000E78020E91345042095
:1026C00005611703FFFF670003F593F70510A9CF16
:1026D0009734FF1F9384846CDC4897000000E780E8
:1026E00020C11737FF1F1307E75C184383C7840116
:1026F000034787036318F700DC4489C7970000008D
:10270000E78080DF85471737FF1F2323F76AB7E786
:102710000400BC4B930500021735FF1F0345856875
:1027200082971345041069BF93F70508BDC7973713
:10273000FF1F83C7B768E91719469735FF1F9385B1
:1027400005681305D10093F4F70F1739FF1F0349EC
:10275000E96697C00000E780404093970401C18379
:102760001737FF1F13070766231DF100231CF10015
:102770009737FF1F938787623ACE3ACAD84323061A
:10278000010009CBDC439315890154080D46E1850E
:10279000680082971345040825B793F72500A5C361
:1027A0009737FF1F9387875FD84B89476306F702E8
:1027B0009737FF1F83C7C75B13F7270011EF918B74
:1027C00099CFB7E70400BC4F1306000A89451735B7
:1027D000FF1F0345255D829713452400D5B5973724
:1027E000FF1F9387274D9C4383C787031737FF1F1E
:1027F0002302F75C97000000E78060DBF1BF93F7EE
:10280000050281CB97000000E78060DA13450402DF
:1028100045BD93F7850081CB97000000E780E0D2AB
:102820001345840071BD93F7150081CB970000001C
:10283000E780A0B41345140061B593F7450081CB40
:1028400097000000E78060B31345440095BD93F7FF
:10285000050495C39737FF1F83C7475491CB970053
:102860000000E780A0A491471737FF1F2322F754E9
:1028700013450404B1B593F705010145E38207E46C
:102880009737FF1F93878751D84B91476310F70401
:102890009737FF1F9387C74D9C4313D72700858326
:1028A000D98F858B91E7B7E7040083A7071D82972F
:1028B000B7E70400FC4F91451735FF1F0345854ED0
:1028C000829785471737FF1F2324F74E13450401CE
:1028D000C5BB9737FF1F2383A75E82801703FFFFC7
:1028E000E70223D19737FF1F23A0074C9737FF1F1D
:1028F00023AE074A85471734FF1F1304A43B17373D
:10290000FF1F2327F74A1C4083C787031737FF1F82
:102910002302F74A9790FFFFE780409329C5971756
:10292000FF1F23AFA7101C40170500001305A5D7F4
:1029300083C787031737FF1F230EF7461717FF1F9D
:10294000A30CF70E9737FF1FA38A0744B7E70400CD
:1029500083A7070882979737FF1F2385A74417038C
:10296000FFFF670043CBB7C7898E938767ED1717C3
:10297000FF1F2327F70C45BF1737FF1F03470742E9
:10298000795555E79737FF1F9387474103C71700CE
:1029900005079736FF1FA383E64003C717008D4640
:1029A0003377D7029736FF1FA38AE63E83C6170008
:1029B0001737FF1F13070730184393F6F60FA9EEDA
:1029C000834787031737FF1F2306F73E85471737CF
:1029D000FF1F2305F73C9737FF1F938767399C43F9
:1029E0000145998BA9E71703FFFFE70283C037E48E
:1029F00004007C48C1451735FF1F0345A53A82975F
:102A00003C4885451735FF1F0345C5398297014569
:102A10001703FFFF670023C083C717008546639530
:102A2000F6008347970379BF8347A70361BF82807E
:102A30009737FF1F83C78736A1CF1703FFFFE70232
:102A400043BB37E404009737FF1F238907347C48D2
:102A500085451735FF1F0345E53482977C4C91452A
:102A60001735FF1F0345053482977C48914517357C
:102A7000FF1F0345253382973C48C1451735FF1F8B
:102A800003454532829701451703FFFF6700A3B84E
:102A9000795582801703FFFFE702A3B52A84035507
:102AA00065FF9780FFFFE780401B9737FF1F9387E5
:102AB000E72ED847BE841DEF9790FFFFE780807711
:102AC0009C48232004009DEB9737FF1F23A0872EEF
:102AD0009737FF1F23AA872CB7E70400BC4B894513
:102AE0001735FF1F0345052C829701451703FFFF8C
:102AF000670063B2630A8700184375BF80C39737C6
:102B0000FF1F23A5872AC9BF7955CDB71703FFFF3C
:102B1000E70223AE9737FF1F9387873A8843232620
:102B2000050023240500510597A00000E780C0336D
:102B30001703FFFF670023AE1703FFFFE70263AB36
:102B40001734FF1F1304C4371C40411199CF9C4711
:102B50002302B5002AC61CC197000000E78040FB95
:102B60001C409C4B99C33245829741011703FFFFDC
:102B7000670063AA1703FFFFE702A3A74111444DB3
:102B8000328532842EC69790FFFFE780C0522AC458
:102B900022859790FFFFE780205403A84400630C30
:102BA0000800B245835744001840224683D54500AB
:102BB000AA862685029841011703FFFF6700A3A597
:102BC0001703FFFFE702E3A2404D1DC808C09705A9
:102BD0000000938565031305440197A00000E7807A
:102BE00040169737FF1F9387A72D9C43014589E720
:102BF0009737FF1F23A6872C1703FFFF6700A3A1AA
